:020000040800F2
:10000000000001208946000805280008072800088C
:10001000092800080B2800080D280008000000002F
:100020000000000000000000000000000F28000891
:1000300011280008000000001328000815280008F7
:10004000D9460008D946000819280008D9460008F2
:10005000D9460008D9460008252800082B280008A2
:10006000D9460008D94600085D280008D94600088E
:1000700031280008332800083528000841280008E6
:100080004D28000859280008D9460008D94600081C
:1000900000000000D94600085F280008D946000883
:1000A000D9460008D9460008D9460008D9460008B4
:1000B000D9460008D9460008D9460008D9460008A4
:1000C000D9460008D9460008D9460008D946000894
:1000D000D946000869280008D9460008D946000812
:1000E000D94600086528000875280008D946000888
:1000F000D94600080000000000000000D9460008B2
:10010000D9460008D946000881280008D9460008C9
:10011000D9460008D9460008D9460008D946000843
:10012000D9460008D9460008D9460008D946000833
:08013000D9460008D946000879
:1001380010B5054C237833B9044B13B10448AFF319
:1001480000800123237010BDCC08002000000000AF
:100158000844010808B5034B1BB103490348AFF332
:10016800008008BD00000000D008002008440108F5
:1001780014214160704714207047406A704700009E
:10018800790100087F01000883010008990100082F
:1001980010B5044604F1100000F05CFCC4F8F80047
:1001A8000148C4F87C0110BD88010008F8B5E6B024
:1001B80004460D4616461F460A4906A800F0CAFE20
:1001C80070996F9A05910492009733466E996D9ACB
:1001D800039102922A466C990191214600F060F839
:1001E80067B0F0BD94010008F8B5E6B004460D46C6
:1001F80016461F46094906A800F0ACFE6F996E9A8C
:100208000491039200976D996C9A0291019233467A
:100218002A46214600F087F867B0F0BD940100082F
:1002280038B500281CBF01680029184A23D1184B8B
:100238001C684FF6F0710C404CF24025AC421FBFD1
:100248001B6819404CF27024A14212D1114D296843
:1002580079B911490B68C3F30B03B3F58A6F1FBF54
:100268000968C1F30B0140F28343994204BF01219D
:10027800117028B905E0094B994204BF012111709A
:100288004068BDE8324001F09FBE00BFE80800208A
:1002980000ED00E0002004E00010005C000037489A
:1002A8002DE9F04104460D46216816464A681F4666
:1002B80090478046B8F5403F2ED122680A99936846
:1002C800204698478046B8F5403F25D12368089ACC
:1002D8000799D3F80CC02046E0478046B8F5403F60
:1002E8001AD12368069A39461F692046B8478046BE
:1002F800B8F5403F10D1236829465D69324620464B
:10030800A8478046B8F5403F06D123680B9A09995B
:100318009D692046A847804621680A68204690477C
:100328004046BDE8F0812DE9F04104460D462168BC
:1003380016464A681F4690478046B8F5403F2ED17A
:1003480022680A999368204698478046B8F5403F46
:1003580025D12368089A0799D3F80CC02046E047AE
:100368008046B8F5403F1AD12368069A39461F6976
:100378002046B8478046B8F5403F10D12368294643
:100388005D6932462046A8478046B8F5403F06D109
:1003980023680999DD6900222046A847804621681C
:1003A8000A68204690474046BDE8F0814FF4403047
:1003B80070470000F0B50C4685B0114600281A4673
:1003C8001CBF0568002D0B4B11D082B104B971B95F
:1003D8000D9860B10F9E0E9F0A9B0290049603979A
:1003E8000B980C9E009001962046A8470346184695
:1003F80005B0F0BD020003002DE9F04F0646D0B06D
:100408000868F56DD6F860E0726EB76EF36E00BAE4
:1004180000906C46486800BA60600DF14008886832
:1004280000BAA060C86800BAE060086900BA206134
:10043800486900BA6061886900BAA061C86900BAF1
:10044800E061086A00BA2062486A00BA6062886A95
:1004580000BAA062C86A00BAE062086B00BA2063FA
:10046800486B00BA6063886B00BAA063C86B00BAB7
:10047800E063402058F80C1C58F820CC58F838ACE9
:100488008CEA010158F840CC8AEA01018CEA01099A
:100498004FEAF979401E48F8049BEBD187EA02003D
:1004A80000EA0E00784010EBF5610098DFF824C4EC
:1004B80041186144C81882EABE032B404FEAF06134
:1004C80053405918636859186144CF194FEAB50366
:1004D80083EABE01014081EABE0111EBF765A1681C
:1004E8004D196544A91883EAB0023A404FEAF1650C
:1004F8005A405519E26855194FEAB70282EAB0071F
:1005080065440F4005EBBE0E97EAB00717EBFE6592
:1005180027697D194FEAB10782EA0701654401EAB4
:100528000E01EB18514011EBF36561694D194FEA63
:10053800BE0187EA010E65440EEA030E15EBB00012
:100548008EEA070E0EEBF065D4F818E075446544A2
:10055800AA1881EAB30505404FEAF26E4D40AE4451
:10056800E569AE44E64477444FEAB00080EAB30E4A
:100578000EEA020E8EEAB30E0EEBF765D4F820E011
:1005880075446544691880EAB2053D404FEAF16E4A
:100598004540AE44656AAE44E6440EEBB3034FEA09
:1005A800B70787EAB20E0EEA010E8EEAB20E0EEB1C
:1005B800F365D4F828E075446544281887EAB1053E
:1005C8001D404FEAF06E7D40AE44E56AAE44E64415
:1005D8000EEBB2024FEAB30383EAB10E0EEA000E45
:1005E8008EEAB10E0EEBF265D4F830E0754465443E
:1005F800EF1983EAB00515404FEAF76E5D40AE4447
:10060800656BAE44E6440EEBB1014FEAB20282EAF2
:10061800B00E0EEA070E8EEAB00E0EEBF165D4F8B6
:1006280038E075446544EB1882EAB7050D404FEA97
:10063800F36E5540AE44E56BAE44E6440EEBB000B5
:100648004FEAB10181EAB70E0EEA030E8EEAB70E41
:100658000EEBF065D4F840E07544654481EAB30ECA
:10066800AA180EEA000E4FEAF2658EEA010E7544EA
:10067800DDF844E04FEAB000754480EAB30E654403
:100688000EEA020E15EBB7078EEAB30E0EEBF7650E
:10069800DDF848E04FEAB202754480EA020E65448C
:1006A8000EEA070E69188EEA000E0EEBF165DDF80A
:1006B8004CE07544654405EBB3034FEAB70E1427C5
:1006C8000DF1500CDFF810528EEA010B82EA0B0B89
:1006D8000BEBF36A5CF804BBDA44AA44504483EA9F
:1006E800B10B4FEAF06A8EEA0B0BDA445CF804BBF4
:1006F800DA44AA44524480EAB30B4FEAF26A8BEA1E
:10070800B10BDA445CF804BBDA444FEAB000AA44FF
:1007180080EA020BD6448BEAB30B0BEBFE6A5CF85B
:1007280004BBDA444FEAB202AA4482EA0E0B0AEB8F
:10073800B10180EA0B0B0BEBF16A5CF804BBDA44FD
:100748007F1DAA44282F0AEBB3034FEABE0EBBD382
:100758003C2F61D3502F4DD204EB870CC7F15407BF
:100768005E4CA7FB04A504465D4FA8088EEA010A63
:1007780082EA0A0A5CF804BB0AEBF3655D447D195A
:100788002C1983EAB10A4FEAF4658EEA0A0A55443D
:100798005CF804AB5CF804BB55447D19AA1884EADC
:1007A800B30A4FEAF2658AEAB10A55445D444FEA52
:1007B800B4047D1984EA020AAE448AEAB30A0AEB51
:1007C800FE655CF804AB55444FEAB2027D1982EA33
:1007D8000E0A15EBB10184EA0A0A5CF804BB0AEBBD
:1007E800F1655D447D1915EBB303401E4FEABE0E5B
:1007F800BCD12046F46D1B19F365336EC9183166F8
:10080800716E71447166B36ED218B266F16E40189B
:10081800F06650B0BDE8F08F4EEA010B0EEA010A0F
:100828000BEA020B4BEA0A0A0AEBF36554F827A015
:10083800DFF8B0C0554443EAB10B654403EAB10A96
:100848000BEA0E0B28184BEA0A0A7F1C0AEBF06524
:1008580054F827A0554440EAB30B654400EAB30AAC
:100868000BEAB10BAA184BEA0A0A7F1C0AEBF265DD
:1008780054F827A055444FEAB00040EA020B6544FB
:1008880000EA020A0BEAB30BAE444BEA0A0A7F1CE1
:100898000AEBFE6554F827A055444FEAB20242EA33
:1008A8000E0B654402EA0E0A0BEA000B15EBB101C8
:1008B8004BEA0A0A7F1C0AEBF16554F827A0554455
:1008C8007F1C65443C2F05EBB3034FEABE0EA3D350
:1008D80040E700BF9979825AA1EBD96ECDCCCCCC38
:1008E800D6C162CADCBC1B8F00B581B00168074A5B
:1008F800914200D110B9064801B000BD7C2113F027
:10090800E9FC4FF4003001B000BD00BFFC0900084D
:10091800030002002DE9F0410B4A92E8F85188B033
:10092800694681E8F8510268084B9A4200D118B923
:10093800074808B0BDE8F0811422083000F04FFBEA
:1009480008B0BDE8F08100BFDC090008FC09000818
:1009580003000200152904D20268044B9A4200D110
:1009680008B903487047083000F048BBFC09000884
:100978000300020010B481B013460268074CA2427B
:1009880000D118B901B010BC0548704701B000F19A
:10099800240210BC083000F035BB00BFFC09000879
:1009A8000300020010B481B013460268074CA2424B
:1009B80000D118B901B010BC054870470A4601B00B
:1009C80000F1240110BC083000F070BBFC090008DD
:1009D800030002000123456789ABCDEFFEDCBA981E
:1009E80076543210F0E1D2C300000000000000008D
:1009F80000000000F10800081D0900085D09000852
:100A08007D090008AD09000801040008790F0008F5
:100A1800C50F0008810F0008F0B5A3B004460B48C5
:100A280002900D4616461F46094B0822402104A88D
:100A380000F0D1FA28980190009733462A462146BB
:100A480002A800F01BF823B0F0BD00BFFC090008A5
:100A5800100A000810B5040008BF002408D0054893
:100A6800054B20600822402104F1080000F0B3FA89
:100A7800204610BDFC090008100A00082DE9F041C5
:100A880004460E46216817464A681D469047804628
:100A9800B8F5003F19D1226806999368204698470F
:100AA8008046B8F5003F10D123683146DE683A46E3
:100AB8002046B0478046B8F5003F06D12368079A1C
:100AC80029461D692046A847804621680A682046AD
:100AD80090474046BDE8F08110B500F033FA4FF476
:100AE800403400280EBF034C4FF4C07113F0F2FBE2
:100AF800204610BD0200030010B5044600F022FA9B
:100B080008B9054810BD0021A160D0F87C21116802
:100B180088474FF4403010BD0200030070B504460A
:100B28000D4600F00FFA064E40B1D0F87C0141683E
:100B38008847A84224BF65604FF44036304670BDF0
:100B4800020003002DE9FF4715000C4600D02CB128
:100B5800064600F0F7F95FEA000801D16448C3E0EF
:100B6800D8F8F80001684A689047B0F5003F17D1F7
:100B7800D8F87C118A68404690478146B9F1810FC0
:100B880080F09E80A94508F1FC0A17D2D8F8F80031
:100B98000368D3F80CC02A462146E047B0F5003F69
:100BA80040F08E80D8F8F8000368D3F810C06A4681
:100BB8005146E047B0F5003F76D10AE0002004E056
:100BC800215C0AF800100098401C00900098A84288
:100BD800F6D34FF0000C4749474A484B01AC009800
:100BE800844558D2D3E9007001ADC5E9007010788A
:100BF80000281ABF042086464FF0000E085854F803
:100C08000E5028443E4D05600127D0F800E087606B
:100C1800019D4F681AF80C007D408EEA050585F0A5
:100C2800040E65680F687D4085F0FC05754485F005
:100C3800A30568400AF80C000CF1010CCFE7D3E9D2
:100C4800004501A8C0E9004510782E4D002814BFC2
:100C58004FF0040E4FF0000E01A8744651F80EE054
:100C68000459A6440127CEF80050DEF80040CEF81B
:100C780008704D68019F40687D406C400D68684071
:100C880084F0040480F0FC00041984F057040AF886
:100C98000C400CF1010CCC45D1D3D8F8F800016810
:100CA8004A689047B0F5003F0AD1D8F8F8000368C1
:100CB800D3F80C804A465146C047B0F5003F01D0F2
:100CC800114811E0002006E05AF8201081F06A313E
:100CD8004AF82010401CB0EB990FF5D3B06840F0EB
:100CE8000100B0604FF4403004B0BDE8F08700BFA9
:100CF8000200030074440108E8080020240F0008DB
:100D0800ADBE4ED70DBE75A10100030038B50C4627
:100D1800017A1546CA0702D500F014F908B908483F
:100D280032BDD0F8F80003682146DC682A46A0479F
:100D3800B0F5003F01D0034832BD4FF4403032BD1A
:100D480002000300010003002DE9F84191B00546B7
:100D58000E461746402101A813F0BCFA297AC807A5
:100D680004D5284600F0EEF8040002D1DFF8A4808C
:100D78004BE0D4F8F800DFF8A0800368D3F810C07F
:100D88006A4601A9E047B0F5003F3ED1D4F8F80023
:100D980001684A689047B0F5003F36D1D4F87C1115
:100DA8008A6820469047D4F8F830024618461B68EF
:100DB800D3F80CC004F1FC01E047B0F5003F24D1A2
:100DC800D4F87C0141688847D4F8F83002461846C0
:100DD8001B68D3F80CC001A9E047B0F5003F14D157
:100DE800D4F8F8000268696893689847B0F5003F3E
:100DF8000BD1D4F8F80003681C693A463146A0477D
:100E0800B0F5003F08BF4FF44038404612B0BDE887
:100E1800F08100BF02000300010003002DE9F84142
:100E2800A5B0074688461646402115A813F052FA81
:100E380000220492402105A813F04CFA387AC10721
:100E48005ED5384600F07EF8050059D0D5F8F80090
:100E58002D4C0368D3F810C06A4605A9E047B0F5E1
:100E6800003F3CD1D5F8F80001684A689047B0F5D2
:100E7800003F34D1D5F87C118A6828469047D5F8C8
:100E8800F830024618461B68D3F80CC005F1FC017F
:100E9800E047B0F5003F22D1D5F87C01416888478A
:100EA800D5F8F830024618461B68D3F80CC005A9D7
:100EB800E047B0F5003F12D1D5F8F800026879682C
:100EC80093689847B0F5003F09D1D5F8F800036852
:100ED8001D6904AA15A9A847B0F5003F01D020460E
:100EE8000FE00A4B0A490B4A0396029101924046C9
:100EF8001C68049B009415AA796800F0E5F900E0E5
:100F0800054826B0BDE8F081010003007C440108D3
:100F1800936E030026C703000200030004B001011A
:100F280000170145E10A0008010B0008250B00081D
:100F3800B50300084D0B0008150D0008510D0008F9
:100F4800250E00080168024A914218BF0020704728
:100F58002C0F000810B5040008BF002404D0034873
:100F68002060204609688847204610BD2C0F0008DD
:100F780020225C3013F0ACB9F0B58468A3080022D5
:100F880004F0030407E000F15C0555F8226035BA67
:100F980041F82250521C9A42F5D300220BE000F18E
:100FA8005C0502EB830755F82360D500C5F11805E9
:100FB800EE40CE55521CA242F1D3F0BD30B5C46804
:100FC80003690022E31AD5188C5C0544521C082AD0
:100FD8002C77F8D330BD0360C1600261704738B523
:100FE800044615460022626023685A68904700202C
:100FF8006061A061A5604FF4003032BD81604FF49C
:10100800003070472DE9F84304462079D4F80C8065
:10101800450748BF244845D466691D46A8F1010024
:1010280000EAD60306EBC506B6EBC50F666102D229
:10103800A669761CA6611746A66906EB5576A661D1
:101048000E46E918884225D2A8EB03094A463146DC
:10105800F81813F03DF92268136839460FE0424644
:10106800384613F035F923681A6839462046904700
:1010780007E0311811F00300F1D122681368204607
:101088009847484600EB0809A9F10101A942F0D3A5
:10109800002300E000202A1A3118F81813F018F974
:1010A8004FF40030BDE8F283040002002DE9FC4F44
:1010B800024685B0D0681369DFF86CC1DFF86C812F
:1010C800A0EB030A506840F004005060002703A812
:1010D80002900DF10C0ED8E9003403A8544DC0E974
:1010E80000342878534D00280CBF00230423994668
:1010F8005CF803305EF80940234401261D601C6833
:101108009E60DCF80430039DDCF80090DEF8046093
:101118005D406540484C654089EA0606474C664094
:101128007519474C6540D8E9006B03AC0028C4E941
:10113800006B0EBF002404200424029E5CF800000B
:10114800345920183F4C04600126046886600398CF
:10115800029E43406340384C7068634089EA00004F
:10116800364C6040034438484340280018BF0120EB
:101178005B1E9B41042F2CBFC0B2D80F02F1140391
:1011880053F8200007F00303C3F10303DB00D84042
:101198000DF807007F1C082F9DD315460C466A6979
:1011A800AB69E868D20842EA4372401E00EA0207C7
:1011B800002302409B420AD8524508D28020E055BD
:1011C8007F1C574516D2AAEB0701E01910E08020D2
:1011D800E05500E0E355E8687F1C8742FAD32A68A7
:1011E800136828469847BAF1000F03D051462046A5
:1011F80013F070F82A68069E059F9368694628468A
:1012080098472A68D2F8009021462846C8472B6894
:10121800DA683946284690470EB1A86830604FF41E
:10122800003007B0BDE8F08F74440108541200087C
:10123800E80800205FC5109304850012FC68017A55
:10124800C0F524FF24AF33D426AF698B04B0010165
:1012580000170145F8B501240094002300240DE08F
:10126800009D065D0F5D7E40F643761CF60F86F006
:10127800010635400095641C009DEB189442EFD39D
:101288001846F2BDF8B5002301240094002A11E0A5
:10129800009C85188F1815F8016C17F8015C6E40D2
:1012A800F643761CF60F86F0010634400094009C45
:1012B800E318521EECD11846F2BD00005D1200087A
:1012C8008D120008010000002DE9F84F1D46DDF8D9
:1012D80028900B9F0D9C4FF0FF3300930E469246CB
:1012E800D9F800B0804632465146D847834664B3A1
:1012F800D9F8043032465146404698476FEA0B0207
:10130800521C42EA0B0200996FEAD2735B1C194027
:10131800C2430091521C024300996FEAD2735B1CCE
:101328001940009186F05531484087EA000181F064
:101338005531216080F05531C943491C0843009A52
:101348006FEAD070401C82430092D9F80800012847
:1013580009D17540E943491C0D4300986FEAD572DD
:10136800521C90430AE0F11C85EA9102D243521CB8
:10137800154300986FEAD5735B1C984386F0AA362C
:10138800009086EA0B0686F0AA33F243DB430C98FA
:10139800C2F3C0725B1C42EAD3720099D243521C5A
:1013A80091430091774000998843009987F0AA37C4
:1013B8000F403843BDE8F28F034613F8012B002A8B
:1013C800FBD1181A0138704781F0004102E000BFD4
:1013D80083F0004330B54FEA41044FEA430594EAED
:1013E800050F08BF90EA020F1FBF54EA000C55EA28
:1013F800020C7FEA645C7FEA655C00F0E2804FEAF9
:101408005454D4EB5555B8BF6D420CDD2C4480EADA
:10141800020281EA030382EA000083EA010180EA0A
:10142800020281EA0303362D88BF30BD11F0004F58
:101438004FEA01314FF4801C4CEA113102D040428E
:1014480061EB410113F0004F4FEA03334CEA1333C9
:1014580002D0524263EB430394EA050F00F0A780E1
:10146800A4F10104D5F1200E0DDB02FA0EFC22FADC
:1014780005F2801841F1000103FA0EF2801843FAD0
:1014880005F359410EE0A5F120050EF1200E012AC1
:1014980003FA0EFC28BF4CF0020C43FA05F3C018FF
:1014A80051EBE37101F0004507D54FF0000EDCF178
:1014B800000C7EEB00006EEB0101B1F5801F1BD321
:1014C800B1F5001F0CD349085FEA30004FEA3C0C25
:1014D80004F101044FEA445212F5800F80F09A801B
:1014E800BCF1004F08BF5FEA500C50F1000041EB1F
:1014F800045141EA050130BD5FEA4C0C404141EB23
:101508000101013C28BFB1F5801FE9D291F0000F1D
:1015180004BF01460020B1FA81F308BF2033A3F1CC
:101528000B03B3F120020CDA0C3208DD02F1140CC3
:10153800C2F10C0201FA0CF021FA02F10CE002F1FE
:101548001402D8BFC2F1200C01FA02F120FA0CFCF7
:10155800DCBF41EA0C019040E41AA2BF01EB045140
:10156800294330BD6FEA04041F3C1CDA0C340EDC3E
:1015780004F11404C4F1200220FA04F001FA02F381
:1015880040EA030021FA04F345EA030130BDC4F13F
:101598000C04C4F1200220FA02F001FA04F340EA34
:1015A8000300294630BD21FA04F0294630BD94F0E5
:1015B800000F83F4801306BF81F480110134013DCC
:1015C8004EE77FEA645C18BF7FEA655C29D094EA3D
:1015D800050F08BF90EA020F05D054EA000C04BFBB
:1015E8001946104630BD91EA030F1EBF00210020A6
:1015F80030BD5FEA545C05D14000494128BF41F045
:10160800004130BD14F580043CBF01F5801130BDA8
:1016180001F0004545F0FE4141F470014FF0000033
:1016280030BD7FEA645C1ABF194610467FEA655CE4
:101638001CBF0B46024650EA013406BF52EA033586
:1016480091EA030F41F4002130BD00BF90F0000F74
:1016580004BF0021704730B54FF4806404F13204B0
:101668004FF000054FF0000150E700BF90F0000F69
:1016780004BF0021704730B54FF4806404F1320490
:1016880010F0004548BF40424FF000013EE700BF60
:1016980042004FEAE2014FEA31014FEA02701FBFF0
:1016A80012F07F4393F07F4F81F06051704732F022
:1016B8007F4208BF704793F07F4F04BF41F4002179
:1016C800704730B54FF4607401F0004521F00041D7
:1016D8001CE700BF50EA010208BF704730B54FF061
:1016E80000050AE050EA010208BF704730B511F062
:1016F800004502D5404261EB41014FF4806404F19A
:1017080032045FEA915C3FF4D8AE4FF003025FEA1F
:10171800DC0C18BF03325FEADC0C18BF033202EBA3
:10172800DC02C2F1200300FA03FC20FA02F001FAFD
:1017380003FE40EA0E0021FA02F11444BDE600BFA0
:101748004FF0FF3C06E000BF4FF0010C02E000BF85
:101758004FF0010C4DF804CD4FEA410C7FEA6C5C68
:101768004FEA430C18BF7FEA6C5C1BD001B050EA0B
:10177800410C0CBF52EA430C91EA030F02BF90EAF6
:10178800020F0020704710F1000F91EA030F58BFB5
:10179800994208BF90422CBFD8176FEAE37040F017
:1017A800010070474FEA410C7FEA6C5C02D150EAB5
:1017B800013C07D14FEA430C7FEA6C5CD6D152EA70
:1017C800033CD3D05DF8040B704700BF8446104635
:1017D80062468C461946634600E000BF01B5FFF734
:1017E800B7FF002848BF10F1000F01BD4DF808ED04
:1017F800FFF7F4FF0CBF012000205DF808FB00BFD5
:101808004DF808EDFFF7EAFF34BF012000205DF82E
:1018180008FB00BF4DF808EDFFF7E0FF94BF01207B
:1018280000205DF808FB00BF4DF808EDFFF7CEFF7C
:1018380094BF012000205DF808FB00BF4DF808EDBB
:10184800FFF7C4FF34BF012000205DF808FB00BF8C
:101858004FEA410212F5001215D211D56FF47873D0
:10186800B3EB625212D94FEAC12343F0004343EA73
:10187800505311F0004F23FA02F018BF404270474E
:101888004FF00000704750EA013005D111F00040D8
:1018980008BF6FF0004070474FF00000704700BF6E
:1018A80080F0004002E000BF81F0004142001FBF0D
:1018B8005FEA410392EA030F7FEA226C7FEA236C16
:1018C8006AD04FEA1262D2EB1363C1BFD21841400B
:1018D80048404140B8BF5B42192B88BF704710F0A1
:1018E800004F40F4000020F07F4018BF404211F044
:1018F800004F41F4000121F07F4118BF494292EAAC
:10190800030F3FD0A2F1010241FA03FC10EB0C00D7
:10191800C3F1200301FA03F100F0004302D5494264
:1019280060EB4000B0F5000F13D3B0F1807F06D311
:1019380040084FEA310102F10102FE2A51D2B1F109
:10194800004F40EBC25008BF20F0010040EA0300FE
:101958007047490040EB0000013A28BFB0F5000F7E
:10196800EDD2B0FA80FCACF1080CB2EB0C0200FA34
:101978000CF0AABF00EBC25052421843BCBFD04083
:101988001843704792F0000F81F4000106BF80F4FD
:1019980000000132013BB5E74FEA41037FEA226CC0
:1019A80018BF7FEA236C21D092EA030F04D092F08B
:1019B800000F08BF0846704790EA010F1CBF0020BF
:1019C800704712F07F4F04D1400028BF40F000401C
:1019D800704712F100723CBF00F50000704700F03C
:1019E800004343F0FE4040F4000070477FEA226263
:1019F80016BF08467FEA23630146420206BF5FEA34
:101A0800412390EA010F40F4800070474FF0000333
:101A180004E000BF10F0004348BF40425FEA000CFA
:101A280008BF704743F0964301464FF000001CE0A2
:101A380050EA010208BF70474FF000030AE000BFF8
:101A480050EA010208BF704711F0004302D5404236
:101A580061EB41015FEA010C02BF844601460020A8
:101A680043F0B64308BFA3F18053A3F50003BCFAC3
:101A78008CF2083AA3EBC25310DB01FA02FC634470
:101A880000FA02FCC2F12002BCF1004F20FA02F277
:101A980043EB020008BF20F00100704702F120026A
:101AA80001FA02FCC2F1200250EA4C0021FA02F2CB
:101AB80043EB020008BF20EADC7070474FEA40029F
:101AC800B2F1FE4F0FD34FF09E03B3EB12620DD964
:101AD8004FEA002343F0004310F0004F23FA02F0CE
:101AE80018BF404270474FF00000704712F1610F75
:101AF80001D1420205D110F0004008BF6FF000404C
:101B080070474FF00000704753B94AB9002908BF21
:101B180000281CBF4FF0FF314FF0FF3000F070B9C4
:101B2800ADF1080C6DE904CE00F006F8DDF804E02C
:101B3800DDE9022304B070472DE9F047089E0D4601
:101B480004460F46002B4AD18A42944665D9B2FA18
:101B580082F343B102FA03FCC3F120029F4020FA4A
:101B680002F217439C404FEA1C4E1FFA8CF5B7FB54
:101B7800FEF1220C0EFB117742EA074201FB05F049
:101B880090420AD91CEB020201F1FF3780F01B8159
:101B9800904240F2188102396244121AA4B2B2FB90
:101BA800FEF00EFB102244EA024400FB05F5A542B4
:101BB8000AD91CEB040400F1FF3280F00681A5422B
:101BC80040F203816444023840EA0140641B00216A
:101BD8001EB1DC400023C6E90043BDE8F0878B4214
:101BE80008D9002E00F0EC800021C6E9000508465F
:101BF800BDE8F087B3FA83F1002949D1AB4202D39B
:101C0800824200F2F780841A65EB0302012017462E
:101C1800002EE2D0C6E90047DFE702B9FFDEB2FADC
:101C280082F3002B40F08F808A1A4FEA1C471FFA74
:101C38008CFE0121B2FBF7F507FB1520220C42EAC6
:101C480000420EFB05F0904208D91CEB020205F198
:101C5800FF3802D2904200F2CA804546121AA4B256
:101C6800B2FBF7F007FB102244EA02440EFB00FE29
:101C7800A64508D91CEB040400F1FF3202D2A645A0
:101C880000F2BA801046A4EB0E0440EA05409FE734
:101C9800C1F120078B4022FA07FC4CEA030C05FA35
:101CA80001F420FA07F3FD40234300FA01F94FEA53
:101CB8001C401FFA8CFEB5FBF0F81C0C00FB1855F5
:101CC80044EA054408FB0EF5A54202FA01F20BD9D5
:101CD8001CEB040408F1FF3A80F08780A54240F22B
:101CE8008480A8F102086444641B9DB2B4FBF0F33D
:101CF80000FB134445EA044403FB0EFEA64508D93D
:101D08001CEB040403F1FF306BD2A64569D9023BF2
:101D1800644443EA0840A0FB0283A4EB0E049C42FF
:101D2800C6461D4655D352D056B1B9EB0E0364EBE7
:101D3800050404FA07F7CB40CC401F43C6E90074FA
:101D48000021BDE8F087C3F1200102FA03FC20FA64
:101D580001F225FA01F19D402A434FEA1C471FFA78
:101D68008CFEB1FBF7F007FB1015110C41EA054199
:101D780000FB0EF58D4204FA03F408D91CEB0101AF
:101D880000F1FF382FD28D422DD902386144491B0A
:101D980092B2B1FBF7F507FB151142EA014205FBC8
:101DA8000EF1914208D91CEB020205F1FF3816D258
:101DB800914214D9023D6244521A45EA004139E77A
:101DC8003146304609E73946E7E61046FCE6C145A4
:101DD800AAD2B8EB020E63EB0C050138A4E745461E
:101DE800EAE7034695E74046D1E7D0467CE7023D5F
:101DF800624433E708460BE76444023843E700BF10
:101E0800704700BF1348144A08B54FF00043C0E9B3
:101E180000230422002342610122C2614FF4805151
:101E280007220383C0E90233C0E90933C0E90C1271
:101E38000361837680F8203080F82C30826380F844
:101E48003C30C36405F02AFB18B1BDE8084000F037
:101E580031BC08BDEC080020002401400268084B92
:101E68009A4282B00AD14FF0B0431A6E42F400721F
:101E78001A661B6E03F400730193019B02B070474E
:101E8800002401400268054B9A4201BF4FF0B0425E
:101E9800136E23F400731366704700BF00240140DB
:101EA80030B585B000240546CDE901440394FFF719
:101EB800A9FF144805F08AFE08B100F0FBFB1148A1
:101EC800039401A9CDE9015405F046FC08B100F0DE
:101ED800F1FB0C4805F0A4FD08B100F0EBFB4FF056
:101EE800FF31084805F0DAFB064805F051FE0548C1
:101EF80005F02EFC0446034805F0F4FD204605B025
:101F080030BD00BFEC080020014B024A1A60704740
:101F1800EC0800200024014008B50948FFF7C0FF7D
:101F280068B1084BB3F8AA304FF6FF72934216BF58
:101F380040F6E442044B5343B3FBF0F398B208BDB8
:101F4800002000B40075FF1FD8084C0013B500230B
:101F5800ADF80630FFF7E0FF04461948FFF7A0FF89
:101F6800184BB3F8C820B3F8A8108A4204FB00F055
:101F780018D040F6E443B0FBF3F364205B1A434304
:101F8800521A93FBF2F31E331BB2ADF80630BDF8BC
:101F980006305BB21B02ADF80630BDF8060000B291
:101FA80002B010BD4FF47A7240F6FF73B0FBF3F342
:101FB8005343A3F53923A3F50C6340F6C412E0E7B5
:101FC800001000B00075FF1F4FF0B04382B09A6A4E
:101FD80022F480529A629A6C42F480529A649B6C02
:101FE80003F480530193019B002002B070474FF027
:101FF800B04382B09A6C02439A649B6C034001938D
:10200800019B02B0704708B50420FFF7F0FF0120DC
:10201800FFF7EDFF0220FFF7EAFF002211460B2031
:1020280005F072FE0B2005F0A1FE002211460C20DF
:1020380005F06AFE0C2005F099FE002211460D20DD
:1020480005F062FE0D2005F091FE002211460E20DB
:1020580005F05AFE0E2005F089FE002211460F20D9
:1020680005F052FE0F2005F081FE002211461020D7
:1020780005F04AFE102005F079FE002211461120D5
:1020880005F042FE112005F071FE002236201146AF
:1020980005F03AFEBDE80840362005F067BE0000AE
:1020A80008B506F0ABF810B16FF0040008BD064B98
:1020B8009A6942F040429A614CF2FA321A6106F08B
:1020C800AFF80028F2D0EFE700400058F0B585B02F
:1020D80000230C4600930646A8B3FFF7E1FF054628
:1020E80070BB06F08BF888BB1A481B4A0223019381
:1020F800D0F8E01506F1784302EA8121B3FBF1F745
:1021080001FB1733DB0A0293D0F8E00504F17841AC
:102118000139314402EA8022B1FBF2F002FB1011CE
:10212800C3EBD1230133694601A8039306F0F8F8FD
:1021380020B102280CBF01256FF0010506F070F8E8
:10214800284605B0F0BD6FF00505F9E76FF0040506
:10215800F6E700BF0070FF1F00FCFF03014B18608B
:1021680000207047500900202DE9F04F89B0B0F1E8
:10217800006F06460F460092C0F0C580DFF89881D0
:10218800664DD8F8E03505EA832303F10063013B87
:10219800984200F2B880002800F0B880002900F0CA
:1021A800B58040EA02035B0740F0B080FFF778FF94
:1021B8000446A0BB06F022F8002840F0AA80D8F810
:1021C800E01506F1784205EA8121B2FBF1F301FB43
:1021D8001322009B03F17843013B3344B3FBF1F036
:1021E80001FB1033DB0A01334FEAD22AA3EBD222D8
:1021F800012A039388BFC6F30A050AF58038C6F199
:10220800080398BF009D069388BFC5F500654FEA8F
:10221800C828B346039B9A4505D306F001F8204623
:1022280009B0BDE8F08FA6F10803069A1A44954252
:1022380019D804950197CDF814B04FF00009059B03
:1022480009EB0301049B99453ED3009BAB442F4403
:102258005D1BB5F5006F28BF4FF400650AF1010A50
:1022680008F50068D6E753F8081F5A68B2F1FF3F2F
:1022780008BFB1F1FF3FD8D0294B186810B96FF0EB
:102288000504CAE7B8F1000F04D04FF400624146D4
:1022980011F0B2FBDFF88890D9F80030CBF30A00D0
:1022A80039461844AAB211F0A7FB4FF40061404622
:1022B800FFF70CFF08BBD9F8003001934FF4006317
:1022C800CDF814800493B8E7019B07914B4402931F
:1022D8000120D3E9002305F0DDFF88B90799019BA8
:1022E800D1E9000259F80310029B5B689A4208BFC3
:1022F800884205D109F10809A1E76FF001048CE7CC
:102308006FF0030489E74FF0FF3488E76FF00504A6
:1023180085E76FF0040482E70070FF1F00FCFF03ED
:1023280050090020B1F1006F70B511D30B4BD3F8F1
:10233800E0650B4B03EA862303F10063013B9942F6
:1023480006D840B139B192B211F056FB002070BDE9
:102358004FF0FF30FBE76FF00500F8E70070FF1F54
:1023680000FCFF03B0F1006F10B40DD3084BD3F895
:10237800E045084B03EA842303F10063013B9842DC
:1023880002D810BCFFF7A2BE4FF0FF3010BC704758
:102398000070FF1F00FCFF034FF0B04382B0DA6CFF
:1023A8000243DA64DB6C03400193019B02B070477F
:1023B8002DE9F04186B01422002101A811F054FF44
:1023C80001203B4EFFF7E8FF0220FFF7E5FF04205E
:1023D800FFF7E2FF08210122304606F015F9012532
:1023E8004FF40417022301A94FF09040CDE90137BB
:1023F800039505F0E3FF4FF4441301A94FF0904013
:102408000024CDE902354FF02008019505F0D6FFEC
:1024180001A93046CDE90187039405F0CFFF01A952
:102428003046CDE90187039405F0C8FF082301A9C8
:102438003046CDE90135CDE9035405F0BFFF4FF42F
:10244800007301A94FF09040CDE90135CDE903545F
:1024580005F0B4FF04230DEB03013046CDE9013547
:10246800CDE9034405F0AAFF22462146062005F0DF
:102478004BFC062005F07AFC22462146072005F091
:1024880043FC072005F072FC22462146162005F081
:102498003BFC162005F06AFC22462146162005F072
:1024A80033FC162005F062FC06B0BDE8F08100BFE1
:1024B8000004004808B51248124A134BC0E900232B
:1024C80000230122C0E90232C0E90433C0E906331F
:1024D800036206F00DFA08B100F0ECF80848002194
:1024E80006F086FB08B100F0E5F80548002106F083
:1024F800A5FB18B1BDE8084000F0DCB808BD00BF76
:10250800140A0020005800405D3E302070B596B097
:1025180005461422002103A811F0A6FE3822002146
:1025280008A811F0A1FE2A68304B9A425BD180239B
:10253800089308A84FF440230E9307F0DBF808B17E
:1025480000F0B8F84FF0B0444FF4C050E36C43F0DB
:102558000103E364E36C03F001030293029B12237B
:102568000026CDE903030323CDE905634FF090402E
:10257800042303A9079305F021FFA36DDFF870C0BA
:1025880043F48003A365A36D1A4C03F480030193FD
:10259800019B26620D23C4E900C320468023C4E9B9
:1025A8000266C4E90436C4E9066605F03FFC08B1D2
:1025B80000F080F8104AEC63A562104C0E23C4E9C1
:1025C80000231021002380222046C4E90213C4E915
:1025D8000423C4E90633236205F028FC08B100F09F
:1025E80069F8AC63A56216B070BD00BF0058004022
:1025F800440002405409002058000240B409002059
:1026080000B59BB04822002108A811F02DFE182221
:10261800002102A811F028FE06F036FB4FF0B04268
:102628000120D2F8903023F01803C2F89030D2F885
:10263800003423F4C06343F40073C2F80034D2F8C2
:10264800003403F4C0630193019B2423089381237E
:102658000B930023CDE91003B02208A8CDE912237B
:1026680006F08AFC08B172B6FEE74F23CDE90230C6
:10267800CDE90400CDE90600022102A806F016FF04
:1026880008B172B6FEE71BB05DF804FB08B504F0AC
:10269800B3FEFFF7B5FFFFF78BFEFFF7B4FCFFF7BC
:1026A80009FF00F0F8FD40F6B83000F049FA00F0F4
:1026B800F9FDFCE772B6FEE700B58DB02C220021CB
:1026C80001A811F0D1FD1748174B03601F23836041
:1026D8004FF080420023C0E90433C0E90723836137
:1026E8004FF48073436207F08BF908B1FFF7E2FFFC
:1026F8000C4807F0B1FA08B1FFF7DCFF4FF00053C0
:1027080000220793074808924FF4807301A90292A8
:1027180006920B9307F0D4F908B1FFF7CBFF0DB081
:102728005DF804FB680A00200028004010B5044644
:1027380090B03822002102A811F096FD2268194BAA
:102748009A422CD14FF48033029302A84FF480733D
:102758000F9306F0CFFF08B1FFF7ACFF4FF0B0437F
:102768000220D3F8902042F40042C3F890209A6DDA
:1027780042F480629A659B6D002203F480631146DF
:102788000193019B05F0C0FA022005F0EFFA002240
:102798002A20114605F0B8FA2A2005F0E7FA10B009
:1027A80010BD00BF002800407047000008B504F0C5
:1027B80039FE044B0120C3F88800BDE8084006F044
:1027C800BBBA00BF0004005804F033BE08B504F0DB
:1027D80030FE00F063FCFFF7EBFDFFF714FCBDE8EB
:1027E8000840FFF767BE08B504F01CFEBDE80840C6
:1027F8000121002006F050BA70477047FEE7FEE757
:10280800FEE7FEE7FEE77047704770477047000035
:10281800014807F047BA00BF680A0020012005F008
:10282800F9BE022005F0F6BE70477047014805F072
:1028380077BC00BF54090020014805F071BC00BFF7
:10284800400B0020014805F06BBC00BFE00A0020E7
:10285800FFF7F2BF7047202005F0DCBE704700008C
:10286800014807F0E3BD00BFA00B0020014807F0B6
:102878004BB800BF680A0020014807F03EBC00BF03
:10288800CC0A00202DE9F04389B080460020109E34
:102898000790894615461F46FDF7C2FCF0B9104C53
:1028A800CDE90090CDE9020407AB0E480593142347
:1028B80004933A46434629460068FDF77BFD2346C4
:1028C800324604F1140153F8044B42F8044B8B428E
:1028D800F9D1079B337509B0BDE8F0830120FAE709
:1028E800A00A0020704401087FB5124C00253C2343
:1028F80002A86375CDE90255257500F0C3F80423D5
:1029080003AA009412210C48FFF7BCFF0B491422BC
:10291800204611F099FC0646B0FA80F0400960752F
:102928000090074B2A462946022010F05DFF3046EA
:1029380004B070BDB40A0020B64401084E0E002051
:1029480098440108054808B50823036007F0F0F922
:1029580018B1BDE80840FFF7ADBE08BDCC0A00209D
:102968004FF0B04307B55A6E42F001025A665B6EEB
:10297800002203F00103019311463220019B05F068
:10298800C3F9322003B05DF804EB05F0EFB900009D
:102998000CB407B5054A05AB1021019311F036FBBD
:1029A80003B05DF804EB02B0704700BFC8440108EB
:1029B80030B585B0044602A80D4611F053F9BDF9AB
:1029C8000C30064A00931021029B2046FFF7E0FFD7
:1029D8002046FEF7F1FC288005B030BDC844010848
:1029E8004FF0B04210B5936823F40043936011F0A0
:1029F800C1F90E4B01241C7000F0B6F810F08AFEE5
:102A08000B4810F0A1FE0B4B4FF400421A61204610
:102A180010F0A0FEFFF778FA00F012F910F096FF18
:102A280021462046BDE8104010F0B0BFD80A00206B
:102A3800B92900080040005810F0BEBF08B5FFF7DC
:102A48006BFA40F6B83398420CD8B0F5E16F0BD367
:102A5800FE23A0F5E16058434FF49663B0FBF3F012
:102A6800C0B208BDFE20FCE70020FAE77FB5684643
:102A780000F0CAF80198FFF721F800B207B05DF836
:102A880004FB0000194A38B5D2F88035591C0446B1
:102A980019D104F0D5FC054604F0DEFC054404F029
:102AA800D5FC2B0EE3712B0CA3712B0A6371030E5B
:102AB800E370C0F30742C0F307232571C0B2A270C8
:102AC8006370207038BD190AC3718171190C1B0E0F
:102AD80041710371D2F88435C370D2F88405C0F30C
:102AE8000722C0F30743000EE9E700BF0070FF1F8D
:102AF80038B5094BD3F8803503600133054609D151
:102B080004F09EFC044604F0A1FC444004F0A4FC3C
:102B180044402C6038BD00BF0070FF1F0121022017
:102B280010F01EBF0021022010F01ABF00207047CD
:102B3800024B187808B100F0BBB87047D80A0020DB
:102B480082B00190019802B000F04EB94FF0B04346
:102B580082B0DA6C42F00202DA64DB6C03F0020342
:102B68000193019B02B070472DE9F043254C87B0D3
:102B780004F078FC04F07EFC04F084FC01230025BA
:102B880002934FF48059032301A9204604934FF47C
:102B9800005803950595FFF7D9FFFFF7D7FFFFF713
:102BA800D5FFFFF7D3FFCDF8049005F007FC01A986
:102BB80020464FF40067CDF8048005F0FFFB01A91B
:102BC80020464FF40046019705F0F8FB01A920467E
:102BD800019605F0F3FB2A464946204605F014FD08
:102BE8002A464146204605F00FFD2A46394620462A
:102BF80005F00AFD2A463146204605F005FD07B0D6
:102C0800BDE8F0830004004810B50446FFF79EF9BC
:102C1800074BA36040F30F20FEF7FCFE054B064A66
:102C28002360064B6060C4E90323002010BD00BF89
:102C38000000484200007A440D093E00AB0305003D
:102C480000207047014B1868704700BFDC0A00205D
:102C58000320704708B501464FF47A7200238002BA
:102C6800890DFEF751FF08BD4FF47A73A0FB0303EB
:102C7800800A40EA83507047034B98689A689042EC
:102C8800FBD1C043704700BF0028004008B5FFF7DC
:102C9800F3FF014B186008BDDC0A002008B5FFF7F8
:102CA800EBFF024B1B68C01A08BD00BFDC0A0020FE
:102CB800024B187808B1FFF7DFBF7047D90A002028
:102CC80010B5074B074C0122DA654FF48071204696
:102CD80006F0E0FD4FF0FF332363002010BD00BF76
:102CE80000280040680A002002460021014806F03A
:102CF800EABF00BF680A002002460121014806F029
:102D0800E2BF00BF680A002010B58CB02C22002159
:102D1800044601A811F0A8FAFFF7D2FF0C4B0D48A2
:102D28001B681C440023089306934FF00053E443A8
:102D3800079301224FF4807301A902940B9306F0C4
:102D4800BFFE08B1FFF7B6FC00200CB010BD00BFF5
:102D5800DC0A0020680A002038B50546FFF78CFF1A
:102D680002210446074806F0B5FFC4F309024FF4F0
:102D78007A71A2FB0121920AA30A2A8043EA8050B1
:102D880038BD00BF680A00200148002106F0A2BF34
:102D9800680A00200148012106F09CBF680A00204B
:102DA800F8B50F4D2E78CEB90E4C4FF0FF3727638C
:102DB800FFF782FCFFF784FF4FF48071204606F08E
:102DC80069FD2046276306F029FF32462046022186
:102DD80006F079FFFFF75AFF01232B700020F8BD9A
:102DE800D90A0020680A0020014610B54FF47A720B
:102DF80000238002890DFEF787FE0146FFF73CFF9E
:102E08000446FFF739FF031B8B4200D310BD00BFF8
:102E1800F7E711F0B7B8000010B5064C02212046BC
:102E280006F058FF0221421C2046BDE8104006F07B
:102E38004ABF00BF680A00201648174A08B54FF471
:102E4800E133C0E9002300230C22C0E90233C0E9C2
:102E58000523C0E90733C0E90933036108F0C7F85F
:102E680008B1FFF727FC0B48002108F03CFA08B12D
:102E7800FFF720FC0748002108F055FA08B1FFF7D2
:102E880019FC044808F00FFA18B1BDE80840FFF72C
:102E980011BC08BDA00B00200044004070B596B0DE
:102EA80005461422002103A811F0DEF9382200217A
:102EB80008A811F0D9F92A68334B9A4261D1022344
:102EC800089308A8314B0A9306F014FC08B1FFF7E1
:102ED800F1FB4FF0B0430C219A6D2D4C42F40032B7
:102EE8009A659A6D02F400320292029ADA6C42F004
:102EF8000102DA64DB6C03F001030193019B0223F6
:102F08000026CDE903130323CDE905634FF0904074
:102F1800072303A9079305F051FA1E4826621423D4
:102F2800C4E900031023C4E9023620468023C4E91B
:102F38000436C4E9066604F079FF08B1FFF7BAFB66
:102F4800154AEC67A562154C1323C4E900232046F3
:102F580000238022C4E90233C4E90423C4E9063308
:102F6800236204F063FF08B1FFF7A4FB2520C5F82E
:102F7800804000220221A56204F0C6FE252004F04C
:102F8800F5FE16B070BD00BF0044004004000C0000
:102F9800400B0020800002406C000240E00A002044
:102FA80002680E4B9A4210B5044616D14FF0B04253
:102FB8000C21936D23F4003393654FF0904005F096
:102FC800A9FAE06F04F0A6FFD4F8800004F0A2FF8D
:102FD800BDE81040252004F0D7BE10BD00440040D5
:102FE80008B50A460146024807F084F9002008BDE2
:102FF800A00B002013B5114B114C18604FF40013AF
:10300800009302AB13E90600204608F0F0F82368A5
:10301800DA69D103FCD4DA695202FCD59A68084807
:1030280042F480029A6008F028F90649044801220F
:1030380008F096F8002002B010BD00BF340C002044
:10304800A00B00203C0C002008B5074B1860FEF7C9
:10305800DAFFFFF7F1FE054AD2F8803043F000634B
:10306800C2F88030002008BD380C00200008005845
:1030780008B54FF0B04308489A6B42F400329A639F
:103088009A6B22F400329A63FFF78AFF0F2004F04C
:103098007BFE002008BD00BFA00B002008B5074834
:1030A80007F0A5FF08B1FFF705FB054804F0BEFED1
:1030B80018B1BDE80840FFF7FDBA08BDA00B002015
:1030C800400B00200268044B9A4203D1034B0020B6
:1030D8001B681847704700BF00440040380C0020A8
:1030E80002680B4B9A4210B504460FD1094B1B6876
:1030F8002BB1D0F8902012B90748012198472046F3
:103108000549BDE81040012208F02AB810BD00BFEB
:1031180000440040340C00203C0C002002480122EE
:10312800102105F071BA00BF0004004802480022CF
:10313800102105F069BA00BF0004004813B5134C0C
:1031480023785BB9E37C03F0FF023BB9104B1146CF
:10315800022002B0BDE8104010F046BBFFF7C4FBE8
:1031680000380C4B18BF0120400018701A78022A4A
:1031780002BF00222270E2741B7800930022064BE3
:103188001146032010F030FB02B010BD4E0E002097
:1031980024450108440C00204045010838B5184C66
:1031A80023785BBBE37C03F0FF023BBB154D2B6828
:1031B800012B0CD92B68042B09D81146124B02207D
:1031C80010F012FB114A0421012000F07DFB2B684E
:1031D800042B13D900220E4B1146022010F004FBD9
:1031E800FFF782FB00380B4B18BF01204000187016
:1031F8001B78022B02BF00232370E37438BD00BF85
:103208004E0E0020400C0020574501087C4501085F
:1032180081450108440C002008B5FFF77FFF002214
:10322800054B1146032010F0DFFA01F019FDBDE847
:103238000840FFF77BBF00BFB4450108022801D84A
:10324800FFF76CBF7047022801D8FFF76FBF7047C0
:10325800022808B51BD8012210210D4805F0D4F921
:103268003220FFF76DFC0A480022102105F0CCF946
:1032780001221021064805F0C7F93220FFF760FC4B
:10328800BDE8084002480022102105F0BDB908BD7C
:1032980000040048704708B5FFF7A2FBBDE80840E6
:1032A80000F0D4BC4FF0FF3010F0EABB7047704715
:1032B800014BD870704700BF5C000020014B1874A8
:1032C800704700BF5C00002007B5064B00221B5C5E
:1032D80000931146044B022010F086FA03B05DF803
:1032E80004FB00BFF0450108D645010808B50220D7
:1032F800002110F08DFBBDE80840014810F0F0BD3A
:103308009C0D00200021012010F082BB13B50D4C4C
:10331800A0B120600C4810F095FD21680A4810F013
:1033280019FE094810F0DCFD236800930022074BC2
:103338001146032010F058FA02B010BD42F2107383
:103348002360E7E7740000209C0D0020F445010885
:1033580013B50D4C206023680BB90C4B23600C4847
:1033680010F070FD21680A4810F0F4FD084810F0CC
:10337800B7FD236800930022064B1146032010F086
:1033880033FA02B010BD00BF0C000020A086010077
:10339800B40D00201D46010837B5044600283AD070
:1033A80090F90650002D38D11F4810F04BFD2A46E1
:1033B80029461E4B022010F017FAE379012B0CBFA7
:1033C8001B4B1C4B2A46294602201B4D10F00CFAB9
:1033D800E3792B70194B1868FFF7BAFF184B186878
:1033E800FFF794FF2978174A174B012918BF13468E
:1033F800002200931146154B012010F0F5F994F9BD
:103408000530019394F9043000930022104B1146C3
:10341800022010F0E9F903B030BD00220D4B11462F
:10342800022010F0E1F9EAE7380D002062460108B1
:103438007746010894460108680D00200C0000201A
:10344800740000205D46010859460108B14601088C
:10345800E9460108D046010838B504460D46074834
:103468004FF40061FEF77EFF30B92A462146034833
:10347800BDE83840FEF778BE38BD00BF00F003084D
:103488000A460149FEF74EBF00F0030870B516481A
:1034980010F0D8FC08F0A0FB044650B10022134BF2
:1034A8001146022010F0A0F9BDE87040104810F055
:1034B80017BD104D104B02460146022010F094F93A
:1034C80001260E4B2E7022462146022010F08CF960
:1034D8000B4808F025FA2878314608F04FF80248DA
:1034E80010F0FEFCE0E700BF9C0D00201247010829
:1034F8006C0D0020000000203047010844470108F7
:103508005C00002030B587B0FFF798FA0021044628
:103518004FF4807010F07CFA02A801F0B9F923B2D8
:1035280003EB4303FE2203EB4313B3FBF2F3404ADE
:10353800392111703F4950680978DBB28DF8143091
:10354800017054680020607054682725A57054687D
:103558000125E57054682371374B1C7844B1187005
:10356800536861F07F0119703A23137005231CE03A
:10357800324B3348197811B901780029F6D0002167
:1035880001701970536804215971BDF808305168E9
:10359800180A88715168CB71BDF8103051681B0A40
:1035A8000B72BDF810304B720A232649264C097855
:1035B800012988BF00235370637A33B107F080FF75
:1035C800012802D1204610F03DFC204B1848D9783C
:1035D800002208F061F80446A8B901461C4B0122F4
:1035E800032010F001F91B4810F02CFC1A4B194865
:1035F8001968A14238BF214610F0ACFC154810F0FC
:103608006FFC07B030BD063410D107F053FF0446F5
:103618000028E8D001224FF47A730021B0FBF3F3BD
:10362800104600930D4B10F0DFF8DCE70024DAE7D2
:1036380004000020370D0020CC0D0020630E002070
:103648004D0E0020440C0020380D00205C000020A6
:10365800634701089C0D0020740000207247010890
:1036680000B503468DB000282CD0407802280AD037
:1036780003282AD0164B0022114602200DB05DF80F
:1036880004EB10F0B1B8DA7E0B929A7E0A925A7E59
:1036980009921A7E0892DA7D07929A7D06925A7DDF
:1036A80005925A680492DA68039293F914200292F8
:1036B800B3F9122001921B7C00930022054B11469E
:1036C80010F092F80DB05DF804FB034BD3E700BF90
:1036D80090470108A74701081948010801284FF039
:1036E80000020CBF024B034B1146022010F07CB8BD
:1036F800384801084A4801081FB50446002831D057
:103708000378002B2ED01D4810F0EAFB002211464A
:103718001B4B022010F068F894F91830039394F9C1
:103728000A300293237C0193E36800930022114638
:10373800144B032010F058F80022134B11460320B5
:1037480010F052F8237A012B0ED1617A0F4A104BF0
:10375800002908BF13460022009311460D4B032091
:1037680010F042F804B010BD00220B4B11460320A4
:1037780004B0BDE8104010F037B800BF840D002039
:103788006348010894480108C54801085E480108D3
:103798005F480108D2480108E348010808B5104B02
:1037A8000122002102201A7010F032F90D4810F0A1
:1037B80097FB0D4B1B788BB10C4B1A7872B9DB7CDD
:1037C80063B90B4B1A68042A9EBF1A6801321A6043
:1037D8000021BDE80840102010F01AB908BD00BF4C
:1037E800CC0D0020B40D0020680D00204E0E0020E6
:1037F800400C0020044B1B78022B03D10021082029
:1038080010F006B9704700BF0000002008B508F0A6
:10381800ECF980B907F054FE01280CD1BFF34F8FA3
:103828000549064BCA6802F4E0621343CB60BFF354
:103838004F8F00BFFDE708BD00ED00E00400FA056A
:1038480010B508F067FA10F1080F07D1064B0022EF
:10385800BDE81040114602200FF0C6BF013001D16B
:10386800024BF4E710BD00BFF14801080749010801
:1038780070477047022813B5014618D0202819D080
:1038880001281AD14FF0904004F0B8FE00220446F7
:1038980000900B4B114603200FF0A6FF012C0CD112
:1038A8000021022002B0BDE8104010F0B1B800219C
:1038B8000820F7E7034B01221A7002B010BD00BFC1
:1038C8001F490108C80E002073B505460C46164668
:1038D80007F0C4FE0346002838D00024264810F01C
:1038E800B1FA264B24481968A14238BF214610F086
:1038F80031FB214802B0BDE8704010F0F1BA4A68C7
:10390800F05CD0540133DAB2A242F8D31C4B0D70EC
:103918001B78012B88BF00244C701A4C637A33B192
:1039280007F0CEFD012802D1204610F08BFA164B85
:103938001648D978002207F0AFFE044640B9014680
:10394800134B012203200FF04FFFC7E70F49DAE7B7
:103958000634C2D107F0AEFD04460028BED04FF4AD
:103968007A730122B0FBF3F3002100930320094B83
:103978000FF03AFFB2E700BF9C0D00207400002052
:10398800440C0020380D00205C00002004000020BA
:103998006347010872470108044B1B7823B9044A9E
:1039A80005210120FFF790BF704700BF440C00209D
:1039B8003D49010810B5002490B03C22214601A8D9
:1039C800009410F051FC2F4B2022DA7219788DF8F0
:1039D800001059788DF8011099788DF80210D9786F
:1039E8008DF8031019798DF8041059798DF80510A0
:1039F80099798DF80610D9798DF80710197A8DF80C
:103A08000810597A8DF80910997A8DF80A108DF8EE
:103A18000B2021460DF10B0258180131007B02F8EA
:103A2800010F1C29F8D193F828208DF8282093F845
:103A380029208DF8292093F82A208DF82A2093F838
:103A48002B208DF82B2093F82C206AB193F83F2077
:103A580052B10DF12B0100229818013290F82C0078
:103A680001F8010F142AF7D107484FF40061FEF757
:103A780079FC20B9044840226946FEF775FB10B06E
:103A880010BD00BF7800002000F80308014940225B
:103A98000FF0B2BF00F8030870B52A4D28796B798A
:103AA8004D2BC0B233D1C0EB001080000A2838BFBC
:103AB8000A204FF47A735843234BAC791860EB799A
:103AC8004D2BE4B22BD1C4EB0414A40095F82C3090
:103AD8001E4E63BB95F83F304BBB42F21070FFF7A8
:103AE80015FC3068FFF734FC2B7A194A1949DBB208
:103AF80013706B7A184ADBB213700023EA1892F835
:103B08002C20D2B2CA540133142BF7D170BD6B7973
:103B1800482B0ABF4FF461636B795843C6E7EB79CA
:103B2800482B0ABF4FF46163EB795C43CEE7FFF79C
:103B3800EDFB012C38BF01244FF47A735C433460E9
:103B4800CFE700BF78000020740000200C000020A0
:103B5800620E00204E0E0020440C002010B590B0DC
:103B680000213C2201A8009110F07EFB402234493C
:103B780068460FF041FF9DF800203AB99DF8010012
:103B8800272803D19DF8021001290FD000222D4BC0
:103B9800114603200FF028FEFFF70CFF4FF47A7050
:103BA800FEF7CEFFFFF778FF10B010BD264B1A7056
:103BB800587099709DF80310D9709DF80410197108
:103BC8009DF8051059719DF8061099719DF8071018
:103BD800D9719DF8081019729DF8091059729DF84D
:103BE8000A1099729DF80B1001F03F01D972D87A2A
:103BF800D1B288421BD89DF8282083F828209DF848
:103C0800292083F829209DF82A2083F82A209DF866
:103C18002B2083F82B200DF12B010022981801325C
:103C280011F8014F80F82C40142AF7D1BAE701F1B6
:103C380040006844194410F8340C08730132D6E780
:103C480000F803084349010878000020F0B50B2369
:103C58008BB00A2200240125CDE906320327272349
:103C68001721CDE9043122465F4B03942146CDE963
:103C780001550097284609940FF0B6FD5B4B009557
:103C880022462146CDE9017402200FF0ADFD02263F
:103C98000523CDE900632246554B02942146304660
:103CA8000FF0A2FD534B009522462146CDE9017441
:103CB80030460FF099FD09A9204607F079FF099BC6
:103CC800C3F307220292C3F307421B0E019200932B
:103CD8002246494B214630460FF086FD09A9284661
:103CE80007F066FF099BDAB20392C3F30722029238
:103CF800C3F307421B0E0192009322463F4B214615
:103D080030460FF071FD3E4B3E48009422464FF47A
:103D1800FA7110F039F83C4B3C48009422464FF4B5
:103D2800FA7110F031F83A4B3A4800942A464FF4A9
:103D3800FA7110F029F82046FEF710FA08B1FEF7DC
:103D4800B9FC354B009400224FF4FA61334810F067
:103D58001BF8334A002101200FF016FF314A0021D9
:103D680002200FF011FF304A002104200FF00CFF51
:103D78002E4A002108200FF007FF00F005FC2C490F
:103D88002C4807F0D7FE2C4807F0CAFD214810F050
:103D9800A7F82A4B0021187807F0F0FB284900946F
:103DA800284B0968284800220FF0EEFF264810F03B
:103DB80097F8FFF7D3FE254A002110200FF0E4FE04
:103DC800234A00214FF480700FF0DEFE214B224879
:103DD8001968224B009400220FF0D6FF1E4810F0FD
:103DE8007FF80BB0F0BD00BF85490108CC49010838
:103DF800ED4901080E4A01082F4A0108504A0108F6
:103E0800B5320008840D00207B380008500D0020D2
:103E180079380008380D0020FD3700086C0D0020A7
:103E280081B400080D3500084938000895340008A9
:103E380000000301100000205C00002000000020AA
:103E480074000020F53200089C0D0020A531000800
:103E5800213200080C000020B40D0020A53700080E
:103E680010B50024A2B07C22214603A8029410F0C9
:103E7800FBF953238DF8083040F22713ADF80A30C8
:103E880001238DF80C30ADF80440FEF7D7FD00B2E1
:103E980000EB400000EB4010FE23B0FBF3F08DF880
:103EA8000D0001A800F004FDA0B958238DF80E30CC
:103EB800072430228021144810F0D6F9224602A99E
:103EC800114810F00AFA104A21460120FFF7FCFCBD
:103ED80022B010BD430001338DF80E308DF80F006D
:103EE80000F0BEFE094B1A6812128DF810201A68ED
:103EF8008DF811205A685B688DF8133012128DF80E
:103F080012200C24D5E700BFCD0D0020F40E0020B0
:103F1800F0B50378592B95B0044640F01E82052968
:103F28005FD84378443B162B5BD8DFE813F0410198
:103F38005A0031015A0039015A005A005A005A00F1
:103F48009A005A001C015A005A005A00B9015A0036
:103F58005A00BE005A005A005A0017008578482DAA
:103F680017D1C34A14210120FFF7AEFC41F2883073
:103F7800FEF7E6FD0022BF4B114603200FF034FC8C
:103F880040F6B830FEF7DCFD15B0BDE8F040FFF7AD
:103F98003DBC532D0ED130228021B74810F064F972
:103FA800FFF75EFF41F28830FEF7CAFDB24A1521DD
:103FB80001208FE0432D16D1002404A88DF810406D
:103FC80007F012FCAC4A4C231370272393709DF81A
:103FD8001030547001204133D07013710521FFF760
:103FE80073FC15B0F0BD442DFBD1A34C59232370AD
:103FF8005A236370A57000F03DFC2C228021201DFF
:1040080010F032F900232570637001252723A3706F
:10401800E5702571FEF712FD9849FE23B0FBF3F019
:104028000B6864229BB2B3FBF2F3A3710B6800EB3D
:10403800400000EB40109BB26071B3FBF2F002FB52
:104048001033E3714B689BB2B3FBF2F323724B68F6
:104058009BB2B3FBF2F102FB1133637222460A21D1
:10406800A6E78378303BDBB2092BBAD8844C854A63
:1040780023702378DBB253727F4A592313704D2380
:10408800537023783033937003210120FFF71CFC11
:104098002378009300227C4B114601200FF0A4FBEB
:1040A80015B0BDE8F040FFF785BC8578482D16D1DE
:1040B800714A5623137000235370272393700323E8
:1040C8001371172353710B23012093710A23D070A6
:1040D800D371082115B0BDE8F040FFF7F5BB432DBB
:1040E8007FF47FAF644C00213C2205A8049110F0B6
:1040F800BBF804A8FFF7CAFC2422802104F10C00B5
:1041080010F0B2F89DF8103063709DF81130A3706C
:104118009DF81230E3709DF8133023719DF8143028
:1041280063719DF81530A3719DF81630E3719DF801
:10413800173023729DF81830257063729DF81B5054
:104148009DF81930A3729DF81A30E3722A4607A920
:10415800257304F10D0010F0C0F805F10D01224699
:10416800C9B201203BE7807839280CD83038C0B272
:10417800FFF764F8404A2378137063785370A37884
:104188009370032114E715B0BDE8F040FFF704BCB5
:1041980080783928F7D83038C0B2FFF754F8E9E703
:1041A80080783928EFD83038C0B2FFF751F8E1E706
:1041B8008378303BDAB2092AE5D8C578303DEAB2CF
:1041C800092AE0D80179A1F14802D2B20B2ADAD83B
:1041D8002E4840FA02F2D007D5D40A224D2902FB14
:1041E80003553FD13C235D43294B4FF47A70684314
:1041F8001860284B1860FFF789F81F4A2378137056
:1042080063785370A3789370E378D370237913712C
:1042180005210120FFF758FB1A4B272200261E70A4
:104228005A7001229A70DA70A178303901EB810056
:10423800E178303901EB4001C9B2197122795A711C
:10424800154A1278D2B21A720D4A1278D2B25A723C
:10425800FFF7B0FB114B00953246314603200FF0B3
:10426800C3FABEE64829BFD14FF46163BBE700BF7C
:10427800744A0108894A0108CD0D0020F40E002077
:10428800440C002078000020AB4A0108DEF7FFFF4D
:10429800740000200C000020620E0020D44A01089F
:1042A8008378303BDAB2092A3FF66DAFC578303DE6
:1042B800EAB2092A3FF667AF0179A1F14802D2B202
:1042C8000B2A3FF660AF734840FA02F2D2073FF577
:1042D8005AAF0A224D2902FB035539D13C235D43CD
:1042E8006D4A4FF47A736B4313601068FFF730F828
:1042F8006A4A2378137063785370A3789370E378CD
:10430800D3702379137105210120FFF7DDFA644B7F
:10431800272200261E705A7001229A70DA70A1783E
:10432800303901EB8100E178303901EB4001C9B245
:1043380099712279DA715B4A1278D2B21A725A4AA2
:104348001278D2B25A72FFF735FB584B009583E7C3
:104358004829C5D14FF46163C1E7502B5DD10229CB
:104368007FF63FAE4378303B012B3FF63AAE837879
:10437800312B7FF436AE0B2904D8FFF70DFB002153
:10438800464A15E6464D4A4F0234002614F8012FD6
:10439800A919303AD2B20A730B7BCDE902632378AC
:1043A8000022CDE9006311463B46032001360FF099
:1043B8001BFA0C2EEAD1FEF76DFF384B50221A700B
:1043C80027229A70002401225C70DA7003F8042F07
:1043D8002A190134127B0C2C02F1300203F8012F48
:1043E800F6D100225023114600930320314B0FF0E1
:1043F800FBF900232B7027236B700123AB70EB7044
:10440800284B1B78DBB22B72274B1B78DBB26B7205
:10441800EC72FFF7CFFA1121B2E7412B7FF4E1AD3F
:104428004378432B7FF4DDAD16297FF4DAAD224DB6
:10443800421C002312F8011FE9540133142BF9D14F
:10444800FEF77CFE1D4B5B7D012B19D1144900231F
:10445800EA5CC8180133D2B2142B80F82C20F7D1AB
:10446800114B00221A701B78DBB24B72FFF7A2FACD
:104478000A4A631E15349C4206D1084A162197E55C
:10448800094B02221A70F3E713F8011F02F8011B07
:10449800F1E700BFDEF7FFFF0C000020CD0D002084
:1044A80078000020620E0020440C00200B4B01080D
:1044B800564B01087E4B01084E0E0020B40A00201E
:1044C80070B5054686B00C4600293BD028480FF049
:1044D80007FD2678EEB1002D48D068682E78C0B167
:1044E800032E0BD0392E2FD0022E12D16978012934
:1044F8000FD00B060DD4FFF70BFD0AE06B78012BEC
:1045080007D10078012802D0022800D008B906F0A7
:10451800EBFF237C052B15D894F90A20059294F912
:1045280009200492134A52F82330039394F908306F
:10453800CDE901630022E368009311460E4B032086
:104548000FF052F906B070BD6B78012BE1D10278FB
:104558000A4B02F001021A702AB9094B11460320CE
:104568000FF042F9D5E7074B0022F7E72E46D0E7D0
:10457800500D0020044C0108AC4B0108370D0020F9
:10458800994B0108A34B0108034B0022C3E90222FF
:104598000122C3E900227047640E002000487047DA
:1045A800640E00204FF0B04382B0DA6C0243DA6444
:1045B800DB6C03400193019B02B070472DE9F04189
:1045C80086B000240220154D0594FFF7EBFF042068
:1045D800FFF7E8FF124F03944FF4807601230DEBA9
:1045E8000001CDE901632846032304934FF40058E2
:1045F80003F0E4FE01A93846CDF8048003F0DEFE9E
:1046080022464146384603F0FFFF284622463146F7
:1046180003F0FAFF204606B0BDE8F0810004004828
:1046280000080048032810B50ED8012810D868B92A
:1046380002460B484FF4807103F0E6FF0022094858
:104648004FF4005103F0E0FF002010BD0122F0E715
:10465800002203484FF4807103F0D6FF0122EEE7F1
:1046680000040048000800480220704700207047F6
:104678000120704700280CBF0F201620704700004B
:104688000D48854602F0B6FE0C480D490D4A002338
:1046980002E0D458C4500433C4188C42F9D30A4AEF
:1046A8000A4C002301E013600432A242FBD30FF04E
:1046B800E3FDFDF7EBFFFEE700000120000000200E
:1046C800CC080020A8590108CC080020382E00206A
:1046D800FEE74FF0B04382B0DA6C42F00102DA64D0
:1046E800DB6C03F001030193019B02B070470000EB
:1046F80030B587B0FFF7EDFF4FF4805101224FF03E
:10470800904003F081FF01224FF400614FF0904088
:1047180003F07AFF4FF4C0551123CDE9015301A9E5
:1047280001234FF09040039303F048FE08240A2524
:1047380000224FF480514FF0904003F065FF0120B4
:10474800FEF7FEF901224FF480514FF0904003F03C
:104758005BFF0120FEF7F4F9013DE9D14FF4006158
:104768004FF0904003F04AFF08B9013CDFD14FF405
:1047780000614FF0904003F041FF68BBFFF7A9FFCD
:1047880004240123039001A92A48CDE9014303F039
:1047980015FE284C01220421204603F035FF212074
:1047A800FEF7CEF900220421204603F02DFF212038
:1047B800FEF7C6F901220421204603F025FF212037
:1047C800FEF7BEF920460022042103F01DFF4FF436
:1047D8002570FEF7B5F9DDE7FFF77BFF4FF0B04333
:1047E80000249A6D42F480029A659B6D03F480035D
:1047F80000934FF4C052009B1223CDE901230323F9
:10480800CDE9034304230DEB03014FF090400593DA
:1048180003F0D4FD08480949094B8460C0E9001336
:104828000123C0E90334C0E90744446104F060F897
:1048380007B030BD00040048740E00200058004046
:104848001A091020FFF754BF10B1012809D070478A
:1048580001394A424A414FF090404FF4007103F049
:10486800D3BE4B1E5A4202485A410821F7E700BFFF
:104878000004004808B50120FEF7E0FC6420FEF7BC
:104888005FF900F0EDF9BDE808400120FEF7DBBC58
:10489800054B1A6802805A689B684381034B028162
:1048A80001221A70704700BFF40E00204D0E002040
:1048B80037B5044600F016F810F0FF051CBFEE23CC
:1048C8002370AA2363700193002223780093114672
:1048D800034B01200EF088FF284603B030BD00BF0F
:1048E8001C4C01082DE9F04F0025484E484C356016
:1048F80089B029462846FFF7A7FF29460120FFF778
:10490800A3FF29460220FFF79FFFDFF80881DFF8A1
:104918000891424F94F86401522301214FF0000A94
:1049280084F86031C4F868A1FFF78EFF0320FEF712
:1049380007F952468821204602F0C2FC0DF11E02FA
:10494800C021204602F00AFD024650B1344B5246BF
:10495800114603200EF048FF0021E8B2FFF774FF6C
:104968003DE0BDF81E304EF6AA618B424AD14FEAAF
:10497800450A0AF1540A5FFA8AFA05905146204618
:1049880000F004FA834610B1264B059AE0E70DF1D2
:104998001E02C021204684F860A102F0DFFC824696
:1049A80010B1214B5A46D3E7204600F0B3FB02462C
:1049B800F0B931680123194431603968C4F86831A5
:1049C800AB400B433B60029394F860310193D4F8F9
:1049D800643100930146154B03200EF005FF0135A5
:1049E800032D04F5C87495D1306809B0BDE8F08F7F
:1049F800BDF81E30009352464B46114603200EF078
:104A0800F3FEA9E700934346F7E700BFEC0E00204A
:104A1800BC000020E34C0108C84C0108E80E002047
:104A2800314C0108434C0108664C01087F4C0108D1
:104A38002DE9F04F4FF4804387B04FF49012CDE941
:104A48000232684CDFF8A0A1DFF8A0B105464FF0AC
:104A58000A094FF00E0848F2E8070026D4F8683132
:104A6800002B00F0AE800022614B00961146032017
:104A78000EF0BAFE204600F041FE28B100225D4B40
:104A8800114603200EF0B0FE0DF112020DF11101D6
:104A9800204600F0EDFB28B10022534611460320C2
:104AA8000EF0A2FE0DF1130205A9204600F02BFF1F
:104AB80028B10022504B114603200EF095FE00212C
:104AC800204600F067F928B100224C4B114603201C
:104AD8000EF08AFE01220021204600F01FFA28B1BC
:104AE8000022474B114603200EF07EFE012211469C
:104AF800204600F013FA28B10022414B114603204A
:104B08000EF072FE022D65D83E4B33F81530029335
:104B18003D4B53F8253003933C4B53F825703C4BE1
:104B280013F805803B4B13F80590029A01212046A3
:104B380000F03FFA28B10022374B114603200EF04F
:104B480053FE039A0021204600F033FA28B10022D0
:104B5800314B114603200EF047FE3946204600F03F
:104B680033F928B100222D4B114603200EF03CFEEC
:104B780042460021204600F029F928B100225B4670
:104B8800114603200EF030FE4A460121204600F06F
:104B98001DF928B100225B46114603200EF024FEC1
:104BA8000DF112020DF11101204600F061FB28B150
:104BB80000225346114603200EF016FE0123C4F8C6
:104BC8007C310136032E04F5C8747FF447AF07B073
:104BD800BDE8F08F0022124B114603200EF004FEB0
:104BE800A3E700BFBC0000203A4D0108334E01087E
:104BF800F54C01081F4D0108604D0108894D010859
:104C0800A74D01080E4F0108144F0108204F010855
:104C18002C4F01082F4F0108D94D0108FC4D010800
:104C2800CB4D010810B50B7E9BB9D0F87C210989C2
:104C380012B1C0E95E1310BD084BD0F878411A686C
:104C4800C2F580734B4304FB02331B12C0F8783162
:104C5800F1E70123C0F87C31EDE700BFB800002080
:104C68002DE9F04FDFF80091404E87B0FFF7EAFDDD
:104C7800D9F800300BB133684BB9FFF733FE002287
:104C880030603B4B0090114603200EF0ADFD3368B9
:104C9800384D0024A3422C606C60AC6055DDDFF811
:104CA800D880364EDFF8D8A00220FFF7C1FE88F87A
:104CB8000040D6F868B1BBF1010F2FD10BFA04F30D
:104CC80004930A272E49304600F078FCC0B90590B5
:104CD80051463046FFF7A6FF9AF81830059ABBBB35
:104CE800D6F8783145F82430049AD9F800301343BF
:104CF800C9F8003098F8003043F0010388F8003014
:104D08000120FDF71DFF9AF818304BB3013F17F04B
:104D1800FF07D7D14FF47A7345F8243005200134C2
:104D2800FDF70EFF032C06F5C876C2D198F80030BF
:104D38005BB12B686A68A9680093CDE9012100225C
:104D4800104B114601200EF04FFD07B0BDE8F08F63
:104D5800CDE9004B0C4B114603200EF045FDCFE783
:104D6800D6F87831D8E700BFE80E0020F00E002012
:104D7800CF4E0108F40E00204D0E0020BC0000208C
:104D8800CC0E0020804E0108ED4E01084A088A2109
:104D980002F096BA152906D8044BCB40DB0702D59A
:104DA8000174002070476FF0070070470B00300057
:104DB80010B50A460C46092102F0A4FA18B923785E
:104DC80003F00103237010BD01F06BBE01F053BD69
:104DD80001F04DBEF7B500230C46174601210DF131
:104DE800070206468DF8073002F08CFA0546D8B956
:104DF800012F9DF8073026D1042C3AD8DFE804F0BB
:104E080003171A1D200043F01004A3420CD02246B9
:104E18000121304602F054FA054628B9716986F82E
:104E280030413046FFF7D0FF284603B0F0BD43F0CD
:104E38002804EAE743F00404E7E743F04004E4E722
:104E480043F08004E1E7042C13D8DFE804F00306FC
:104E5800090C0F0003F0EF04D7E703F0D704D4E7F9
:104E680003F0FB04D1E703F0BF04CEE703F07F04AF
:104E7800CBE76FF00305D7E713B500230C460DF118
:104E8800070201218DF8073002F03CFA78B99DF845
:104E98000730C3F300122270C3F3C002A270C3F339
:104EA80080026270C3F38012DB09E270237102B0E2
:104EB80010BD37B50D460DF10202F821044602F087
:104EC8004DFA70B901AA0421204602F067FA40B9E8
:104ED800BDF802201AB1019BB3FBF2F32B602B68DB
:104EE800A36103B030BD037F0B700020704737B556
:104EF8000D460DF106022021044602F02FFA28B9CA
:104F0800BDF8063023B9236A2B60207703B030BD83
:104F1800DB002B60236201232377F7E70529F8B527
:104F280004460E46154635D862B100EB81030121CF
:104F38005A6B0023701E042807D8DFE800F00E170C
:104F48001A1D240011460123F4E784F8281034447C
:104F5800E5B984F82850002007E0C2F34F22442125
:104F6800204602F0BDF90028F1D0F8BD84F82A10D7
:104F7800EDE784F82B10EAE75B00FE22602120466B
:104F880002F0D5F9EFE71B01EF22F7E7012384F8D8
:104F98002830E0E76FF00300E7E7052996BF4018DF
:104FA800002390F82830137094BF00206FF003009E
:104FB800704770B54318044693F828000E46154606
:104FC80018B904EB8106726370BD05291BD8DFE8A8
:104FD80001F0030912141616626304EB860400201C
:104FE8006563F1E7C2F34F224421204602F078F9C5
:104FF8000028E9D1F1E7E263EFE72264EDE7C2F3C5
:105008004F226421F1E76FF00300DDE737B504466E
:10501800154605292CD8DFE801F0030717191B1BD3
:10502800436B2B60002021E00DF10602442102F0C1
:1050380095F9D8B9BDF8062053029AB12B60A3633D
:10504800012384F8293011E0C36BEAE7036CE8E731
:105058000DF10602642102F081F938B9BDF8063075
:105068005B02DEE7A36B2B6084F8290003B030BD38
:105078006FF00300FAE737B50D460DF1070201217D
:10508800044602F03FF938B99DF8073084F830310A
:10509800DB092B7084F84C3003B030BD2DE9F843A0
:1050A800037C0C4601F8083B0546FFF702FF40BBAE
:1050B800207304F110012846FFF719FF08BB04F11B
:1050C8001401284600F021FCD8B904F1240705F1A1
:1050D800270904F1170806463A46B1B22846FFF7F1
:1050E80095FF70B9013619F8013F08F8013F062EFF
:1050F80007F10407F0D104F13C012846FFF7BBFF94
:1051080008B1BDE8F883211D2846BDE8F84301F041
:1051180030BD0000F0B50022054693B0882102F0AA
:10512800CFF84FF47A72A5F852214FF4C872A5F857
:1051380054214C4AC5F8582100234B4A85F8F030D1
:10514800C5F8D4202B6202A92846FFF7A7FF04461A
:1051580070B9ADF8080002AE0FCE05F110070FC701
:105168000FCE0FC70FCE0FC796E80F0087E80F00C6
:105178003E4BC5F834314FF4FA730126A5F838319F
:105188004FF42063A5F83C313246802185F8506100
:10519800284602F095F832460746FF21284602F0D5
:1051A8008FF8002211460743284602F089F83C434D
:1051B80064B204430DF107029121284602F0A2F8D7
:1051C80064B29DF8073085F83A310443324600212D
:1051D800284602F075F864B204430022FF212846ED
:1051E80002F06EF864B2044300228021284602F0DF
:1051F80067F864B2204340B2002488BBA1B2012200
:1052080028460134FFF78AFE062CF6D140BB044637
:105218006885024604212846FFF780FE00BB024647
:1052280005212846FFF77AFED0B94FF490136B6337
:105238004FF4804201212846FFF7BBFE80B94FF4A6
:105248000C13FF22C5E90F3085F8302101212846CB
:1052580002F036F8012385F8323108B985F815418E
:1052680013B0F0BD856B0100A470090064008403CD
:10527800012300F079BD2DE9F0428EB00C460C23D5
:1052880004AA1421054602F005F8844600286CD1CA
:105298009DF81A309DF81B609DF817209DF818108E
:1052A800A07506EB03269DF81630206002EB03225A
:1052B8009DF81930606003EB01239BB25B029DF8F7
:1052C800121023619DF81330B5F8520103EB012346
:1052D80092B252029BB2E260A382B0F57A7F9DF847
:1052E800101095F83171B6B20AD0704300F5FA7013
:1052F8004FF47A76B0FBF6F02E7F002E39D186B2C5
:10530800002F40D0B001C0B2B608E0750DF10F0013
:105318002681CDE90040284601F086FE844620BB60
:105328009DF80FE084F818E005F150060FCE07AF9E
:105338000FC796E80700E37D87E80700D4E9030173
:10534800A28AADF83020D4E90149CDE90A01CDE9B6
:10535800084907AC8DF833308DF834E00FCC503560
:105368000FC597E8070086E8070060460EB0BDE85D
:10537800F0822E8C5E43B2EB262F4FEA262C04D106
:1053880057B948F6E0260020BFE780B25043A2EBA9
:105398000C06B0FBF6F0B2E742F2B826B2E700001E
:1053A800F7B517460E210DF106021D460B4C0646B1
:1053B80001F0D4FFBDF8063004EA43433B6050B91E
:1053C8000DF106020C21304601F0C8FFBDF8063089
:1053D80004EA43442C6003B0F0BD00BF0000FE1F88
:1053E80073B590F8DA30013B022B06460C4634D8E8
:1053F80001AB6A460121FFF7D3FF009BB3F57F0F8E
:10540800054603D8019BB3F57F0F23D915BB34B1EB
:105418001349304602B0BDE8704001F00FBC0422C9
:10542800FF21304601F04CFF2A46044670213046E1
:1054380001F046FF2A460443FF21304601F040FFB1
:1054480064B204432A468021304601F039FF64B231
:10545800044365B2284602B070BD0025FAE700BFD4
:105468005F06002037B5044601228021057C01F043
:1054780027FF0122FF21204601F022FF00221146CA
:10548800204601F01DFF94F83A219121204601F0B1
:1054980017FF01220021204601F012FF0022FF2100
:1054A800204601F00DFF00228021204601F008FF70
:1054B800012D29D0032D37D0002D3CD101222946BA
:1054C800204601F0FDFE01238DF80730A0B103B09E
:1054D80030BD01460DF10702204601F013FF9DF88B
:1054E8000730DB0705F1010508D538B9B5F5FA6FBE
:1054F800EFD16FF00600EAE70546F0E7B5F5FA6F79
:1055080008BF6FF00600E2E718B929462046FFF702
:1055180067FF02220021204601F0D2FE0028D6D1E2
:10552800042384F83231D2E718B901212046FFF765
:1055380057FF0422EEE76FF00700C8E738B5057C8F
:10554800044625B1204600F054FD28B138BDFFF7C8
:1055580089FF0028F6D0F9E7002DF7D1032384F856
:105568003231F3E773B50646002501220B21304698
:1055780001F0A6FE002204460B21304601F0A0FEF1
:105588000DF1070204431321304601F0BBFE9DF8DC
:10559800073064B2044301355B0760B2EDB205D051
:1055A800032D08D00028E0D002B070BD032D08BF3D
:1055B8006FF00B00F8E76FF00B00F5E738B5002344
:1055C800037404460D46FFF7B9FF50B92946204633
:1055D800FFF751FE28B901462046BDE83840FFF7DD
:1055E800C1BF38BD152970B5054616461C4667D19A
:1055F8000122FF2101F064FE0022114604462846DC
:1056080001F05EFE00220443FF21284601F058FE07
:1056180064B2044301228021284601F051FE64B29D
:10562800044302228521284601F04AFE64B204435D
:105638000422FF21284601F043FE64B204430022FD
:10564800CD21284601F03CFE64B204431122CC214E
:10565800284601F035FE64B204430722FF2128469C
:1056680001F02EFE64B204430022BE21284601F058
:1056780027FE64B204430622FF21284601F020FEDB
:1056880064B204430922CC21284601F019FE64B211
:1056980004430022FF21284601F012FE64B20443AD
:1056A8000122FF21284601F00BFE64B200220443C8
:1056B8001146284601F004FE64B2204340B270BD92
:1056C800042A17D80A2101F0FBFD0028F7D1231E70
:1056D80018BF01231B01EF228421284601F027FE71
:1056E8000028ECD185F8DA6001462846BDE870400C
:1056F800FFF738BF6FF00A00E1E7000070B594B01B
:1057080005464022002104A80EF0AEFD0023012129
:105718002846ADF806308DF803308DF80430029332
:1057280000F0B8FC95F8142195F81311012A04D853
:1057380040F0AD80202940F2AC8001AA02A9284699
:1057480000F02DFB0446002840F09E8095F850316B
:10575800002B40F0A280D5F84C11284601F06EFAD3
:105768000446002840F0908023462146042228461B
:10577800FFF738FF0446002840F086800122FF2109
:10578800284601F09DFD0DF10602064684212846B3
:1057980001F0E4FD22460643FF21284601F090FD72
:1057A80076B2064374B2002C6ED1BDF806301B01E8
:1057B800C5F8D43004A92846FFF770FC0446002831
:1057C80062D10DF103012846FFF7F2FA04460028DA
:1057D8005AD19DF8033085F8313104AE0FCE05F16A
:1057E80010040FC40FCE0FC40FCE0FC496E80F00DD
:1057F80084E80F000DF103020121284601F082FD23
:105808000446002840D19DF8033085F8303102461F
:1058180001462846FFF7DEFA0446A8BB02460221E5
:105828002846FFF7D7FA044670BB0323014685F8DC
:1058380032310DF10502284601F019F9044618BB6A
:105848009DF8053085F8E8300DF10502012128465C
:1058580001F00DF90446B8B99DF8053085F8E03037
:1058680003AA0321284600F001FF044660B9039B00
:10587800C5F8E43003AA0421284600F0F7FE0446E0
:1058880010B9039BC5F8DC30204614B070BD0C2954
:1058980051E7284600F010F954E701495DE700BFD9
:1058A8006C05002013B50C460DF10702132101F019
:1058B80029FD9DF8073013F0180F03F0070218BFF1
:1058C8006FF00500226002B010BD13B590F8DA3011
:1058D800042B0C460BD101A9FFF7E4FF019B042B15
:1058E80001D1012300E00023237002B010BD01AAFA
:1058F800142101F007FD0028F7D19DF80430DB07DB
:10590800EFD42070F1E700F04ABA13B50C460DF158
:105918000602282101F022FD78B9BDF80620C2F35D
:105928000B0312F4006F18BFA3F580534FF0FA026F
:1059380014BF13FB02F35343236002B010BDF0B54C
:105948004FEAD20C4FF0FF341C6002F007026646A3
:1059580000278E4200D207B1F0BD845D664503BFC3
:105968001441E4B215463D4614F0010704D005EB96
:10597800C6051D600136ECE70135082D4FEA5404D1
:10598800F2D1F7E7034B800953F82000003818BF1D
:10599800012070471808002010B5B1EBD20F4FEA6C
:1059A800D20402F0070381BF01229A40035D13432A
:1059B8008ABF03556FF03100002010BD0A46062348
:1059C800B02101F049BC0A460623B02101F062BCAF
:1059D8002DE9F04F85B08046109E0E9D01968A46AF
:1059E80093461C464FF00009119B994508D10023A6
:1059F800129A1660F3B16FF0310005B0BDE8F08F70
:105A080001AB324629465846FFF799FF019F7B1C98
:105A18000DD00F9BF818FFF7B5FF504507D13A4650
:105A28002046FFF7B9FF7E1C09F10109DCE76FF09A
:105A38003103DDE721464046FFF7C0FF0028DCD1EF
:105A480002A94046FFF7BFFF2544234602AAAB42FE
:105A5800D3D013F8014B12F8011B8C42F7D0CAE7D8
:105A680070B5C02288B00E46012190F83041054635
:105A780001F026FCF0B901A92846FFF79FFDC8B937
:105A88000122FF21284601F01BFC98B93246B621B5
:105A9800284601F063FC68B90246FF21284601F058
:105AA8000FFC38B922460121284601F009FC08B943
:105AB80085F8304108B070BDF0B50F4689B016467C
:105AC800FF210122044601F0FBFB0246A8B94F2141
:105AD800204601F0F5FB80B92C224E21204601F02A
:105AE800EFFB024648B9FF21204601F0E9FB20B947
:105AF800B422B621204601F0E3FB0025C4F8245166
:105B0800A4F82851DEB9354607ABB422CDE90373B2
:105B18000623CDE90032029504F5927304F59572D7
:105B280031462046FFF754FF30B9012384F8153178
:105B380084F8137184F8146109B0F0BD013505F1DA
:105B4800B400FFF71FFF0028DED12C2DF6D1DBE7CC
:105B580010B541F001020021044601F0B1FB78B90B
:105B6800204600F046FA58B901462046FFF7FAFCED
:105B780030B9024601462046BDE8104001F0A0BBFE
:105B880010BD2DE9F74F4FF0000B88461746FF214F
:105B9800012205461E469DF838A09DF83C908DF8D8
:105BA80007B001F08DFB5A4604465946284601F0D5
:105BB80087FB5A460443FF21284601F081FB64B263
:105BC800044364B2B8F1000F32D0BAF1000F06D026
:105BD8000C9ACB21284601F095FB204344B2B9F139
:105BE800000F07D00DF10702EE21284601F08AFBCD
:105BF800204344B20122FF21284601F061FB012223
:105C080004430021284601F05BFB64B204430022F0
:105C1800FF21284601F054FB64B29DF807300D9A25
:105C2800204323F0100340B2137003B0BDE8F08F97
:105C3800BAF1000F06D03A46CB21284601F040FBC6
:105C4800204344B2B9F1000FD4D033468022EE216C
:105C5800284601F06CFBCBE72DE9F04387B091466D
:105C68000022054688468DF817201E461BB390F87B
:105C7800307101221146284601F022FB044658BB28
:105C880040212846FFF764FF044628BBB9F1010FFD
:105C980013D10DF11703CDE90290CDE90083024637
:105CA800034649462846FFF76CFF40B104462046A4
:105CB80007B0BDE8F0831F46DBE788F80000002E38
:105CC800F5D03A460121284601F0FAFA04460028A0
:105CD800EDD185F83071EAE7002388F800302046D6
:105CE800E4E72DE9F043054687B0884691461E460D
:105CF80023B390F8307102220121284601F0E0FA1E
:105D0800044660BB01462846FFF722FF044630BB25
:105D1800B9F1010F14D10DF11703CDE90209009370
:105D280002460346CDF8048049462846FFF729FF76
:105D380040B10446204607B0BDE8F0831F46DAE7C5
:105D480088F80000002EF5D03A460121284601F0D7
:105D5800B7FA04460028EDD185F83071EAE7002348
:105D680088F800302046E4E7F8B51D4616460023BB
:105D78002A4690F830710446FFF76EFF70B9034663
:105D88002A4631462046FFF7ACFF38B93A4601218A
:105D9800204601F095FA08B984F83071F8BD2DE96C
:105DA800F04F002393B0CDE90A12C0F82431A0F8CF
:105DB80028310122FF21CDE90E33B0F83C818DF85E
:105DC800343005468DF8353001F07AFA044600285B
:105DD80040F0E38002464F21284601F071FA04465C
:105DE800002840F0DA802C224E21284601F068FA7B
:105DF8000446002840F0D1800246FF21284601F0E1
:105E08005FFA0446002840F0C880B422B62128462C
:105E180001F056FA0446002840F0BF80024680216F
:105E2800284601F04DFA0446002840F0B6800346A3
:105E38000DF135020DA92846FFF796FF0446002804
:105E480040F0AB800323CDE90203B421062305F516
:105E5800957A05F592790EAECDE9003104960146A2
:105E68004B4652462846FFF7B3FD0446002840F04B
:105E780094800DF1360128460E9FFFF7F1FD044688
:105E8800002840F08A80BDF83630434540F2AA80A9
:105E9800C5F82401A5F8280107F1B400FFF772FD41
:105EA80008B92B2F7DD90623B4224FF0030BCDE977
:105EB8000032CDE9027B04964B4652460121284622
:105EC800FFF786FD002840F08B800DF1360128464B
:105ED8000E9FFFF7C5FD064600287CD1BDF8363079
:105EE800434540F2828001260696BDF83630434588
:105EF80060D2A3EB080383EAE372A2EBE3729DF896
:105F08001860099205F592734FF0030B0793079BEE
:105F180018689B881090ADF844303A460FAB0621BC
:105F28005046FFF70CFD0F9F7B1C56D007F1B400BD
:105F3800FFF728FD069B98423CD10BF101033A4636
:105F480048460893FFF728FD002849D149462846C6
:105F5800FFF734FD002843D10DF136012846FFF73D
:105F68007FFD00283CD1BDF83620A2EB0803002BAA
:105F7800B8BF5B42424516D9099A934218D910A96D
:105F88002846FFF71BFD079A0799034610981060EB
:105F9800BDF844208A806BB11C46204613B0BDE88A
:105FA800F08F013778E7DDF820B009930137AEE7C5
:105FB800DDF820B00A9BC3F800B00B9B1E700123CC
:105FC80085F815310A9B1B6885F813310B9B1B78E4
:105FD80085F81431E1E70446DFE76FF03104DCE7C8
:105FE8000446DAE70026B3467EE701238346069394
:105FF8007BE737B5002304468DF807304FF4FA6580
:106008000DF107012046FFF760FC58B99DF80730ED
:10601800012B07D0013D03D0204601F0E5F9EFE759
:106028006FF0060003B030BD02464FF08043934244
:1060380002D8002013B970479B08F8E7C1189142AD
:106048004FEA50009CBFC018521A9B08F2E773B57C
:1060580000228321054601F033F9044688B94FF43C
:10606800FA660DF107028321284601F04BF99DF8E5
:1060780007300343DBB204461BB9013EF1D16FF090
:10608800060401228321284601F01AF9204340B270
:1060980002B070BD2DE9F04F90F8F06091B04FF06C
:1060A8000009072ECDE9079904460F4600F0A282A1
:1060B8000122802101F004F901228046FF212046B7
:1060C80001F0FEF84A4648EA00084946204601F031
:1060D800F7F84FFA88F848EA00080622FF21204618
:1060E80001F0EEF84FFA88F848EA00080DF11502B9
:1060F8008321204601F006F99DF815204FFA88F80B
:1061080048EA000842F004028321204601F0D8F84A
:106118004FFA88F848EA00080722FF21204601F0D4
:10612800CFF84FFA88F80122812148EA0008204672
:1061380001F0C6F84FFA88F848EA0008204601F04E
:1061480053F94FFA88F848EA0008012280212046CE
:1061580001F0B6F84FFA88F848EA000517F0010B85
:106168006DB200F01E82F20700F11E826B229421AC
:10617800204601F0A5F880462046FFF768FF06AAEA
:1061880048EA00089021204601F008F945EA080588
:10619800069B6DB22422942105432046C3F3062AA8
:1061A800C3F3C03901F08CF86DB205432046FFF700
:1061B8004EFF6DB2054306AA9021204601F0EEF885
:1061C800069B6DB21BBA25229421054320460993EC
:1061D80001F076F86DB205432046FFF738FF6DB23F
:1061E800054306AA9021204601F0D8F8069B6DB217
:1061F8001A0E05431B0C6DB28DF828208DF8293036
:1062080017F00203029300F0DB8016F0020840F05A
:10621800D78002229421204601F052F801902046AE
:10622800FFF715FF019B0DF116020343902120464D
:106238001D4301F067F86DB27B2294210543204687
:1062480001F03EF86DB205432046FFF700FF6DB23E
:1062580005430DF117029021204601F053F86DB265
:10626800772294210543204601F02AF86DB20543B0
:106278002046FFF7ECFE6DB2054306AA90212046A2
:1062880001F08CF8069B5A0E8DF82C20C3F3864239
:106298008DF82D20C3F3C6228DF82E206DB2C3F3DE
:1062A8000612DB0003F07803942105438DF82F20B4
:1062B800204678228DF8153001F002F86DB20543BA
:1062C8002046FFF7C4FE6DB2054306AA902120467A
:1062D80001F064F8069B9DF8152002EB53728DF8C7
:1062E8003020C3F386528DF83120C3F3C6328DF8BF
:1062F8003220C3F306228DF833206DB2C3F3460271
:106308009B0103F04003942105438DF83420204677
:1063180079228DF8153000F0D3FF6DB20543204681
:10632800FFF795FE6DB2054306AA9021204601F0BD
:1063380035F8069B9DF8152002EB93628DF8352001
:10634800C3F3C6428DF83620C3F306328DF83720E2
:106358006DB2C3F346129B0003F07C0394210543FE
:106368008DF8382020467A228DF8153000F0A8FFE5
:106378006DB205432046FFF76AFE6DB2054306AAD3
:106388009021204601F00AF8069B9DF815208DF80B
:106398003E8002EB93728DF83920C3F3C6526DB27A
:1063A8008DF83A20C3F3064205438DF83B20C3F32A
:1063B8004622C3F386036DB28DF83C208DF83D303C
:1063C80017F00403019300F0F180730700F1EE80E9
:1063D8007B229421204600F073FF80462046FFF779
:1063E80036FE07AA48EA00089021204600F0D6FFAA
:1063F80045EA08084FFA88F848EA00057C22942103
:10640800204600F05DFF6DB205432046FFF71FFEF2
:106418006DB2054308AA9021204600F0BFFF6DB277
:10642800732294210543204600F04AFF6DB20543CC
:106438002046FFF70CFE6DB2054306AA90212046C0
:1064480000F0ACFF069B6DB21B0274229421054339
:1064580020461FFA83F800F033FF6DB2054320464B
:10646800FFF7F5FD6DB2054306AA9021204600F01E
:1064780095FF6DB29DF81B30752294210543204687
:1064880043EA080800F01CFF6DB205432046FFF7F9
:10649800DEFD6DB2054306AA9021204600F07EFF7E
:1064A800069B6DB21B029BB27622942105432046BF
:1064B800039300F005FF6DB205432046FFF7C7FDC3
:1064C8006DB2054306AA9021204600F067FF6DB221
:1064D8009DF81B20039B05436DB2134300228121C5
:1064E8002046039300F0ECFE06220543FF212046D8
:1064F80000F0E6FE6DB205430DF11502832120463A
:1065080000F000FF9DF815206DB2054302F0FB0274
:106518008321204600F0D4FE6DB205430122FF21FD
:10652800204600F0CDFE6DB2054301220021204631
:1065380000F0C6FE6DB205430022FF21204600F0A0
:10654800BFFE6DB2054300228021204600F0B8FE50
:106558006DB205436DB2039BFDB9BBF1000F29D1A4
:10656800029AAABB019AAAB1720713D4079AC4F86F
:106578001821089AC4F81C214FEA4822C4F820219F
:106588003BB1A3F5C8534FF47A7253431B095B42DE
:106598001BB2E3603E4384F8F060284611B0BDE8C2
:1065A800F08FD946DA462BE6CA4629E64FF00008AE
:1065B800434693E7F007D3D40998BDF8282084F818
:1065C80013A184F81491C4F82A01A4F82E21C7E76E
:1065D800B107C7D49DF8162084F8F1209DF817203C
:1065E80084F8F2200BA904F1F30002930DF068FE81
:1065F800029BB7E74D46D0E750B10138002330F091
:10660800FF019AB203F1010303D100EB022080B22B
:1066180070474008F3E7C3B2000A03FA00F00130FC
:1066280070470000084B5A434FF47A7302F5FA7228
:106638004FF4FA60B2FBF0F0B2FBF3F203FB010097
:10664800B0FBF2F0704700BF002F3A00064B5A43E8
:106658004FF47A7002F5FA72B2FBF0F24A4302F58F
:10666800FA72B2FBF0F07047002F3A002DE9FF41B3
:1066780002294FF00005074616468DF80350ADF87D
:1066880004501CD80DF102022946FEF7A1FB04466E
:1066980030B90DF103024621384600F033FE0446B6
:1066A8009DF80300FFF7B7FF81B29DF80220384636
:1066B800FFF7CCFF3060204604B0BDE8F081032925
:1066C80018D10DF102022946FEF782FB0446002884
:1066D80046D101460DF102023846FEF779FB044621
:1066E80028B901AA5121384600F038FE0446BDF801
:1066F8000400D7E7042935D102A9FEF7BDFB9DF8B0
:106708000B30ABB10DF1020229463846FEF760FBAB
:10671800044658B901AA5121384600F01FFE044624
:10672800BDF80400FFF777FF85B214B1002015E02B
:106738001D460DF1020201213846FEF749FB0446C9
:106748000028F3D10DF106027121384600F006FE4B
:106758000446BDF80600FFF75EFF80B2401BA3E7C2
:106768002846A7E728462C46A4E7F0B5022985B0B5
:10677800054616461ED80DF105020021FEF728FB36
:106788000446A0B99DF8052031462846FFF74AFF80
:1067980083B2B3F5807F9ABF00F1FF32D2B2FF22F5
:1067A800A5F8D8204621284600F08AFD0446204650
:1067B80005B0F0BD03291FD10DF105020021FEF738
:1067C80007FB9DF80520314604462846FFF72AFFB7
:1067D80080B2FFF711FF0246ADF80600A5F8D80011
:1067E800002CE4D15121284600F07AFD0446002807
:1067F800DDD1C5F8E460DAE7042939D102A9FEF74A
:106808003BFB9DF80B70B7B10DF10502002128463E
:10681800FEF7DEFA04460028C9D10DF1060251211F
:10682800284600F09BFD0446BDF80600FFF7F3FE7E
:1068380087B2002CBBD10DF1050201212846FEF7D5
:10684800C7FA04460028B2D19DF8052031462846EB
:10685800FFF7E8FE3844FFF7CFFE712102462846CD
:1068680000F03EFD04460028A1D1C5F8DC609EE793
:106878006FF003049BE7F0B585B000238DF8033073
:10688800D30705460F46164605D439B9A2F10C03BD
:10689800DAB2062A11D96FF00300E6E0012921D106
:1068A800A2F10803DAB2062AF5D8062B1AD8DFE8CF
:1068B80003F03B1969198A199D00062B12D8DFE8E5
:1068C80003F004112D112F113100182257212846E9
:1068D80000F0F6FC08225621284600F0F1FC0028BA
:1068E80040F0C3807408013CE4B2002F00F09180AE
:1068F800012FD0D101AA04212846FFF7B7FE50B9CD
:1069080022467021284600F0DBFC20B9019A0421B8
:106918002846FFF72AFF85F8E06099E03022D5E79E
:106928004022D3E75022D1E71022482100F0C8FCCA
:1069380008224721284600F0C3FC022204463221DF
:10694800284600F0BDFC0C2204433021284600F004
:10695800B7FC64B204430122FF21284600F0B0FCD2
:1069680064B2044364B230223021284600F0A8FC07
:1069780000220443FF21284600F0A2FC64B2204311
:1069880040B2ACE72822482100F09AFC08224721AF
:10699800284600F095FC032204463221284600F0E0
:1069A8008FFC044364B209223021284600F088FC99
:1069B80001220443FF21284600F082FC64B204430C
:1069C80064B22022D0E73822482100F079FC08225E
:1069D8004721284600F074FC032204463221284649
:1069E80000F06EFC044364B20822DDE74822114639
:1069F80000F066FC08224721284600F061FC0322CB
:106A080004463221284600F05BFC044364B20722A6
:106A1800CAE702AA03212846FFF728FEB0B903AA4D
:106A280002212846FFF722FE80B922465021284637
:106A380000F046FC50B9029A03212846FFF795FE5C
:106A480020B9039A02212846FFF78FFE85F8E860EF
:106A580058B969692846FEF7B7F930B902460123E3
:106A68000DF103012846FFF73CF905B0F0BD13B559
:106A7800144629B1012910D06FF0030002B010BDEF
:106A88000DF10702502100F03DFC0028F6D19DF8D9
:106A9800073001335B002370F0E70DF10702702126
:106AA800F1E7F0B5002385B04FF4FA62CDE9002391
:106AB80044F61F63994206460F4604D86FF0030553
:106AC800284605B0F0BD02A9FEF7D6F9054600280C
:106AD800F6D19DF809209DF8083013439DF80A2047
:106AE8001343A7F636341BD06A4602213046FFF717
:106AF800BDFD00283BD19DF808302BB1009B03F267
:106B08004E239C42DAD9E41A9DF80A3023B3009B3D
:106B180003F2B223B4EB430F4FEA4302CED9A41ACF
:106B28009DF80B305BB101AA03213046FFF79EFDAB
:106B3800019B03F52573A342C0D2C0B9E41A9DF89E
:106B48000C30002BBCD0A4F2262204213046FFF7DB
:106B58000CFE77610546B3E79DF80930002BDFD0BE
:106B6800009B03F525739C42A8D9E41AD8E705468B
:106B7800A6E770B54FF4FA6286B00023CDE9022388
:106B880040F636330B600C4604A90646FEF774F946
:106B98000546002836D19DF811209DF81030134382
:106BA8009DF81220134319D002AA02213046FFF79C
:106BB8005DFD002840D19DF810302BB1029B03F2F7
:106BC8004E222368134423609DF81230EBB1029BD8
:106BD80003F2B222236803EB420323609DF81330CB
:106BE800EBB99DF814305BB101AA04213046FFF7D8
:106BF8003DFD019B03F22622236813442360D8B984
:106C080023687361284606B070BD9DF81130002BCB
:106C1800E4D0029B03F5257223681344DDE703AA39
:106C280003213046FFF722FD039B03F525722368F5
:106C3800134423600028D4D00546E3E72DE9F74341
:106C4800002406460D46204615F80480B8F1000FCA
:106C580000D010B103B0BDE8F083671CB8F1FF0F96
:106C680015F8079029D1A71CEB5DB9F1030F36D8A9
:106C7800DFE809F0020B131B271D2C44E27802EB16
:106C88000323A6F834313C46DEE7271D2C44E2787E
:106C980002EB0323A6F83631F5E7271D2C44E278EA
:106CA80002EB0323A6F83831EDE7271D2C44E278E0
:106CB80002EB0323A6F83C31E5E7B8F1040F0ED840
:106CC80002344246291901A80DF007FB434601AAE0
:106CD8004946304604EB080700F0BEFAD3E76FF0E8
:106CE8000300D0E773B500230E4613600DF10701CA
:106CF80005461446FEF7F7F840B99DF807302BB162
:106D0800B38A2A6A534380331B0A236002B070BDDA
:106D180013B5CB681360144601AAFFF7E3FF18B94F
:106D28002368019A1344236002B010BDF8B5B0F887
:106D38005451D0F8580168438030000A0E46454344
:106D4800DDE90717144652B1B60206EB5202B2FB50
:106D5800F4F202EB4202524302F50042140C069A86
:106D6800534301F50042120C06200332B2FBF0F245
:106D7800C2EBC202B2F5803F38BF033103F50043CE
:106D88003EBFB1FBF0F1C1EBC10101F500414FEA93
:106D9800134334BF090C1B4903FB03F338BF4943B2
:106DA80003EB57030B44B3FBF7F39B03FE2205F1F8
:106DB80020007F33B3FBF2F35C434FF47A7704F59A
:106DC800FA748009B4FBF7F42401FFF72DF904F5F0
:106DD800FA74BC4228BF4FF4FA63064629BFB4FBD5
:106DE800F3F300205B19B4FBF7F428BFB3FBF4F00E
:106DF800FFF71AF9099B864294BF1E6018600020AD
:106E0800F8BD00BF0000F0FF2DE9F04F91B0CDE9CB
:106E18000723036A0E930B6909930546CB680B9306
:106E28000F460FAAFFF774FF0EAA39462846FFF748
:106E380059FF58BB0F9C95F8E0B0D5F8DC300593A6
:106E48004FF47A7606FB04F101F5004104910E999E
:106E58000A910499D5F8E4300693BBF1080F04F1C0
:106E680080040CBF0223032324F0FF0A090C95F8C1
:106E7800E820DFF8A081CDF83CA00C9109D1079B50
:106E8800C3F80080089BC5F84081186011B0BDE8C0
:106E9800F08F06990D932846FFF7C4FB5A460599CB
:106EA80081462846FFF7BEFB0D9B5B490C9A81443F
:106EB80003FB09F94FEAC92940F2776309F5FA7922
:106EC800240AB9FBF6F903FB09F909F5FA79B9FBC4
:106ED800F6F909FB04F404F18003099C74430C409F
:106EE800B4FBF2F44D4A1B0A944228BF1446012B06
:106EF80038BF01230C204FF4167258435443FFF750
:106F080093F83B7E3A894FEA400B002B7FD14249E8
:106F1800049B0B4003F5FA71414B5A4341F25C2341
:106F2800B2FBF3F20A9B7343B3F5481F28BF4FF433
:106F38004813A1EB4303B1FBF6F1B3FBF6F31B02D5
:106F4800B3FBF1F63602C6F58036564306F5004621
:106F5800360C06F5803676087643B60B4FF4487043
:106F6800704304F5004300F500401B0C5B43000C24
:106F780000FB0030FFF758F803046422323341F273
:106F88008837B3FBF2F340F6B532B3FBFBF302FBF1
:106F98000377244B9F429CBF42F21073B7FBF3F771
:106FA800DDE90532134403F5FA734FF47A7B4FF4A5
:106FB800FA62B3FBFBF0B3FBF2F202F5C812B2FBC4
:106FC800F0F088BF4FF47047FFF72EF8000200F585
:106FD800FA70B0FBFBF0404307FB0700FFF724F80B
:106FE8000BFB00F0079B0B9A404528BF40461860F2
:106FF800089BC5F84001CDE902934FF4487300930C
:107008000194334651462846FFF790FE3EE74FF479
:107018008036A3E7AE878F020000FFFF6666660032
:107028009A9906000F279F242DE9F04F8BB000276F
:1070380011F0780FDDE914B80446019299468DF8ED
:107048000E708DF80F708DF810708DF81170ADF806
:1070580012700997C1F3C30A00F0AF80AAF10503C3
:10706800DBB20A2B01D86B4AD75C0DF10E02002166
:107078002046FDF792FF9DF80E500646D5B1002830
:1070880040F09D8009AB05AA59462046FFF7BCFE93
:10709800002840F09680099BABF80A30014606AA02
:1070A8002046FDF7B3FF069D25B1059B9D422CBFE9
:1070B8000025012520B904AA02212046FDF76DFF0D
:1070C8009DF8106026B300287DD107AA022120462A
:1070D800FDF79CFF88B90122FF21204600F0F0F857
:1070E80058B90DF11202B621204600F037F920B93F
:1070F8000246FF21204600F0E3F8BDF81230079E53
:107108005B02C4F848311EB19E422CBF00260126FE
:1071180028B90DF1110203212046FDF73EFF9DF825
:10712800113093B1002873D1B9F1000F03D0019B3E
:107138001B02B3FBF9F908AA03212046FDF766FFF5
:10714800089B4B4594BF0023012320B9012F3CD154
:10715800FF2288F8002098F800200AB9ABF80A2026
:107168000DF10F02012120460193FDF716FF08BB20
:107178009DF80E20019B002A08BF0125BAF1040FD3
:1071880018BF9DF80F2084F82E501ABFB2FA82F269
:107198005209012284F82F209DF81020002A9DF81A
:1071A800112008BF0126002A08BF012384F8306097
:1071B80084F831300BB0BDE8F08F012755E7002582
:1071C8007EE735467CE70026A9E70AF1FF32092A5F
:1071D8000AD8DFE802F0050505090907090B070BBE
:1071E8000522B6E70422B4E7012E01D10322B0E755
:1071F800BAF1040F01D0012B01D10222A9E7012D18
:107208001BBF002388F8003088F800502B46A2E7FF
:107218000023A0E7324F010807B502F10A030093E3
:1072280093B20A4690F86011D0F85C0101F0B2FB05
:1072380003B05DF804FB13B502F10A0390F860414E
:107248000093D0F85C0193B20A4644F0010101F0C2
:1072580037FC02B010BD00003F2BF8B50E460546BE
:1072680011461C4611D80A4F38461A4600F8016BD9
:107278000DF033F8621C39462846FFF7CDFF002889
:107288000CBF00206FF01300F8BD6FF00300FBE7A0
:10729800000F002073B515468DF8071001220DF177
:1072A800070104461E46FFF7B7FF28B932462946AC
:1072B8002046FFF7C0FF08B16FF0130002B070BDA1
:1072C80008B5064B19705A7019460222FFF7A4FF39
:1072D800002814BF6FF01300002008BD000F002025
:1072E80008B5074B1970110A59709A70194603228C
:1072F800FFF792FF002814BF6FF01300002008BDAD
:10730800000F002037B515468DF8071001220DF142
:1073180007010446FFF780FF28B9012229462046C5
:10732800FFF789FF08B16FF0130003B030BDF7B560
:1073380015460DF1070206460F461C46FFF7E2FF09
:1073480050B99DF807301D4044EA050239463046D9
:107358008DF80720FFF7B4FF03B0F0BD73B51446EE
:107368008DF8071001220DF107010646FFF754FFBB
:1073780018B16FF0130002B070BD074D0222294604
:107388003046FFF758FF0028F3D12A786B7803EBD3
:1073980002232380EFE700BF000F002073B51446D7
:1073A8008DF8071001220DF107010646FFF734FF9B
:1073B80018B16FF0130002B070BD0A4D04222946BF
:1073C8003046FFF738FF0028F3D16B782A781B0482
:1073D80003EB0263EA781344AA7803EB02232360E1
:1073E800E9E700BF000F002008B50220FBF7A8FB63
:1073F800002008BD7047000010B5032000F072FCA3
:1074080001F0AAFD064B18600F20FBF78FFB04461E
:1074180018B9FBF7F2F9204610BD0124FBE700BFBD
:10742800280800204FF0E022136923F002031361BB
:1074380070474FF0E022136943F00203136170476D
:10744800014BD3F8900570470070FF1F014BD3F82C
:10745800940570470070FF1F014BD3F898057047DB
:107468000070FF1F024A536823F0010353607047FE
:10747800002004E0024A536823F002035360704777
:10748800002004E0024A536823F004035360704765
:10749800002004E08068C0F380007047F7B500233F
:1074A80001930446002800F0E980856D25B9FAF7B4
:1074B800D5FCE56584F8545023689A68D00040F1FB
:1074C800A1809A68D10000F1B480A26D42F0100248
:1074D800A265E26D42F00102E26501251846FFF758
:1074E800D9FFA26D02F01002024340F0C980A26DDC
:1074F800206922F4817242F00202A2659A68D207DA
:107508005DD4226BA67E94F82CC0003A18BF0122E5
:107518001703D4E902120A43217E42EA8132617ECE
:1075280042EAC13242EA4632002842EA4C02B4BF7B
:1075380020F000414FF400113A430A4394F8201018
:10754800012903D1002E76D142F48032616A21B13B
:10755800A66A01F4E07131430A43D968E66C21F464
:10756800FE3121F4FF711143D96094F83C20616821
:10757800012A01F0404C4CEA060609D1D4E910274B
:107588003A433243A66C324342EA0C0242F0010607
:107598001F693E4A3A4032431A6121F00042B2F173
:1075A800804F0CD0B1F1004F09D0394ED6F80827DA
:1075B80001F4701122F470120A43C6F808275A69B8
:1075C800666BA16B22F0070232435A615A6922F0B6
:1075D800700242EA01125A61002835D19A6A62F0B3
:1075E8000F029A625B6903F007039E423CD10023B5
:1075F800E365A36D23F0030343F00103A365284665
:1076080003B0F0BD9A68234922F0104222F0170215
:1076180042F080529A60204A1268B2FBF1F20132BD
:1076280052000192019A002A3FF44BAF019A013AA5
:10763800F7E7002552E7A16D41F02001A165E16D52
:1076480041F00101E16581E7B0F5001FCAD19A6AEE
:10765800E269013A92006FF00F0102F01C0201FA90
:1076680002F2216E0A43BCE7A36D23F0120343F034
:107678001003A365E36D43F00103E3650125BEE74D
:10768800A36D43F01003A365F8E700BF02FCFF1FDA
:1076980000200140400D030028080020F8B5456986
:1076A800082D04460E460AD00368DB68D80705D5BE
:1076B800A36D43F02003A3650120F8BD0425FBF763
:1076C80037FA074623681A682A4221D0A26D42F485
:1076D8000072A265DA6812F4406F14D1A27E92B9E2
:1076E8001A6812070FD51846FFF7D4FE28BB5A6848
:1076F80022F00C025A60A26D22F4807222F001027C
:1077080042F00102A265207E00BB0C221A60D4E779
:10771800711CD8D0FBF70CFAC01BB04201D8002E60
:10772800D0D123681B682B40CCD1A26D84F854308B
:1077380042F00402A2650320BFE7A26D42F02002D6
:10774800A265E26D42F00102E265DCE70020B4E7E1
:107758000368186C70470000F7B50023019390F890
:107768005430012B044600F0C580056806690123E2
:1077780080F854302846FFF78DFE002840F0B4808A
:10778800D1E90020022826F0040300F08280B3F13A
:10779800004FC2F3110E13D1AB6A43EA0E03AB627A
:1077A8008B68686903EA022323F07C4323F0FF0314
:1077B80020EA02210B43002A6B6126DB002055E0FA
:1077C800236E00F01F074FF00F0C0CFA07FC6FEA4E
:1077D8000C0623EA0C0CBEF1000F11D1C2F384632E
:1077E800BB4043EA0C0323668008E36901309842F2
:1077F800D6D8A86AC2F38363BB4006403343CEE7BA
:1078080092FAA2F3B3FA83F3EAE73B493B48D1F88B
:107818000837824203F0E07519D11B02CED4D1F8A3
:10782800083723F0E0732B4343F40003C1F808370B
:10783800334B1A68334BB2FBF3F20C2302FB0333CE
:107848000193019B002BB9D0019B013BF8E72E481F
:10785800824210D113F08070B0D1D1F8083723F0EC
:10786800E0732B4343F08073C1F80837002384F892
:10787800543003B0F0BD254882429FD113F48000F4
:107888009CD1D1F8083723F0E0732B4343F48003ED
:10789800EAE7B3F1004F01BFAB6AC2F311018B43B2
:1078A800AB62002A8ADA154813498242D1F80837B0
:1078B80009D1D1F8082703F0A07322F0E07213432E
:1078C800C1F808377AE71048824204D1D1F808276E
:1078D80003F44003F1E70D4882427FF46FAFD1F81B
:1078E800082703F0C073E8E7A26D42F02002A26502
:1078F8001846BBE70220BCE700200140001000B09A
:1079080028080020400D0300004000B8002000B403
:10791800026838B504461046FFF7BCFD08B90020D8
:1079280038BD9368990707D4936823F0004323F080
:10793800170343F010039360FBF7FAF80546236832
:107948009B685B07EBD5FBF7F3F8401B0228F6D9D9
:1079580023689B685A07F2D5A36D43F01003A3650B
:10796800E36D43F00103E3650120D9E773B5002314
:10797800026801939368DD07044602D5002002B02F
:1079880070BD9168214B194209D0A36D43F01003D3
:10799800A365E36D43F00103E3650120EFE7936816
:1079A80023F0004323F0170343F001039360184BBF
:1079B800D3F8083718021CD4637E012BDED0FBF7FE
:1079C800B7F8144E054622681368DB07D6D49368C7
:1079D800D9075FBF9368334043F001039360FBF717
:1079E800A7F8401B0228EED923681B68DA07EAD4F7
:1079F800CBE7094B094A1B68B3FBF2F30133019348
:107A0800019B002BD8D0019B013BF8E717000080B1
:107A180000200140E8FFFF7F28080020400D0300F8
:107A280038B504460068FFF735FD054620BB94F8D5
:107A38005430012B20D0012384F854302046FFF71E
:107A480095FFB0B9A36D226823F4706323F0010396
:107A580043F48073A3651C23E065136084F8540025
:107A6800936823F0004323F0170343F00403936063
:107A780038BD84F85450FBE70220F9E7026838B5AE
:107A8800936891680446C80701D4002038BD990757
:107A9800FBD4936803F00503012B19D1936823F0F5
:107AA800004323F0170343F002039360032313609A
:107AB800FBF73EF8054623689B68DB07E5D5FBF72F
:107AC80037F8401B0228F6D923689B68DA07F2D5F5
:107AD800A36D43F01003A365E36D43F00103E36571
:107AE8000120D3E770B5044600284BD0836D43F0DE
:107AF80002038365FFF70CFF054668B92046FFF7C8
:107B0800BDFF054608B90123A3652268936823F0E1
:107B1800104323F01703936023685A6822F46772AE
:107B280022F003025A6040F29F321A60D968164A5E
:107B38000A40DA601A6922F040421A615A6922F052
:107B480007025A611A6A02F0F0221A625A6A02F0AF
:107B5800F0225A62DA6A02F0F022DA629A6A0B4A72
:107B680000269E62D2F8083723F0FE73C2F8083761
:107B78002046FAF787F9E6652666A66584F8546014
:107B8800284670BD0125FBE700023E830020014026
:107B980010B590F85430012B044615D0012380F815
:107BA8005430FFF7B5FE58B92046FFF767FF38B9DC
:107BB800A36D23F4807323F0010343F00103A3654D
:107BC800002384F8543010BD0220FCE7F7B50023E9
:107BD800019390F85430012B04467FD0012380F89C
:107BE8005430FFF74BFF23689A6812F001020546EC
:107BF80007D0A36D43F01003A365002384F8543025
:107C08002DE0A16D364F21F4817141F00201A1658B
:107C1800DE68D96826F4FF4626F07C0621F4004188
:107C2800360421F00301360CD960082099683940E0
:107C380041F0004199609968002913DA01990131EE
:107C480001910199B1F52E3FF5D3A36D23F01203ED
:107C580043F01003A365002384F854300125284617
:107C680003B0F0BDD3F8B410013801F07F010A4425
:107C7800DCD199681A48014041F001019960D3F8B4
:107C8800B41021F07F0141EAD202C3F8B4209A6807
:107C9800024042F002029A60FAF74AFF0746236858
:107CA8009A68D20708D4DA683243DA60A36D23F001
:107CB800030343F001039FE7FAF73AFFC01B0228CA
:107CC800EDD923689B68D907E9D5A36D43F0100364
:107CD800A365E36D43F00103E365BFE70225BEE753
:107CE800E8FFFF7F0749CA6822F4E0620302120432
:107CF80003F4E063120C134343F0BF6343F400330F
:107D0800CB60704700ED00E0164B30B5DC68C4F37B
:107D18000224C4F10703251D042B28BF0423062DC4
:107D28004FF0FF358CBF033C002405FA03F321EA2A
:107D38000303A54022EA0502A340002843EA020300
:107D4800ACBF00F16040084A4FEA0313B8BF00F027
:107D58000F00DBB2AABF00F56140135480F800336E
:107D680030BD00BF00ED00E014ED00E0002807DBA7
:107D7800044A4109012300F01F00834042F82130E2
:107D8800704700BF00E100E000280CDB430906490A
:107D980000F01F0020330122824041F82320BFF366
:107DA8004F8FBFF36F8F704700E100E070B5D0E9E7
:107DB80013456560446D14B1D0E916456560D0E996
:107DC800105404F01C060124B4406C60046863601D
:107DD8008368102B0BBFA260A160E160E26070BDF8
:107DE8000268416CD3B210B5083B1424B3FBF4F31A
:107DF8000B4CA24288BF0B4A21F0030199BF01F145
:107E0800804202F50232521807338264064AC2647D
:107E180003F01F03012202FA03F3036510BD00BF3C
:107E2800070402401C0802408008024038B50028B8
:107E38005ED002682F4B9A424FF014014CD82E4B5B
:107E48001344B3FBF1F32D499B00C0E9101302233F
:107E580080F825301368056923F4FF4323F0700385
:107E68001360D0E9024323432B43456911682B4330
:107E780085692B43C5692B43056A2B430B43136064
:107E8800FFF7AEFFB4F5804F04BF0023436042689C
:107E9800816C02F07F030B60D0E91314013A032AC6
:107EA8004C6020D8164A174981651A44013B920054
:107EB800012103F0030301FA03F300214265C365BE
:107EC8001160114A536400230122C36380F82430EF
:107ED80080F82520184638BD0C4B1344B3FBF1F34A
:107EE8000B499B00B1E70023C0E91533C365EAE7F6
:107EF8000120F0E707040240F8FFFDBF0000024040
:107F08003F8200104009024000090240F8FBFDBF13
:107F18000004024038B5002841D00268136823F0F5
:107F2800010313601F4B9A424FF0140130D81E4BC7
:107F38001344B3FBF1F31D499B00C0E9101301245E
:107F480003F01C0304FA03F3002515604B60FFF7E8
:107F580047FF836C41681D60D0E913325A604A1E9E
:107F6800032A06D8124B0B449B0094401D60114B0A
:107F78005C640023C363C0E91533C0E90B33C0E96F
:107F88000D33C36580F8253080F82430184638BD95
:107F9800094B1344B3FBF1F308499B00CDE70120DB
:107FA800F5E700BF07040240F8FFFDBF00000240EC
:107FB8003F82001000090240F8FBFDBF00040240A8
:107FC80070B590F82450012D04463BD090F82560F8
:107FD8000125AE4280F824504FF000062CD102252E
:107FE80080F825500568C6632E6826F001062E60C5
:107FF800FFF7DCFE036BBBB12B6843F00E032B606D
:10800800A36C1A68D20342BF1A6842F480721A60DD
:10801800636D1BB11A6842F480721A602B6843F0D2
:1080280001032B60002070BD2B6823F004032B6034
:108038002B6843F00A03E2E78023C36380F82460D7
:108048002846F0E70220EEE7034640B190F82520E5
:10805800022A06D00422C263002280F824200120CC
:1080680070470268806C116821F00E011160016888
:1080780021F480710160116821F001011160D3E9D8
:10808800100202F01C0101228A404260D3E9132148
:1080980051605A6D32B1116821F480711160D3E9D1
:1080A800162151600122002083F8252083F824003E
:1080B800704710B590F82530022B03D00423C36312
:1080C800012010BD03681A6822F00E021A601A68AF
:1080D80022F001021A60826C136823F48073136023
:1080E800D0E9101303F01C02012393404B60D0E940
:1080F80013325A60436D33B11A6822F480721A60E1
:10810800D0E916325A60012380F82530836B0024A9
:1081180080F8244013B198472046D2E71846D0E7A4
:1081280070B4426C046C036826681D6802F01C0277
:108138000421914031420FD015F0040F0CD01A6879
:1081480092065EBF1A6822F004021A60036B61602F
:10815800002B33D070BC184702219140314217D010
:1081680015F0020F14D01A68940606D41A6822F083
:108178000A021A60012280F82520114A93428CBF16
:10818800104B114B5960002380F82430C36ADFE795
:1081980008219140314211D029070FD5196821F0E3
:1081A8000E011960012303FA02F26260C36380F8CA
:1081B8002530002380F82430436BC9E770BC704732
:1081C8008000024000040240000002400A4A53694D
:1081D80043F4802330B55361EFF3108472B6002363
:1081E800CD58C5500433B3F5807FF9D11369DB034B
:1081F800FCD484F3108830BD00400058064B5A69FF
:10820800002ABFBF054A9A6002F188329A60BABF55
:108218005869C00F00207047004000582301674587
:10822800044B5A6942F000425A615869C043C00F72
:10823800704700BF0040005870B50546FAF778FC53
:10824800124E04463369D90313D43369DA0744BF9D
:10825800012232614CF2FA32134011D10B4E3069CF
:1082680010F480200BD0FAF763FC001BA842F6D369
:1082780004E0FAF75DFC001BA842E3D3032070BDBD
:10828800024A1361024A01205360F8E7004000588F
:10829800400F00202DE9F041184D98462B78012B0E
:1082A80006460C46174626D001232B704FF47A70E9
:1082B80000236B60FFF7C0FFA0B9012E16D1104A4A
:1082C800536943F0010353612760BFF36F8FC4F80C
:1082D80004804FF47A70FFF7AFFF094A536923EA25
:1082E8000603536100232B70BDE8F0813946204610
:1082F800FFF76CFFEDE70220F6E700BF400F002014
:1083080000400058054A536923F47E7343EAC000CD
:1083180040F4803040F0020050617047004000583F
:108328002DE9F041234F3B78012B054688463FD085
:1083380001233B704FF47A7000237B60FFF77CFFCA
:10834800044688B92B68042B13D11B4A536943F49C
:10835800803343F0040353614FF47A70FFF76CFFE6
:108368000446154B1A681B6800233B702046BDE87D
:10837800F0814FF0FF33C8F800306E68D5E901325C
:108388001344B3420AD93046FFF7BCFF4FF47A7062
:10839800FFF752FF50B1C8F800600446064A536917
:1083A80023F47E7323F002035361DAE70136E5E72D
:1083B8000224DBE7400F0020004000582DE9F04F71
:1083C800524C00234FF00F090A6832FA03F501D125
:1083D800BDE8F08F012505FA03F818EA020200F05B
:1083E8008E804E68032706F003054FEA430E07FA0E
:1083F8000EFC6F1E012F6FEA0C0C32D8876807EA53
:108408000C0ACF6807FA0EF747EA0A078760476839
:1084180027EA0808C6F300179F4047EA080747609D
:10842800C76807EA0C088F6807FA0EF747EA0807D3
:10843800022DC76017D14FEAD30800EB880803F074
:10844800070AD8F820704FEA8A0A09FA0AFB27EACD
:108458000B0B0F6907FA0AF747EA0B07C8F82070F1
:1084680001E0032DDCD1076805FA0EF507EA0C07D1
:108478003D4316F4403F056041D023F0030707F160
:10848800804707F5803703F0030CBD684FEA8C0C72
:108498004FF0070E0EFA0CFEB0F1904F25EA0E0EC3
:1084A8002FD01B4DA8422ED005F58065A8420CBFE1
:1084B8000225072505FA0CF545EA0E05BD60256875
:1084C800D74316F4801F0CBF3D40154325606568EF
:1084D80016F4001F0CBF3D4015436560D4F880506A
:1084E80016F4803F0CBF3D401543C4F88050D4F8C3
:1084F8008450B60354BF3D401543C4F8845001333B
:1085080062E70025D6E70125D4E700BF0008005838
:1085180000040048374A2DE9F04F00234FF0010AC4
:108528004FF0070B4FF00F0931FA03F401D1BDE802
:10853800F08F0AFA03FC1CEA010654D023F0030466
:1085480004F1804404F5803403F00307A568BF00F4
:108558000BFA07F8B0F1904F08EA050E45D0264D02
:10856800A84244D005F58065A8420CBF022507251E
:10857800BD40754517D1D2F8805025EA0605C2F8E6
:108588008050D2F8845025EA0605C2F88450156850
:1085980025EA06051560556825EA06055560A568AB
:1085A80025EA0805A560056803265C0006FA04F4B8
:1085B80023FA06F6254300EB8606056003F0070557
:1085C800376AAD0009FA05F527EA050737628568B5
:1085D80025EA04058560456825EA0C054560C568F7
:1085E80025EA0404C46001339EE70025C0E701259D
:1085F800BEE700BF0008005800040048036919429C
:1086080014BF0120002070470AB181617047816260
:1086180070470000044AD168014208B502D0D06012
:10862800FBF728F908BD00BF0008005803689A69DD
:10863800910744BF00229A629A69D2075EBF9A697D
:1086480042F001029A61704730B5039D04682B43DC
:1086580043EA0243064A6068C1F309010B4342EA50
:10866800555223F0004320EA02000343636030BD03
:10867800FF63FF0303682DE9F0419C6914F01004BF
:1086880005460F4616466FD010220024DA61A04630
:108698002B689A69900661D4B8F1000F35D044F080
:1086A800040401202E68B369D90541BF4FF48072D4
:1086B800F26144F0010401205A0541BF4FF4806281
:1086C80044F00804F26101209B054FD54FF4007374
:1086D80044F00204F3612846FFF7A8FF736823F00B
:1086E800FF7323F48B3323F4FF7323F001037360C8
:1086F8006B6C23436B64202385F84130002385F895
:10870800423085F84030012032E07A1CC1D0FAF7B7
:108718000FFA801BB84201D8002FB9D12B685968CD
:1087280095F8422098690004D2B20AD5490408D4C1
:10873800202A06D05A6842F480425A60FAF7F8F9BB
:1087480006462B689B699B06A2D4FAF7F1F9801BB1
:108758001928F6D920244FF0010899E7B8F1000F3D
:108768009DD12022DA619AE720469BE70028B2D102
:10877800BDE8F08170B504460D46164623689B692E
:108788009B0701D5002070BD324629462046FFF7D9
:1087980071FFA0B96A1CF1D0FAF7CAF9801BA84288
:1087A80001D8002DEAD1636C43F0200363642023D1
:1087B80084F84130002384F8423084F840300120A6
:1087C800E1E770B504460D46164623689B695B07CA
:1087D8000ED4324629462046FFF74CFF38BB2368A3
:1087E8009A69910625D59A69520703D5228D0AB14F
:1087F800002070BD9A6912F010021CBF1022DA61C5
:108808004FF0200118BF04226264D9615A6822F02F
:10881800FF7222F48B3222F4FF7222F001025A60B6
:10882800002384F8411084F8423084F84030012055
:10883800DFE7FAF77DF9801BA84201D8002DC4D1E3
:10884800636C43F020036364202384F841300023E1
:10885800EBE72DE9F041069F0446884616461D467B
:108868002268936938EA03030CBF01230023B3424B
:1088780001D0002015E06B1CF3D0FAF759F9C01BA2
:10888800A84201D8002DEBD1636C43F02003636448
:10889800202384F84130002384F8423084F84030A3
:1088A8000120BDE8F08170B504460D4616462368E0
:1088B8009B699B0601D5002070BD3246294620469B
:1088C800FFF7D8FE90B9FAF733F9801BA84201D810
:1088D800002DECD1636C43F020036364202384F8FB
:1088E8004130002384F8423084F840300120E3E727
:1088F80010B5044600284AD090F8413003F0FF0232
:108908001BB980F84020F9F701FE242384F8413090
:1089180023681A6822F001021A60626822F0706205
:108928001A619A6822F400429A60D4E90221012966
:1089380024D142F400429A605A6842F0007242F42C
:1089480000425A60DA6822F40042DA60D4E904216D
:108958000A43A16942EA0122DA60D4E907210A43FD
:108968001A601A6842F001021A600020202360642D
:1089780084F84130206384F8420010BD42F4044278
:1089880002299A6004BF4FF400625A60D4E70120BC
:10899800F3E700002DE9F347984690F841300A9F25
:1089A800202B04460E46914640F0868090F84030D1
:1089B800012B00F081804FF0010A80F840A0FAF7FF
:1089C800B7F819230546009052464FF40041204657
:1089D800FFF73FFF18B1012002B0BDE8F08721235F
:1089E80084F84130102384F842306064A4F82A8067
:1089F800638DC4F824909BB2FF2B60632F4B26D95C
:108A0800FF22228500934FF0807331462046FFF7FE
:108A18001BFE638D9BB22A4639462046FBB9FFF7F9
:108A280042FF0028D7D123682021D9615A6822F053
:108A3800FF7222F48B3222F4FF7222F001025A6094
:108A480084F8411084F8400084F84200C4E7628D3D
:108A5800009392B222854FF00073D2B2D5E7FFF7A8
:108A680089FE0028B7D1636A226813F8011B916256
:108A78006362638D228D013B9BB26385638D013AEE
:108A880092B29BB22285002BC3D0002AC1D1009597
:108A98003B4680212046FFF7DCFE00289BD1638DF2
:108AA8009BB2FF2B03D9FF2222850090ABE7628D92
:108AB800009092B22285CEE702208DE70020008048
:108AC8002DE9F347984690F841300A9F202B044639
:108AD8000E46914640F0878090F84030012B00F018
:108AE80082804FF0010A80F840A0FAF721F8192394
:108AF8000546009052464FF400412046FFF7A9FE74
:108B080018B1012002B0BDE8F087222384F8413073
:108B1800102384F842306064A4F82A80638DC4F876
:108B280024909BB2FF2B6063304B26D9FF2222850D
:108B380000934FF0807331462046FFF785FD638D23
:108B48009BB22A4639462046FBB9FFF7ACFE0028FF
:108B5800D7D123682021D9615A6822F0FF7222F404
:108B68008B3222F4FF7222F001025A6084F841101D
:108B780084F8400084F84200C4E7628D009392B202
:108B880022854FF00073D2B2D5E7FFF71AFE00280E
:108B9800B7D123685A6A636A1A70636A228D0133EF
:108BA8006362638D013B9BB26385638D013A92B228
:108BB8009BB22285002BC2D0002AC0D100953B462B
:108BC80080212046FFF745FE00289AD1638D9BB28D
:108BD800FF2B03D9FF2222850090AAE7628D00901F
:108BE80092B22285CDE702208CE700BF00240080E6
:108BF80010B590F84120202A0346D4B21CD190F831
:108C08004020012A18D0242280F8412002681068E8
:108C180020F001001060106820F480501060106887
:108C2800014311601168002041F00101116083F8CF
:108C3800414083F8400010BD0220FCE710B590F8D1
:108C48004120202A0346D4B21BD190F84020012AA3
:108C580017D0242280F841200268106820F0010013
:108C68001060106820F4706040EA012111601168FA
:108C7800002041F00101116083F8414083F8400071
:108C880010BD0220FCE70000024A136843F4807319
:108C980013607047000400580D4B10B55B690C4613
:108CA80028B99A0507D500F027F820B110BD9B0513
:108CB80001D400F019F8074A1369012C23F00403C2
:108CC800136101D130BFF1E740BF20BF20BFEDE7FE
:108CD8000004005800ED00E0024B186800F4C06082
:108CE800704700BF00040058024A136843F48043E9
:108CF80013607047000400580C4A136823F480433B
:108D080013600B4B1B6832214B430A49B3FBF1F349
:108D18005169890500D533B9536913F4007F14BF2D
:108D2800032000207047013BF2E700BF0004005811
:108D38002808002040420F000B4A136823F007035D
:108D480043F002031360094B1A69012842F0040238
:108D58001A6105D130BF1A6922F004021A617047FE
:108D680040BF20BF20BFF6E70004005800ED00E038
:108D78004FF0B0431868C0F3404070474FF0B0431D
:108D88001868C0F3400070474FF0B042536823F4AE
:108D98007F4343EA0023536070474FF0B04318689D
:108DA800C0F34060704700007FB54FF0B0432C4AD5
:108DB800D3F80831C0F3031003F00F0352F8204032
:108DC800284A52F82330B4FBF3F4FFF785FF264B0B
:108DD800054693E80700B5F5007F04AB03E90700F3
:108DE80010D0224B9C4218D303F5B70303F67F53E8
:108DF8009C4229D903F5741303F510639C4225D8C6
:108E080002230BE01A4B9C4207D91A4B9C421BD9F0
:108E180003F5370303F5D853F0E7002304AA02EB60
:108E2800830353F80C4C144D2B6823F0070323439A
:108E38002B60F9F77DFE06462B6803F007039C427A
:108E480006D1002004B070BD0123E7E70024EAE75B
:108E5800F9F76EFE801B0228EED90320F2E700BF67
:108E6800A04F0108404F010820440108C0CF6A0004
:108E7800BFEA21013F933402004000584FF0B0434D
:108E880010B59A68D96812F00C0205D00C2A4AD19C
:108E980001F00303012B50D14FF0B0412B480B6870
:108EA80013F0080306D00B6813F0080337D1D1F884
:108EB800941007E00C68240756BFD1F8943009686D
:108EC800C3F3032350F82330002A0CBF18460020B0
:108ED8004FF0B0418A6802F00C020C2A1ED1CA6811
:108EE80002F00302022A2ED0032A06D10B68184A80
:108EF80013F4801F174B18BF13464FF0B042D068C9
:108F0800D168D268C0F306205843C1F30213013375
:108F1800B0FBF3F0530F0133B0FBF3F010BD0B6857
:108F2800C3F30313CEE7042A0AD0082A05D11B6825
:108F380013F4801304D10748CAE700231846C7E78B
:108F480003480023C4E7024BD7E700BFA04F01083E
:108F58000024F4000048E80108B5FFF78FFF4FF040
:108F6800B043044A9B68C3F3031352F82330B0FBA1
:108F7800F3F008BD404F01082DE9F04104460028F0
:108F880053D04FF0B0439D68DE6803689B0605F038
:108F98000C0506F0030668D5026A1DB10C2D46D1F2
:108FA800012E44D1002A40D04FF0B043A16A1A687C
:108FB800170756BFD3F894301B681B0903F0F0035A
:108FC80099421FD90846FFF7EFFE00282DD14FF030
:108FD800B042136843F0080313601368A16A23F0D2
:108FE800F0030B431360606AFFF7CEFEFFF7B4FF90
:108FF800AB4B1860AB4B1868F9F798FD002834D0D4
:10900800BDE8F0814FF0B042136843F008031360E5
:10901800136823F0F0030B431360606AFFF7B4FE94
:109028000846FFF7C1FE0028E0D00120E8E74FF02E
:10903800B043002A54D01A6842F001021A60F9F7C6
:1090480077FD0746FFF79AFE002842D04FF0B0425E
:10905800136843F0080313601368A16A23F0F00350
:109068000B431360606AFFF78FFE2368D80748D464
:109078002368990700F18C8023681E0740F1FA8065
:10908800A3694FF0B046002B00F0E180D6F8943089
:10909800E16903F01002914200F0C48003F003027A
:1090A800022AC2D0D80740F1B380D6F8943023F012
:1090B8000103C6F89430F9F73BFD0746D6F894301B
:1090C800990740F1A580F9F733FDC31B112BF5D99A
:1090D80004E0F9F72DFDC01B0228B3D903208FE760
:1090E8001A6822F001021A60F9F722FD0746FFF715
:1090F80045FE0028B9D0F9F71BFDC01B0228F6D998
:10910800ECE7082D03D00C2D05D1032E03D163689D
:10911800002BADD189E74FF0B043A1681A6822F45B
:1091280080120A431A606268B2F5803F10D11A684B
:1091380042F480321A60F9F7FBFC0746FFF718FE85
:10914800002895D1F9F7F4FCC01B6428F6D9C5E7C7
:10915800B2F5041F04D11A6842F400121A60E6E757
:10916800196821F480311960196821F40011196017
:10917800002AE0D1F9F7DCFC0746FFF7F9FD0028E3
:109188003FF476AFF9F7D4FCC01B6428F5D9A5E7FE
:10919800042D236903D00C2D0ED1022E0CD1002BE7
:1091A8003FF443AF4FF0B0426169536823F0FE4388
:1091B80043EA016353605FE74FF0B046BBB13368E1
:1091C80043F480733360F9F7B3FC074633685A05F4
:1091D80007D57368626923F0FE4343EA026373604C
:1091E8004AE7F9F7A5FCC31B022BEFD976E73368EA
:1091F80023F480733360F9F79BFC074633685B05FB
:109208007FF53AAFF9F794FCC31B022BF6D965E753
:109218004FF0B042E169D2F8943023F010030B43C9
:10922800C2F894304FF0B047D7F8943043F00103B8
:10923800C7F89430F9F77CFC0646D7F894309A07BB
:1092480018D4F9F775FC831B112BF6D946E7D6F825
:10925800943023F00103C6F89430F9F769FC074607
:10926800D6F894309B0705D5F9F762FCC31B112B80
:10927800F6D933E72368580754D50B4F3B68D9050F
:1092880014D4FFF701FDF9F753FC06463B68DA05ED
:109298000CD4F9F74DFC831B022BF7D91EE700BF4E
:1092A800280800202C08002000040058E3684FF02C
:1092B800B046002B58D023F08003052B02BFD6F808
:1092C800903043F00403C6F890304FF0B046F9F7F9
:1092D8002FFCD6F8903043F001030746C6F89030CB
:1092E80041F28838D6F890309B0705D4F9F720FC6E
:1092F800C31B4345F6D9F1E6E36823F00403812B49
:109308001BD1F9F715FCD6F8903043F08003C6F866
:10931800903007464FF0B04641F28838D6F8903082
:10932800180504D5E06A00284AD1002068E6F9F754
:10933800FFFBC01B4045F1D9D0E6F9F7F9FBD6F899
:10934800903023F08003C6F8903007464FF0B046BF
:1093580041F28838D6F890301905E3D5F9F7E8FBDB
:10936800C01B4045F6D9B9E6F9F7E2FBD6F89030CC
:1093780023F080030746C6F8903041F28838D6F8C3
:1093880090301A0516D4F9F7D3FBD6F8903023F0AD
:109398000103C6F8903007464FF0B04841F28836CE
:1093A800D8F890309B07BDD5F9F7C2FBC31BB34271
:1093B800F6D993E6F9F7BCFBC01B4045DFD98DE62B
:1093C8000C2D4ED04FF0B04302281A6822F080725C
:1093D8001A6033D1F9F7ACFB0546FFF7DEFC38BB62
:1093E800D4E90C314FF0B0420B43D0682D4901400D
:1093F8000B43E16B0B43216C0B43616C0B43A16B7B
:1094080043EA0123D360136843F080731360D36881
:1094180043F08053D360F9F78BFB0446FFF7BDFC9C
:10942800002882D1F9F784FB001B0A28F6D955E6F3
:10943800F9F77EFB401B0A28CFD94FE6F9F778FBEE
:109448000446FFF7AAFC30B94FF0B042164BD1687A
:109458000B40D360D4E5F9F76BFB001B0A28F0D961
:109468003CE601283FF4CCAD4FF0B043226BDB68FB
:1094780003F0030191427FF4D8AD616B03F07002F1
:109488008A427FF4D2ADA16B03F4FE42B2EB012F06
:109498007FF4CBAD626C03F0604393423FF445AF79
:1094A800C3E500BF8C80C111FCFFFEEE2DE9F04141
:1094B8000D46044610B90120BDE8F081684E3368B6
:1094C80003F007038B4216D323689A0727D54FF07A
:1094D800B047A268BB6823F0F0031343BB60F9F7F9
:1094E80027FB0646BB68DB0319D4F9F721FB831B6E
:1094F800022BF7D911E0336823F007030B433360DD
:10950800F9F716FB0746336803F00703AB42DBD0D5
:10951800F9F70EFBC01B0228F5D90320CCE7236816
:10952800580617D54FF0B0476269D7F8083123F0CD
:109538000F0343EA1213C7F80831F9F7F9FA064698
:10954800D7F80831D90305D4F9F7F2FA831B022BAF
:10955800F6D9E2E723685A0713D54FF0B047E26817
:10956800BB6823F4E0631343BB60F9F7E1FA0646EE
:10957800BB689B0305D4F9F7DBFA831B022BF7D9E9
:10958800CBE72368180714D54FF0B0472269BB68AA
:1095980023F4605343EAC203BB60F9F7C9FA0646ED
:1095A800BB68590305D4F9F7C3FA831B022BF7D913
:1095B800B3E72368DA070FD4294C236803F00703BD
:1095C800AB4239D8FFF7C8FC264B1860264BBDE8DC
:1095D800F0411868F9F7AABA6268022A1DD1FFF7A4
:1095E800C7FB00283FF467AF4FF0B04641F2883818
:1095F800B36823F003031343B360F9F799FA0746F6
:10960800B368626803F00C03B3EB820FD4D0F9F7A8
:109618008FFAC01B4045F3D97FE7032A02D1FFF731
:10962800BCFBDEE712B9FFF7A9FBDAE74FF0B0435E
:109638001B685B05D8D43EE7236823F007032B4358
:109648002360F9F775FA0646236803F00703AB426F
:10965800B8D0F9F76DFA801B0228F5D95DE700BF8D
:1096680000400058280800202C08002008B5FFF703
:1096780073FC4FF0B043044A9B68C3F3022352F8CB
:109688002330D84008BD00BF804F010808B5FFF758
:1096980063FC4FF0B043044A9B68C3F3C22352F8FB
:1096A8002330D84008BD00BF804F01084FF0B043B9
:1096B800D3F89000C0F3400070474FF0B041020962
:1096C800D1F8883002F47F22000123EA020300F473
:1096D8007F200343C1F8883070474FF0B041020C37
:1096E800D1F88830120423EA020343EA0040C1F8A3
:1096F8008800704770B5066816F48036044638D07E
:10970800FFF7C2FAF9F714FA614E05463368DB052C
:1097180029D54FF0B043616BD3F8902002F4407222
:10972800914214D0D3F89010D3F8902042F48032AC
:10973800C3F89020D3F8902021F4407022F48032AE
:109748008D07C3F89020C3F8900000F190804FF087
:10975800B042616BD2F8903023F440730B43C2F8E7
:109768009030002605E0F9F7E3F9401B0228CDD92F
:1097780003262568E8070AD54FF0B0416268D1F89A
:10978800883023EA124392B21343C1F88830A907FC
:109798000AD54FF0B041A268D1F8883023EA1243C5
:1097A80092B21343C1F88830AA0609D54FF0B042E7
:1097B8002169D2F8883023F440630B43C2F888301B
:1097C800AB0502D5206AFFF788FF680502D5606AF5
:1097D800FFF783FF290502D5A06AFFF77EFF6A0617
:1097E80002D56069FFF769FF2B0602D5A069FFF76C
:1097F80064FFE80502D5E069FFF75FFFE90610D5C9
:109808004FF0B042E168D2F8883023F440730B433C
:10981800C2F88830B1F5807F02BFD36843F0807307
:10982800D3602A040ED54FF0B042216BD2F88830AD
:1098380023F040430B43C2F8883019B9D36843F08A
:109848008073D3606B0410D54FF0B042E16AD2F850
:10985800883023F040530B43B1F1005FC2F88830E1
:1098680003D1D36843F48033D360304670BDF9F731
:109878005FF941F288360546FFF718FF01283FF4E3
:1098880066AFF9F755F9401BB042F5D970E700BF4C
:109898000004005830B590F82C30012B02464FF0E8
:1098A800020022D0174B82F82D00CA24012582F825
:1098B8002C505C6253245C62B1F5807F146B99690B
:1098C80014D121F488519961596C24F0010421F0D4
:1098D800004159641463DD650A4BFF215962002079
:1098E800012382F82D3082F82C0030BD21F4085174
:1098F8009961D96C24F0020421F00041D964146301
:10990800D865E9E70028004070B50B4E036B756D0C
:109918001D40EA07044603D50123F365F9F779FAF0
:10992800AB0704D50223F365204600F0CBF90123E9
:1099380084F82D3070BD00BF0028004038B50A4CAF
:10994800E36823F02003E360F9F7F2F80546E368DB
:109958009B0601D5002038BDF9F7EAF8401BB0F5A1
:109968007A7FF4D90320F6E7002800402DE9F0417A
:10997800114DEC6814F0400407461AD1EB6843F027
:109988008003EB60F9F7D4F84FF003080646EB685C
:109998005B0601D4032C02D12046BDE8F081F9F71B
:1099A800C7F8801BB0F57A7F84BF87F82D80032421
:1099B800EDE70024F0E700BF0028004038B50F4C61
:1099C800E36823F08003E360A3699B06054606D499
:1099D800FFF7B4FF10B1032085F82D0038BDA36947
:1099E80023F02003A361FFF7A9FF10B1032085F836
:1099F8002D00A36943F02003A361EFE7002800408E
:109A080038B5044600284BD090F82D3003F0FF02FB
:109A18001BB980F82C20F8F789FE0223214D84F821
:109A28002D30EB68DB0632D4CA236B6253236B629A
:109A38002046FFF79BFF78BBAB6923F08E6323F0CA
:109A48004003AB6121696368AA690B431343A269A8
:109A58001343AB61D4E9022343EA02432B61D4E9FF
:109A68000931EA680B4322F4F8521343EB602046AD
:109A7800FFF7A4FF80B9D4E90713AA690B4322F0C2
:109A88006042134362691343AB61FF236B62012396
:109A980084F82D30002002E0024BFF225A6238BDC4
:109AA8000120FCE7002800400023092803D840EAE9
:109AB8000310C0B270470A380133C0B2F5E700009E
:109AC8002DE9F04790F82C30012B05464FF00200A5
:109AD80069D0012385F82C304E4B85F82D00DE68BF
:109AE80006F44076B6F5807F78D04C69087891F80E
:109AF800019091F802A091F82470002A55D19B6931
:109B080013F0400308BFCB70FFF7CEFF80464846EE
:109B1800FFF7CAFF02465046FFF7C6FF81463846A0
:109B2800FFF7C2FF0B6ACF78234343EA875343EA20
:109B3800090343EA084343EA022343EA0063354A38
:109B4800CA205062532050628C6A8869B4F5807FBD
:109B5800946945D124F4885494610124D465B6F5F8
:109B6800807F09BFCB6913640343536418BF5064F3
:109B7800284B4A681A672A6B42F001022A639A69DD
:109B880042F488529A61244AD2F8803043F4003370
:109B9800C2F880301F4BFF225A620020012385F84B
:109BA8002D3085F82C00BDE8F087B4F1803F07D050
:109BB800B4F5000F04D09B6913F0400308BFCB70C5
:109BC8000B6ACA781C4344EA0A0444EA004343EA9D
:109BD800092343EA825343EA0763B0E70023AEE769
:109BE80024F4085494610224D465B6F5807F09BF33
:109BF800CB6993640343D36418BFD064054B4A68A8
:109C08005A672A6B42F002022A639A6942F40852A0
:109C1800B8E700BF002800400008005890F82C2042
:109C2800012A03464FF0020012D00A4A83F82D0099
:109C3800CA21516253215162916941F02001916119
:109C4800FF2151620020012283F82D2083F82C0087
:109C5800704700BF0028004090F82C20012A0346D6
:109C68004FF0020019D00D4A83F82D00CA21516225
:109C78005321516291690A4841F080019161D0F8FD
:109C8800801041F48021C0F88010FF21516200202B
:109C9800012283F82D2083F82C007047002800400B
:109CA80000080058064B5A6D520610B5044603D5F5
:109CB8004022DA65F9F7B0F8012384F82D3010BD99
:109CC800002800407047890001F1804101F53141C9
:109CD8000A607047890001F1804101F53141086847
:109CE80070470000034AD2F8903043F40043C2F8AA
:109CF8009030704700040058034AD2F8903023F49B
:109D08000043C2F89030704700040058074B1A68A7
:109D180022F040021A6040F441704FF4B8521860C3
:109D28005A601A6842F040021A60704700000158F1
:109D380037B5054600284ED0837903F0FF046BB190
:109D4800032C0BD0254B4FF400629A612868FFF76B
:109D5800DDFF002401232B71AC602FE000236B7121
:109D68002846F8F7FDFD1E4AD2F8903043F4805398
:109D7800C2F89030002CE5D102234FF0B042AB710D
:109D8800D2F8943023F40043C2F89430154B1B6882
:109D98001C214B43DB0C64214B430193019B93B97A
:109DA8000124AC60FFF79EFF0C4B9A6842F40062F6
:109DB8009A604FF400629A61002CC7D00123AB71FE
:109DC800204603B030BD019B013B0193D2F894308B
:109DD8005B04E3D4E6E70124F2E700BF000400587F
:109DE800000800582808002037B5174D2B68024690
:109DF8001C204343DB0C6420434314480193019B1C
:109E080093B901209060114C21732B681C214B439E
:109E1800DB0C64214B430193019B6BB901209060DB
:109E28000A4BDB6803B030BD019B013B019383689B
:109E38009C07E4D50020E6E7019B013B0193A3685A
:109E4800DB07E9D5ECE700BF28080020000001582F
:109E580037B5184D2B6802461C204343DB0C6420A1
:109E6800434315480193019BA3B901209060124C0C
:109E7800FF2323732B681C256B43DB0C64256B4382
:109E88000193019B73B9012090600B4BDB680B7049
:109E980003B030BD019B013B019383689C07E2D569
:109EA8000020E4E7019B013B0193A368DB07E8D5A9
:109EB800EBE700BF28080020000001580F4B13B53E
:109EC8001B680F4C182253431B0D64225343014651
:109ED80001936269019B02F0040223B902238B609B
:109EE800012002B010BD019B013B0193606910F095
:109EF8000200F6D0002AECD11046F2E7280800202C
:109F08000004005807B50379012B0FD10A4B1B68D1
:109F1800182253431B0C0193FFF7EEFE019B013BF4
:109F28000193019B002BF9D1FFF7DCFE03B05DF82C
:109F380004EBFFF7C3BF00BF28080020F8B51E4692
:109F48008379012B154604460F46DAB22DD14379A1
:109F5800012B2AD0022342718371FFF7D3FF0D2111
:109F68002046FFF7C9FEFFF73FFF390A2046FFF7F3
:109F78003BFFF9B22046FFF737FF2E44B5420ED11A
:109F88002046FFF7AFFEFFF799FFA06801230038CE
:109F9800A3714FF0000318BF01206371F8BD15F8D5
:109FA800011B2046FFF720FFE8E70220F6E7F8B597
:109FB8001E468379012B154604460F46DAB22FD187
:109FC8004379012B2CD04271FFF79CFF1D212046BD
:109FD800FFF792FEFFF708FF390A2046FFF704FF54
:109FE800F9B22046FFF700FF00212046FFF7FCFEEC
:109FF8002E44B5420ED12046FFF774FEFFF75EFFF0
:10A00800A06801230038A3714FF0000318BF012096
:10A018006371F8BD29462046FFF71AFF0135E8E7C6
:10A028000220F6E7F8B51F468379012B154604464A
:10A038000E46DAB22CD14379012B29D04271FFF7B1
:10A0480061FF06F0EF03A3F18402534253412371E9
:10A0580031462046FFF750FEFFF7C6FE2F44AF42B9
:10A0680010D1FFF73FFE842E02D02046FFF726FFCF
:10A07800A06801230038A3714FF0000318BF012026
:10A088006371F8BD15F8011B2046FFF7ADFEE6E742
:10A098000220F6E7F8B51E468379012B15460446DB
:10A0A8000F46DAB227D14379012B24D04271FFF74A
:10A0B80029FF39462046FFF71FFEFFF795FE0021CE
:10A0C8002046FFF791FE2E44B5420ED12046FFF7F9
:10A0D80009FEFFF7F3FEA06801230038A3714FF0D3
:10A0E800000318BF01206371F8BD29462046FFF719
:10A0F800AFFE0135E8E70220F6E737B50023ADF8F3
:10A10800043001AA022312210546FFF7C3FFBDF858
:10A118000440022364BA01AAA4B219462846FFF7EC
:10A1280081FFE20702D5284609F0F6F9A30702D510
:10A13800284609F0F7F9600702D5284609F01CFA05
:10A14800210702D5284609F01DFAE20602D528465D
:10A1580009F01EFAA30602D5284609F007FA600698
:10A1680002D5284609F0E4F9210606D514F48071D1
:10A1780018BF0121284609F0E1F9A20502D52846B1
:10A1880009F0ECF9630402D5284609F007FA03B090
:10A1980030BDF8B51E468379012B154604460F4697
:10A1A800DAB227D14379012B24D04271FFF7AAFEF6
:10A1B8000E212046FFF7A0FDFFF716FE3946204680
:10A1C800FFF712FE2E44B5420ED12046FFF78AFD56
:10A1D800FFF774FEA06801230038A3714FF0000355
:10A1E80018BF01206371F8BD15F8011B2046FFF761
:10A1F800FBFDE8E70220F6E7F8B51E468379012B58
:10A20800154604460F46DAB22BD14379012B28D0E4
:10A218004271FFF777FE1E212046FFF76DFDFFF71D
:10A22800E3FD39462046FFF7DFFD00212046FFF712
:10A23800DBFD2E44B5420ED12046FFF753FDFFF754
:10A248003DFEA06801230038A3714FF0000318BF3A
:10A2580001206371F8BD29462046FFF7F9FD013555
:10A26800E8E70220F6E7026852E8003F23F0C0035F
:10A2780042E8003102680029F5D102F1080353E8E9
:10A28800003F23F4000302F1080C4CE800310029D8
:10A29800F3D12023C0F888307047000010B5026859
:10A2A80052E8003F23F4907342E800310268002925
:10A2B800F5D10F4C02F1080353E8003F234002F1A7
:10A2C800080C4CE800310029F4D1C36E012B07D1EA
:10A2D80052E8003F23F0100342E800310029F7D18B
:10A2E8002023C0F88C300023C366436710BD00BF2D
:10A2F800FEFFFFEFF8B504461346D4F88850202D2A
:10A3080032D1F1B1EAB1E06FA4F85620A4F8542094
:10A3180000262122C4F890602165C4F888202268AC
:10A3280088B1124FC762124F0763124F2832C0E933
:10A338000D76FDF745FE30B11023C4F89030C4F80F
:10A34800885001200FE0236840221A62226802F137
:10A35800080353E8003F43F0800302F1080141E895
:10A3680000300028F3D1F8BD0220FCE781A30008E3
:10A37800C9A30008D5A3000808B50346806A1B686E
:10A388001B6813F0200317D1A0F85630026802F1B9
:10A39800080353E8003F23F08003083242E8003105
:10A3A80002680029F2D152E8003F43F0400342E836
:10A3B80000310029F7D108BDF8F784FEFBE77047A4
:10A3C80008B5806AFFF7FBFF08BD7047806A38B59B
:10A3D8000468D0F88830D0F88C50A268120606D5E8
:10A3E800212B04D10023A0F85630FFF73CFFA368C7
:10A3F8005B0606D5222D04D10023A0F85E30FFF7B6
:10A408004DFFD0F8903043F01003C0F89030FFF7BC
:10A41800DCFF38BD08B5806A0023A0F85E30A0F8DC
:10A428005630FFF7D2FF08BD704700000368D969AE
:10A438001A682DE9F04140F60F0631429D6804463E
:10A4480010D18E0640F1978002F0200605F0805763
:10A458003E4300F09080436F002B00F08580BDE8FC
:10A46800F0411847AB4EAC482E401040304300F046
:10A478008280CF0709D5D00507D501201862D4F806
:10A48800900040F00100C4F890008F0709D5E80754
:10A4980007D502201862D4F8900040F00400C4F8F0
:10A4A80090004F0709D5E80707D504201862D4F8AB
:10A4B800900040F00200C4F890000F070BD502F09E
:10A4C8002000304307D008201862D4F8900040F0EC
:10A4D8000800C4F890000E050AD5500108D54FF4BD
:10A4E80000601862D4F8903043F02003C4F890302C
:10A4F800D4F89030002B37D08B0609D502F0200213
:10A5080005F080552A4303D0636F0BB12046984766
:10A518002668D4F89020B36802F0280203F04003BC
:10A5280053EA0205204621D0FFF7B8FEB3685F065C
:10A5380017D5226802F1080353E8003F23F04003CF
:10A54800083242E800310029F3D1D4F8800040B144
:10A55800724B8363FDF7ADFD30B1D4F88000836B97
:10A568007DE72046FFF731FFBDE8F081FFF72DFFBB
:10A57800C4F89050F8E7E06E012840F08980CE06D4
:10A5880040F18680D00640F1838010221A629A68D2
:10A5980051064BD5D4F8802011684A6892B2002A37
:10A5A800E2D0B4F85C009042DED9A4F85E200A68D4
:10A5B80092062FD453E8002F22F4807243E800213A
:10A5C8000029F7D103F1080252E8002F22F0010216
:10A5D80003F1080040E800210029F3D103F1080243
:10A5E80052E8002F22F0400203F1080040E8002161
:10A5F8000029F3D12022C4F88C20E16653E8002F0B
:10A6080022F0100243E800210029F7D1D4F8800095
:10A61800FDF71AFD02232367B4F85E30B4F85C1026
:10A62800C91A89B22046FFF7FFFE9DE7B4F85E20FD
:10A63800B4F85E00B4F85C1080B292B2002893D0EF
:10A64800891A89B200298FD053E8002F22F490721A
:10A6580043E800200028F7D1314D03F1080252E801
:10A66800002F2A4003F1080646E800200028F4D10C
:10A678002022C4F88C206067E06653E8002F22F09F
:10A68800100243E800200028F7D102232367C9E716
:10A69800CF0209D56E0207D54FF4801220461A6200
:10A6A800BDE8F04100F0A0BD08060BD502F080001F
:10A6B80005F40005284305D0A36F002B3FF454AFE1
:10A6C8002046CCE64F0611D556060FD553E8002F85
:10A6D80022F0400243E800210029F7D12023C4F8E2
:10A6E8008830A1672046F8F7EDFC3DE70D0206D556
:10A6F800500004D52046BDE8F04100F077BDCB01FD
:10A708007FF532AF002ABFF62FAF2046BDE8F041F3
:10A7180000F06BBD01000010200100041DA400081A
:10A72800FEFFFFEFD0F88C20B0F86010222A08B5A1
:10A73800036855D15B6A826D0B401370836D0133DA
:10A748008365B0F85E30013B9BB2A0F85E30B0F88C
:10A758005E309BB2002B42D1026852E8003F23F4DE
:10A76800907342E8003103680029F5D103F108022B
:10A7780052E8002F22F0010203F1080C4CE80021F6
:10A788000029F3D12022C0F88C20184A416793424F
:10A79800016705D1C26E012A0ED0F8F7A1FC1EE0B0
:10A7A8005A681102F6D553E8002F22F0806243E878
:10A7B80000210029F7D1EDE70022C26653E8002FF7
:10A7C80022F0100243E800210029F7D1DA69B0F835
:10A7D8005C10D20644BF10221A62FFF725FE08BD9E
:10A7E8009A6942F008029A61F9E700BF00800040C8
:10A7F800D0F88C20B0F86010222A08B5036852D12E
:10A808005A6A1140826D22F8021B8265B0F85E20F8
:10A81800013A92B2A0F85E20B0F85E2092B2002A07
:10A8280040D153E8002F22F4907243E80021002918
:10A83800F7D103F1080252E8002F22F0010203F1D8
:10A84800080C4CE800210029F3D12022C0F88C2004
:10A85800174A41679342016705D1C26E012A0ED09B
:10A86800F8F73EFC1EE05A681102F6D553E8002FAF
:10A8780022F0806243E800210029F7D1EDE70022A9
:10A88800C26653E8002F22F0100243E80021002995
:10A89800F7D1DA69B0F85C10D20644BF10221A6208
:10A8A800FFF7C2FD08BD9A6942F008029A61F9E70C
:10A8B800008000402DE9F74F0368B0F86080DF6939
:10A8C8001A689D68D0F88C1001922229044640F03D
:10A8D800B480B0F86890DFF86CA1DFF86CB100269E
:10A8E800B9F1000F01D0BB0621D4B4F85E309BB299
:10A8F800D3B1B4F868209A4216D9226802F1080345
:10A9080053E8003F23F08053083242E800312268C0
:10A918000029F2D14D4B636752E8003F43F0200312
:10A9280042E800310029F7D103B0BDE8F08F236871
:10A93800A26D5B6A03EA08031370A36D0133A36574
:10A94800B4F85E30013B9BB2A4F85E302368DF693F
:10A9580078072CD0F9070AD5019AD20507D5012125
:10A968001962D4F8901041F00101C4F89010B807AA
:10A9780009D5E90707D502211962D4F8901041F0EA
:10A988000401C4F890107A0709D5E80707D504210F
:10A998001962D4F8903043F00203C4F89030D4F828
:10A9A800903023B12046FFF710FDC4F89060B4F84A
:10A9B8005E309BB2002B93D1216851E8003F23F40D
:10A9C800807341E8003023680028F5D103F10802BC
:10A9D80052E8001F01EA0A0142E800100028F5D1F8
:10A9E80020215B45C4F88C10606720670AD059683D
:10A9F800090207D553E8001F21F0806143E80010E1
:10AA08000028F7D1E16E012913D1E66653E8001F4B
:10AA180021F0100143E800100028F7D1D969CA06CF
:10AA280044BF102119622046B4F85C10FFF7FCFC03
:10AA380056E72046F8F754FB52E79A6942F00802B5
:10AA48009A6171E7FEFFFFEF008000402DA7000824
:10AA58002DE9F74F0368B0F86080DF691A689D68D0
:10AA6800D0F88C1001922229044640F0B280B0F848
:10AA78006890DFF868A1DFF868B10026B9F1000F27
:10AA880001D0BB0621D4B4F85E309BB2D3B1B4F880
:10AA980068209A4216D9226802F1080353E8003F59
:10AAA80023F08053083242E8003122680029F2D1AD
:10AAB8004C4B636752E8003F43F0200342E8003103
:10AAC8000029F7D103B0BDE8F08F2368A26D596A59
:10AAD80008EA010122F8021BA265B4F85E20013AD7
:10AAE80092B2A4F85E20DF6978072CD0F9070AD55E
:10AAF800019AD20507D501211962D4F8901041F0C6
:10AB08000101C4F89010B80709D5E90707D5022153
:10AB18001962D4F8901041F00401C4F890107A0733
:10AB280009D5E80707D504211962D4F8903043F015
:10AB38000203C4F89030D4F8903023B12046FFF7D0
:10AB480044FCC4F89060B4F85E309BB2002B95D1F9
:10AB5800216851E8003F23F4807341E800302368FE
:10AB68000028F5D103F1080252E8001F01EA0A01A2
:10AB780042E800100028F5D120215B45C4F88C106C
:10AB8800606720670AD05968090207D553E8001F93
:10AB980021F0806143E800100028F7D1E16E012917
:10ABA80013D1E66653E8001F21F0100143E80010B6
:10ABB8000028F7D1D969CA0644BF10211962204676
:10ABC800B4F85C10FFF730FC58E72046F8F788FA2D
:10ABD80054E79A6942F008029A6173E7FEFFFFEFB3
:10ABE80000800040F9A7000838B5044603682169C9
:10ABF800A2681D68C0690A4361690A437D49024326
:10AC080029400A431A605A68E16822F440520A430C
:10AC18005A60794AA16993421CBF226A11439A6813
:10AC280022F06E4222F430620A439A60DA6A616A5C
:10AC380022F00F020A43DA62704A93421CD14FF0A5
:10AC4800B043D3F8883003F0030343F44033A3F54B
:10AC58004033013B022B00F2C780694A9B5CB0F588
:10AC6800004F40F08980082B24D8DFE803F061C04A
:10AC78008323802323236500624A934209D14FF03E
:10AC8800B043614AD3F8883003F00C0343F44023FF
:10AC9800E4E7594A93420DD14FF0B043D3F88830D6
:10ACA80003F44063B3F5006F1AD005D853B1B3F578
:10ACB800806F12D0012009E0B3F5406FFAD14FF44C
:10ACC80000400EE0FEF7D2FC58B900204FF0011307
:10ACD800A3660023C4E91D3338BDFEF7CFF8F3E7B8
:10ACE8004A4865684A4B626A05EB450133F8122009
:10ACF800B0FBF2F39942DDD8B3EB053FDAD8002375
:10AD08001946F6F701FF090241EA10616B080002D3
:10AD1800C0182A464FF0000341F10001F6F7F4FE8F
:10AD28003C4BA0F540729A42C4D82368D860CCE75F
:10AD3800FEF79CFC0028C8D06168354B626A33F87E
:10AD48001220B0FBF2F24B0803EB42034FF6EF720E
:10AD5800B3FBF1F3A3F110019142ABD823F00F023A
:10AD6800216892B2C3F342031343CB60ADE7FEF709
:10AD780085F8DFE72548DFE7082B9BD801A252F8C2
:10AD880023F000BFD5AD0008E1AD0008EDAD000827
:10AD9800BDAC0008E7AD0008BDAC0008BDAC0008BC
:10ADA800BDAC0008B1AD00084FF400406368616AAB
:10ADB800174A32F81120B0FBF2F000EB5300B0FB59
:10ADC800F3F04FF6EF73A0F11002ACE7FEF74EFC7C
:10ADD80000283FF47AAFE9E7FEF758FCF8E7FEF7FA
:10ADE8004DF8F5E70948E1E7B0F5004FF4D1FEF773
:10ADF8004DFC9FE7F369FFCF008000400038014019
:10AE0800E04F010800440040E34FF5070024F40038
:10AE1800F04F0108FFFC0F00836ADA0710B506D56A
:10AE28000168C46A4A6822F4003222434A609C07D7
:10AE380006D50168046B4A6822F4803222434A60CE
:10AE4800590706D50168446B4A6822F480222243D8
:10AE58004A601A0706D50168846B4A6822F40042E2
:10AE680022434A60DC0606D50168C46B8A6822F46E
:10AE7800805222438A60990606D50168046C8A6864
:10AE880022F4005222438A605A060FD50168446CA6
:10AE98004A6822F480122243B4F5801F4A6005D123
:10AEA8004A68846C22F4C00222434A601B0606D515
:10AEB8000268C16C536823F400230B43536010BD30
:10AEC8002DE9F041DDF8188004460E4615461F4668
:10AED8002268D36936EA03030CBF01230023AB427F
:10AEE80001D0002027E0B8F1FF3FF2D0F7F720FEAD
:10AEF800C01B4045206802D8B8F1000F1DD150E8AA
:10AF0800003F23F4D07340E80032002AF7D100F163
:10AF1800080353E8003F23F0010300F1080141E86A
:10AF28000032002AF3D12023C4F88830C4F88C30CA
:10AF380084F884200320BDE8F08103685A07C7D548
:10AF4800C3691B05C4D54FF40063036250E8003F92
:10AF580023F4D07340E80032002AF7D100F1080347
:10AF680053E8003F23F0010300F1080141E80032F3
:10AF7800002AF3D12023C4F88830C4F88C30C4F8F0
:10AF88009030D5E773B504460026C0F89060F7F70F
:10AF9800CFFD23681B681A07054619D423681B6868
:10AFA8005B070AD56FF07E43009300222B464FF4CF
:10AFB80080012046FFF784FFB0B900202023C4F8A1
:10AFC800883084F88400C4F88C30E06620670CE090
:10AFD8006FF07E430093324603464FF4001120463B
:10AFE800FFF76EFF0028D9D0032002B070BD10B55E
:10AFF800044650B3D0F888301BB980F88430F7F78E
:10B008004DFF22682423C4F88830136823F0010315
:10B0180013602046FFF7E8FD012816D0A36A13B194
:10B028002046FFF7F9FE23685A6822F490425A60D6
:10B038009A6822F02A029A601A6842F001022046B1
:10B048001A60BDE81040FFF79DBF012010BD000049
:10B0580030B581658168A0F85C200023B1F5805F78
:10B06800A0F85E20436735D10369002B40F2FF1337
:10B0780018BFFF23A0F860300023C0F890302223C7
:10B08800C0F88C30016801F1080353E8003F43F031
:10B098000103083141E800340368002CF2D1456E01
:10B0A80084680169B5F1005F34D1B0F86850954201
:10B0B80030D8B4F5805F1DD1254A264C002918BF29
:10B0C80022464267C1B153E8002F42F4807243E838
:10B0D8000021F7E729B90369002B14BF7F23FF2359
:10B0E800C8E7B1F1805FC5D10369002B0CBF7F238E
:10B0F8003F23BFE7174AE4E703F1080252E8002FAD
:10B1080042F0805203F1080040E800210029F3D101
:10B11800002030BDB4F5805F0FD10F4A0F4C0029D5
:10B1280018BF2246426751B153E8002F42F490728B
:10B1380043E800210029F7D1EAE7084AF2E753E893
:10B14800002F42F0200243E800210029F7D1DFE771
:10B1580059AA0008BDA80008F9A700082DA70008EB
:10B16800D0F88C30202B30B415D1B9B1B2B100234E
:10B178000468C3660A4B9C420AD063681B0207D561
:10B1880054E8003F43F0806344E80035002DF7D1D0
:10B1980030BCFFF75DBF022030BC70470120FBE7E1
:10B1A80000800040436E30B52BB90123A0F86A3007
:10B1B800A0F8683030BD0368094D9A689968094C51
:10B1C800490FC2F342626B5C615CDB00B3FBF1F3D5
:10B1D800A0F86A30AB5CA25CDB00B3FBF2F3E7E7F4
:10B1E80010500108085001087047704770471FB594
:10B1F80004AB03E9060090F88430012B04463AD0EA
:10B20800012380F884302423C0F8883003681A6842
:10B2180022F001021A609A6822F440120A439A60E6
:10B2280071B95A68BDF80C009DF80E1022F0100292
:10B2380002435A605A6822F07F4242EA01625A6029
:10B248001A6842F001021A60F7F772FC6FF07E424A
:10B25800034600924FF4800100222046FFF730FE9B
:10B2680038B92023C4F88830002384F8843004B027
:10B2780010BD0320F8E70220F9E790F88430012B8D
:10B288000FD0012380F88430016851E8002F42F084
:10B29800020241E80023002BF6D180F884301846DA
:10B2A80070470220704710B590F88430012B04468F
:10B2B80017D02423C0F8883003681A68196821F069
:10B2C8000101196042F000524FF0005141661A60C6
:10B2D800FFF768FF2023C0F88830002084F8840036
:10B2E80010BD0220FCE770B590F88430012B0446AD
:10B2F80017D005682423C0F888302E682B6823F0FF
:10B3080001032B60AB6823F060431943A960FFF782
:10B3180049FF20232E60C0F88830002084F884007C
:10B3280070BD0220FCE770B590F88430012B04460C
:10B3380017D005682423C0F888302E682B6823F0BE
:10B3480001032B60AB6823F060631943A960FFF722
:10B3580029FF20232E60C0F88830002084F884005C
:10B3680070BD0220FCE7000038B5094D002455F8EF
:10B37800043B33B90134E3B2052B64B2F7D10020A2
:10B3880038BD002CF6D01B6998470028F2D0F7E7A3
:10B39800701000207FB50A2301A88DF8043003F04F
:10B3A800D9F80038044B059A1A6018BF01204042AA
:10B3B80007B05DF804FB00BF6810002070B50446B4
:10B3C8000B46144962784A700020A2780A72087005
:10B3D8001A884A729A788A72DB780B746368CB6031
:10B3E8000D4B1B68DA6A2AB1237803F0FB030B2B99
:10B3F80000D09047094E002556F8043B1BB19B6AC4
:10B408000BB1204698470135EBB2052B6DB2F3D14D
:10B4180070BD00BF480800206C100020701000208C
:10B4280070B5044611480123037063784370A3780C
:10B438008372E368C360E3780376236943762379EC
:10B4480043720B4B1B689B6A03B19847094E002552
:10B4580056F8043B1BB1DB690BB120469847013510
:10B46800EBB2052B6DB2F3D170BD00BF5C080020B4
:10B478006C1000207010002038B501F011FE0C4D42
:10B48800052455F8043B5BB15B694BB155F8043CA6
:10B498009B682BB1984718B155F8043C5B699847ED
:10B4A800013C14F0FF04ECD1BDE83840FFF75CBF65
:10B4B80070100020014B1868704700BF681000200A
:10B4C80000B58BB0012368468DF8003002F0BCFC53
:10B4D80038B99DF80400003818BF01200BB05DF89A
:10B4E80004FB0020FAE7000030B58BB0054601F0F8
:10B4F800BBFD0446002839D1FFF7E2FF012838D107
:10B5080068468DF8004002F09FFC10B14FF0FF3004
:10B5180004E09DF80430AB4202D100200BB030BDEE
:10B52800012DF3D0022D11D0002DF7D1002BF4D02E
:10B5380068468DF8045002F099FD0028E6D10E4BBC
:10B548001B681B6B002BE8D09847E6E7002BDDD182
:10B5580068468DF8045002F089FD0028D6D1064BC4
:10B568001B681B6B002BD8D02846EDE76FF0010055
:10B57800D4E76FF00200D1E76C10002070B5324CB0
:10B58800324B94F9042094F9055090B00126022812
:10B598008DF804608DF809208DF80A500AD18DF8CD
:10B5A8000800D871197202F09FFB01A802F0D2FFBF
:10B5B80010B070BD4FF480701A715D71D880197227
:10B5C800234B8DF808601B7853BB1E2306A88DF803
:10B5D8001C208DF8183002F049FD1F238DF8183013
:10B5E80006A823798DF81C3002F040FD21238DF840
:10B5F800183006A863798DF81C3002F037FD202337
:10B608008DF8183006A863798DF81C3002F02EFDED
:10B6180028238DF8183006A80E4B079302F026FD54
:10B6280002F062FB012306A88DF818308DF81C3053
:10B6380002F01CFD084B1B685B6A0BB10348984776
:10B648006078FFF751FFB3E784100020300800202E
:10B6580064100020000300016C10002008B501F000
:10B6680003FD40B9FFF72CFF012806D0084B197AD3
:10B67800D879FFF783FF012008BD064B1B68DB68FC
:10B6880098470028F7D1BDE80840FFF76DBE00BF16
:10B6980030080020701000202DE9F04186B00546E2
:10B6A8000C46164601F0E0FC002840F08D8001F0C1
:10B6B800EDFC40B9FFF704FF012807D0444B197A85
:10B6C800D879FFF75BFF6FF002046DE0414F3B68EC
:10B6D800DB68984730B13A682B7812789A4201D0E3
:10B6E800002B6ED13C4FDFF8F4803C72003C18BF51
:10B6F800012498F8043068788DF8044069468DF87C
:10B70800123002F049FB002840D000238DF80430A5
:10B718000393ADF810306FF0060495E80300304B42
:10B7280083E8030098F80430BB72314601A803F09F
:10B7380009F82C4B059A1A6011283FD801A353F831
:10B7480020F000BFABB70008D1B70008C5B70008A4
:10B75800C5B70008C5B70008C5B70008C5B70008D1
:10B76800CFB60008C5B70008C5B70008C5B70008B8
:10B77800BFB70008C5B70008C5B70008D1B70008AB
:10B78800D1B70008D1B70008B9B700082B788DF8F1
:10B7980008306B78ADF810306B6803934FF0FF34C6
:10B7A800BBE7E31D18BF0024204606B0BDE8F081C2
:10B7B8006FF00404F8E76FF00504F5E74FF0FF3485
:10B7C800F2E76FF00304EFE76FF00104ECE700BF66
:10B7D80030080020701000205C0800208410002031
:10B7E8006C0800206810002010B504468AB018B90B
:10B7F8004FF0FF300AB010BD002368468DF80030C6
:10B8080002F022FB0028F3D19DF804302370F1E701
:10B81800F0B587B000220B462A498DF8072001228F
:10B828000A7042784A700446002A41D102790A72A5
:10B838001A884A729A788A72DB780B740369CB602B
:10B84800C378214D8DF80830037B8DF80930836863
:10B8580003932B68DB6A0BB102A898472B689B6B94
:10B8680013B1227E02B19847184E0025374656F884
:10B87800043B53B11A6A42B11A78E3789A4219D153
:10B8880056F8043C20461B6A98470135EBB2052B55
:10B898006DB2ECD10DF10700FFF7A6FF63793BB15C
:10B8A8000021012204A8ADF810100591FFF7F4FE5D
:10B8B80007B0F0BD002DE8D13B68DB689847002849
:10B8C800DED1E2E7480800206C100020701000204C
:10B8D80010B504468AB018B94FF0FF300AB010BD51
:10B8E8001F2368468DF8003002F0AEFA0028F3D125
:10B8F800024A9DF9043023701371EFE78410002089
:10B9080000B58BB02223019068468DF8003002F014
:10B91800ADFB003818BF012040420BB05DF804FBB6
:10B9280070B5634C014618228EB0204605F066FFBC
:10B93800F8F734FE23784068012202FA03F1014047
:10B9480004D15C4B084607F04FFFFEE75A495B48B5
:10B958001A4602F011F818B14FF0FF300EB070BD62
:10B96800262304A88DF8103002F080FB544E554D64
:10B97800002870D1012333702B68DB690BB10020DC
:10B988009847262304A88DF8103002F05DFA059B2D
:10B9980093F84820227093F8182193F81A316270AE
:10B9A800A370454BD3E9020105F01AFE05460028AD
:10B9B800D2D1454E062304A88DF8103002F044FA7F
:10B9C800059B736104A802F051FB022304A88DF8BB
:10B9D8001030059602F038FA0836032304A88DF8CB
:10B9E8001030059602F030FA0F2605F0BDFE01234F
:10B9F80004A88DF814308DF8106002F037FB10237E
:10BA08000DEB03008DF810308DF8145002F02EFB6A
:10BA180004238DF8103004A8A3788DF8143002F0B0
:10BA280025FB39238DF8103004A86369059302F0CB
:10BA38001DFB02A920788DF8086003F051FF00383B
:10BA480018BF0120E0711420FFF75AFFE07903F0D6
:10BA580003F8284682E727238DF810302B681B69E6
:10BA680043B104A802F0F0F92B6805981B694FF45C
:10BA7800EE619847262304A88DF8103002F0F6FAF4
:10BA880050B9012304A88DF8103002F0DDF99DF8B3
:10BA98001430002B7FF46EAF3378002B7FF46CAF3B
:10BAA800052204A88DF81020059302F0DFFA78E744
:10BAB80084100020185001089C100020B4100020A9
:10BAC800641000206C1000204C10002037B50023B3
:10BAD8000D4601930446C0B900F0D0FA0190019BCD
:10BAE800C3B10E4A0E4942F824300E4ADA620E4AB1
:10BAF8001A630E4A5A630E4A126892699A61284676
:10BB08005B68F2229847002006E001A900F0BCFA21
:10BB18000028E4D04FF0FF3003B030BD7010002093
:10BB2800580F002085B50008A1B600089DB300088D
:10BB38006C100020154B07B51860154B154A1A6094
:10BB4800154A5A60154A9A60154ADA60154B026818
:10BB58001A6042685A6082689A60C268DA60124A5B
:10BB680001911A61114982695A610020FFF7AEFFFD
:10BB780048B901A800F086FA003818BF01204042F1
:10BB880003B05DF804FB4FF0FF30F9E76C100020BC
:10BB9800B410002029B4000819B8000835BC000802
:10BBA800C5B300089C10002099F800083C08002044
:10BBB80051B118B1012804D000207047044B0B6024
:10BBC8007047044B0B60F7E74FF0FF30704700BF3A
:10BBD800000300010300010108B502F059FF002825
:10BBE80014BF6FF00100002008BD08B502F0A4F8EA
:10BBF800002814BF6FF00100002008BD10B50446EE
:10BC08008AB018B94FF0FF300AB010BD202368463B
:10BC18008DF8003002F018F90028F3D1024A9DF996
:10BC2800043023705371EFE7841000202DE9F041B0
:10BC38002F4D304F00232B7043786B703B689B6A05
:10BC48008AB004460BB128469847DFF8AC80002636
:10BC580058F8043B1BB15B6A0BB120469847013684
:10BC6800F3B2052B76B2F3D12378052B2FD00C2B0A
:10BC780035D0012B25D1214C062368468DF800309C
:10BC880002F0E2F80199E07905F0F0FC10B91C4BDC
:10BC9800019A5A611B48FFF71BFE1B48FFF7AEFFCE
:10BCA8006B788BB9A371194B5878FFF71DFC3B686B
:10BCB8005B6A0BB1114898476B7813B9E07905F0C6
:10BCC80065FD0AB0BDE8F081FF23A371EFE7104BD3
:10BCD80001225A74227A9A74627ADA74F1E76378E4
:10BCE800002BEED00AB0BDE8F041FFF753BB00BF10
:10BCF8005C0800206C100020701000203008002024
:10BD08004C10002034080020350800208410002042
:10BD18004808002030B58BB0FFF767FF0446F0B93C
:10BD280003F0BEFD831C1DD0F8B9134D2B685B6969
:10BD3800DBB1262368468DF8003002F085F82B68C1
:10BD480001985B694FF4EE61984703F0BBFD78B941
:10BD58002CB9094B1B68DB690BB1012098472046B9
:10BD68000BB030BD6FF00704EFE74FF0FF34ECE79E
:10BD78004FF0FF34F3E700BF6C10002030B5064DDC
:10BD8800064C30B129B12860A1606271012323708B
:10BD980030BD00232B60FAE7F0100020C41000200B
:10BDA800014B1878704700BFC4100020024B187868
:10BDB80000B15878704700BFC410002070470000D9
:10BDC800064B1A784AB15A783AB10278012A04D156
:10BDD800027912B19A8901329A817047C410002001
:10BDE800074B1A7852B15A7842B10278052A05D120
:10BDF800017A427AD973012098731A74704700BF88
:10BE0800C410002013B51A4C23783BB363782BB3C6
:10BE1800A27BA36862B10022A2730322A271052249
:10BE28001A70E27B5A70227C9A700122A27004E098
:10BE3800A278012A14D0042AF7D0E0228DF8002035
:10BE48000C48A27901938DF8012008F049F80A4BB3
:10BE58001B6B1BB1E17801226846984702B010BD00
:10BE68000222A271A2895A70110A1970E5E700BF6F
:10BE7800C4100020D810002078080020FFF7C2BFA7
:10BE880030B5794C23788DB0002B43D0437B002B01
:10BE980040D0657825B1837B13B9A3890133A38189
:10BEA800C178E02936D1002D36D1027B042A31D160
:10BEB8008368187801282DD1587801282AD19878D4
:10BEC800012827D1DB78012B24D102206380A071BF
:10BED800E56002A863708DF80C3021718DF8082098
:10BEE800257402F0C3F8284602F0B6FD5F4B1B68C4
:10BEF8005B6803B1984700225D4B00924FF0FF3119
:10BF08005C4807F041FF41F288315A4808F022F8AE
:10BF1800FFF778FF0DB030BD83681A78A2700A2A3F
:10BF2800F8D8DFE802F0062124282A3D44658D8FE1
:10BF38009900504807F086FF00236370A3814B4C9B
:10BF480004238DF80830236802A81B788DF80C307C
:10BF580002F08CF82368587802F07EFD23689B680D
:10BF6800002BD7D09847D5E70223A371D2E740F238
:10BF780001136380CEE70123FBE7A568037BA37168
:10BF880004222A7062799A4228BF1A460023013394
:10BF9800D9B28A42BED98168C95C0131E954F6E751
:10BFA80005238DF8083002A802F0D4FAB2E7314828
:10BFB80007F048FF00236370A3812C4C04238DF8FD
:10BFC8000830236802A81B788DF80C3002F04EF870
:10BFD8002368587802F040FD23689B6803B19847AE
:10BFE800254BDB6A002B95D001210220984791E769
:10BFF800027B032A0DD106228DF80820B3F8013000
:10C008005BBAADF80C3002A802F0A4FA0123A370C1
:10C0180080E7072AF7D18DF80820B3F8012052BA33
:10C02800ADF80C201A79D978120242EA01425979FE
:10C038000A4364214A4304929B798DF81430E2E75D
:10C048000A23AEE700228DF808205B788DF80C30C3
:10C0580002A802F00BF85DE70D228DF808205B7846
:10C068008DF80C309FE700BFC4100020F0100020AE
:10C0780085BE0008D81000207808002000487047C6
:10C0880078080020002070474FF0FF30704700000C
:10C09800044B054A93F81831022B18BF062382F87F
:10C0A8008034704764180020D81F0020034BD3F851
:10C0B800483313B15B6903B118477047D81F002094
:10C0C800034A137843F002031370FFF7EFBF00BF72
:10C0D800D41F00201FB50A4B8DF8090093F87C2067
:10C0E8008DF80A2093F88C2093F848000D3202A9A5
:10C0F8008DF8082003F0F4FBC0B205B05DF804FB2E
:10C108006418002010B50D4C04F57D7007F09AFEF8
:10C1180094F8103413B1012384F80F34084B93F8C2
:10C128001831022B02BF94F8813443F0100384F8CD
:10C138008134BDE81040FFF7B9BF00BFD81F002009
:10C148006418002010B50C4CD4F8403343F0800339
:10C15800C4F8403394F8103413B10020FFF7D2FF2D
:10C1680094F8813423F0120343F0120384F88134E5
:10C17800BDE81040FFF78CBFD81F00202DE9F04123
:10C188002C4D95F81831022B07460E4602D02A4B43
:10C19800DB6A984702F01BFD044628B1022002F032
:10C1A8000CFD002002F00EFD95F81831012B17D177
:10C1B80002F00FFD804630B1002002F0FFFC0020A5
:10C1C80002F001FD444602F006FD48B1002002F0ED
:10C1D800F6FC002002F0F8FCBDE8F041FFF758BF7C
:10C1E800002CF9D1154C94F8802494F81034B2B985
:10C1F8000BB184F83574384602F090FEE86A07F00F
:10C20800E7FDD4F8B4339842E6D30D4807F01AFE98
:10C2180094F8813443F0100384F88134DCE70BB1DF
:10C2280084F83564304602F079FE95F81831022B0F
:10C23800EED1D1E76418002020570108D81F00204C
:10C2480070230020074A10B5137843F001031370D8
:10C25800FFF72CFFBDE81040034B0122002102200C
:10C2680007F0C2BAD41F002061500108074A10B570
:10C27800137843F004031370FFF718FFBDE810406C
:10C28800034B01220021022007F0AEBAD41F002080
:10C29800715001082DE9F0410F4616461D468046AB
:10C2A80007F08CFD0A4A0B4C1378278143F00803EA
:10C2B800C4E90008137066812573FFF7F7FEBDE82F
:10C2C800F041054B01220021022007F08DBA00BF82
:10C2D800D41F0020E02400208150010813B507F086
:10C2E8006DFD0D4B6C461860204607F0BBFC94E8CA
:10C2F80003000A4A0A4B83E80300137843F010034B
:10C308001370FFF7D3FE074B01220021022002B071
:10C31800BDE8104007F068BAF0240020D41F0020C0
:10C32800102300208E5001082DE9F04192B00646F6
:10C3380002F04DFC002840F05681AC4D95F81831BC
:10C34800012B09D02B6BAA4C93B194F80431BBB1E3
:10C35800042B6FD0032003E002F03BFC18B10F2040
:10C3680012B0BDE8F08102F036FC0028EAD0F6E70A
:10C37800B5F81E31D4F81424013B53432B63E4E78A
:10C388009C4803F0E4F9002840F0298194F80C3126
:10C3980023802B6B0C930DF1180895F839308DF824
:10C3A8003830404695F81C318DF83A3007F080FC5B
:10C3B800D5F82431009302AF98E80600D5F820316B
:10C3C800384607F00CFC97E803000FAB83E803003E
:10C3D800EB6A0D9300238DF844302388ADF846307E
:10C3E80095F82C3101228DF839201BB98DF844209D
:10C3F8008DF83930804B0093804B95F84800A3F1B5
:10C4080073020CA903F0E1FAC0B10B28A8D1D4F843
:10C41800841499B1002EA3D0D4F84033784843F05F
:10C428002003C4F8403307F095FD754807F058FD20
:10C43800002095E76F4803F0BEF9A4E795F8487027
:10C4480095F9693095F9392095F87D106D4E384683
:10C4580003F0CDFA009641B2EB6C95F850203846BF
:10C46800143603F063FA0096EB6C95F8502095F9B2
:10C47800701095F8480003F059FAD4F8C413AB6D5E
:10C48800D4F8D8230B44C4F8B033EB6D1344C4F884
:10C49800B43394F80431042B07D02B6E0B44C4F842
:10C4A800B0336B6E1344C4F8B4330023089395F883
:10C4B8002C3183B108A802F061FC00284AD195F913
:10C4C800390094F837629DF82070FFF703FE3E4468
:10C4D80080B2B0423CD300238DF8133095F8393040
:10C4E8008DF8213095F838308DF82230D5F8803025
:10C4F8000993D5F884300A93238894F81164ADF829
:10C508002C3095F84800404B8DF820600DF113024F
:10C5180008A903F01FFA012384F8353495F8393057
:10C5280084F836349DF8133084F83734D4F814344A
:10C53800C4F84464C4F83C34C4F84C3402F04DFBED
:10C5480050B1D4F8140402F05AFB28B1102007E7C0
:10C55800082005E7132003E795F81831012B01D1CE
:10C5680002F04FFB02F03CFB0023059394F80431E2
:10C5780095F9395094F81164BBB1042B7FF4EAAEF5
:10C5880005A802F037FE60BB94F80C341BB994F888
:10C598000E34012B02D9059B013B0593154B0598D9
:10C5A8003246E9B202F098FE02E0124802F06CFE50
:10C5B800A8B9D4F8403394F80C11218043F0020351
:10C5C800C4F8403394F8103423B994F80C34013388
:10C5D80084F80C340D4B0E489B6A984728E71120C5
:10C5E800BEE61220BCE60E20BAE600BF64180020A2
:10C5F800D81F0020E0200020941800205C24002090
:10C608004023002090230020EC230020205701081D
:10C61800DA1F002073B5144C144D04F57876EB6CD2
:10C6280095F8502095F9781095F84800009603F091
:10C638007DF940F2012395F84800A4F8F23304F29A
:10C648001C42314603F07EF958B194F81C3484F842
:10C658005E34074B00205B6B984794F8F33384F8FB
:10C66800803402B070BD00BFD81F002064180020BD
:10C6780020570108F8B5334D95F81841012C0646A6
:10C688004BD0022C51D064B938B9D5E91B0105F15A
:10C69800740383E803002046F8BD01283DD0022832
:10C6A80001D00324F7E7284F85F8180107F5737EB2
:10C6B800BEE80F0007F5787CACE80F00DEF8003024
:10C6C800CCF8003095F8E93087F8F363E3B195F8D2
:10C6D8000031022B18D1D5F804316B67C7F8E43361
:10C6E80095F87D3095F8082187F8F03395F88C3067
:10C6F80085F8782087F8F13397F8112487F8E02334
:10C7080040F20133A7F8F233002387F810340F4BB7
:10C71800DB6A9847FFF77EFFBDE702F063FA04463D
:10C728000028B8D185F81861B5E70028B9D1064BBB
:10C7380085F81801062283F88024044BDB6A9847A1
:10C748003446A8E764180020D81F002020570108A5
:10C75800F0B5484C484EB4F8DC202287D4E92D01C6
:10C7680094F8B12084F8692004F16C0282E803008F
:10C77800D4E92F0104F1740282E80300B4F8C4205C
:10C78800A4F87C20D4F8CC20C4F884208FB0D4F846
:10C79800D020D4F8C810C4F888200025374AC4F837
:10C7A80080100123A4F81E31C6F80C24C4E94E55A4
:10C7B80084F82C51A56284F81B5184F83A50C4F8C7
:10C7C8003051A4F8345186F8105484F841518DF84A
:10C7D800143004F5087394F84800A4F84251039300
:10C7E80003A904F52D73049303F088F8E36EC6F8E3
:10C7F800D03394F87D3086F8DC3394F88C3086F8A2
:10C80800DD334FF48073A6F8DE3386F8CC5306F593
:10C8180073770FCF06F578740FC43B68236040F236
:10C828000123A6F8F233D6F8483386F81154CDE937
:10C8380001551BB15A685B6901920293104B06932C
:10C84800A3F144020792A3F1140208920D4A0A9236
:10C8580025330993A2F19C030B93A2F198030C933F
:10C8680001A9131D06A802F274620D9302F0A4F93F
:10C878000FB0F0BD64180020D81F0020000101008F
:10C888003424002048190020F8B50D4F0D4C0E4EE9
:10C898000D4607F0D7FA3B6B984796F8480004F224
:10C8A8001C42294603F04EF848B194F81C3484F829
:10C8B8005E34706D7B6B9847EB7C84F88034F8BDF0
:10C8C80020570108D81F0020641800200D4890F850
:10C8D800113480F8B8330C4B93F8692080F8BB23E7
:10C8E80093F87D2093F88C3080F8C933002380F8C2
:10C8F800C823A0F8CA3300F56E7100F56070FFF721
:10C90800C3BF00BFD81F0020641800200F4890F84C
:10C918008034CBB190F8113480F8CC330C4BDA6EFC
:10C92800C0F8D02393F87D2093F88C3080F8DD335D
:10C938004FF4807380F8DC23A0F8DE3300F57371C0
:10C9480000F56670FFF7A0BF704700BFD81F002032
:10C958006418002070B5344C2421204604F064FF8C
:10C96800636A984218BF60624FF01C012F4814BFD9
:10C978000125002504F058FF636C984218BF6064D5
:10C988004FF0FC012A4818BF45F0020504F04CFF9F
:10C99800D4F84431984218BFC4F844014FF0D40188
:10C9A800244818BF45F0040504F03EFFD4F81C32B3
:10C9B800984218BFC4F81C024FF090011E4818BFD7
:10C9C80045F0080504F030FFD4F8B032984218BF9B
:10C9D800C4F8B0024FF49461184818BF45F0100528
:10C9E80004F022FFD4F85437984218BFC4F854070B
:10C9F8004FF01401124818BF45F0200504F014FF49
:10CA0800D4F86C3798420F4B18BFC4F86C07D3F8AA
:10CA1800483318BF45F040052BB11B691BB12846A8
:10CA2800BDE87040184770BD641800208C180020BD
:10CA3800AC180020AC190020841A0020181B002014
:10CA4800BC1F0020D81F00202DE9F04F91B0002610
:10CA5800BD4F8DF81560054688469346ADF81860B9
:10CA6800B146C14502D311B0BDE8F08F15F80900F1
:10CA780002F0C2F948444045F5DC15F8093009F1DF
:10CA88000104023BE4B2112BEDD801A252F823F0C5
:10CA9800E1CA000811CB0008D1CB0008FDCB000883
:10CAA8008DCC0008B1CC000825CD000859CD000870
:10CAB800D7CD00086FCA00086FCA000837CE000833
:10CAC8006FCA00086FCA0008EDCE000813CF00082F
:10CAD80057CF000895CF0008052002F039FA88B131
:10CAE8000521002002F0F8F92B5D87F8503409F190
:10CAF800030409F102095FFA89F9E4B215F809306B
:10CB080087F85134A146ACE700238DF816308DF82C
:10CB180017308DF81C308DF82030002E52D18B4EF6
:10CB2800631E2B440D9396F81A318DF83A3096F817
:10CB38007C308DF8393096F839308DF83B3096F8DE
:10CB480038308DF83C3096F868308DF83D30D6F89E
:10CB580028310C9308AB019307AB009396F8480073
:10CB6800A8EB09090DF117030DF116020CA98DF8B0
:10CB7800389002F0FBFE8DF8150000F0070007283A
:10CB88000BD19DF8163086F839309DF8173086F8A5
:10CB980038309DF81C3086F8683000264FF00509BB
:10CBA80006E001220DF11501032002F03BF80136E1
:10CBB800F2B29DF82030B3FBF9F19142F1D8013B74
:10CBC8002344DCB201269DE72B5D604903F00F0387
:10CBD800012281F81B3109F1020902FA03F3A1F8D5
:10CBE8001E315FFA89F9002206A9042002F01AF81A
:10CBF8004C4687E707238DF815302B5DC3F30212E7
:10CC080003F00F038DF8303009F10303DBB28DF820
:10CC18003120EA5C09F10403DBB209F10504EB5C9D
:10CC280009F102095FFA89F91B0443EA022315F89E
:10CC38000920DFF8189113436422534399F84800F8
:10CC48000D930CA902F0A1FE00F00703072BE4B234
:10CC58008DF815000ED19DF8303089F8703089F8BC
:10CC680078300D9BC9F86C30C9F874309DF83130B4
:10CC780089F869308DF81800012206A9052001F00D
:10CC8800D1FF3FE7D7F8483363B11B6853B19847E2
:10CC98000BF03F038DF818008DF81930022206A911
:10CCA8000620ECE7FF20F3E703238DF815302B5D12
:10CCB8008DF824300CAB089309F10303DBB209F1BA
:10CCC8000604EA5C09F10403DBB208A9EB5C1B0467
:10CCD80043EA022309F10202D2B209F10509AA5C6A
:10CCE8001343642253435FFA89F90C9300230D938D
:10CCF80015F809308DF83830144B93F8480002F0D5
:10CD08004AFEC3B20028E4B28DF81530FFF6FAAE39
:10CD18008DF81830012206A90720B0E72B5D03F033
:10CD28000F03012B4FF47A7238BF01235343074A8C
:10CD380009F10209936503F57A73D3655FFA89F9F6
:10CD4800002206A9082051E7D81F002064180020F7
:10CD58002B5D9C4CC3F340128DF81D2094F84800BD
:10CD6800C3F3001207A903F00F038DF81C208DF8F8
:10CD78001E3002F016FE09F1020901305FFA89F946
:10CD88003FF436AFBDF81C308F4AA4F87C309DF8CC
:10CD98001E309DF81CA0D05CF4F738FE0223C4F8BE
:10CDA80080000CA994F848008DF830308DF832A036
:10CDB80002F096FD94F93930089040B29842B8BF15
:10CDC800184684F83900002206A909200EE7032333
:10CDD8008DF815302B5D8DF8303009F10303DBB287
:10CDE80009F10504EA5C09F10403DBB209F102095F
:10CDF800EB5C5FFA89F91B0443EA022315F8092062
:10CE08001343642253430D936E4B0CA993F84800C7
:10CE180002F0CDFDC3B20028E4B28DF81530FFF65C
:10CE280071AE8DF81830012206A90A2027E70A20DA
:10CE380002F08EF800283FF465AE0A21002002F0C7
:10CE48004BF80023ADF8263009F10203DBB24FF4AA
:10CE58007A71EA5C09F10303DBB20DF1300AEB5C8D
:10CE68001B0443EA02232A5D134309F10402D2B2E8
:10CE780009F1060409F10509AA5C5FFA89F943EA90
:10CE8800026315F8092003934A4312125046ADF87D
:10CE9800242006F0E7FE039B03F1965303F5A9133C
:10CEA80003F5EC530893D7F83C3300930DF12009B0
:10CEB80099E80600D7F838330AA806F090FE0B9BCD
:10CEC80000939AE806000A9B484606F06DFE99E82A
:10CED800030006F09FFE01F08FFE0123E4B287F8FD
:10CEE80030340FE60D2002F033F800283FF40AAE84
:10CEF8000D21002001F0F0FF97F88034043B012B4E
:10CF08007FF600AE01F074FEFCE509F10203DBB226
:10CF18002A5DE95C09F10303DBB209F10504EB5C66
:10CF280009F104095FFA89F91B0415F8090043EAB5
:10CF3800012313436421594300F00F0001F059FE07
:10CF4800E4B28DF81800012206A9112097E60E20F8
:10CF580001F0FEFF00283FF4D5AD0E21002001F0BE
:10CF6800BBFF09F10203DBB2184AE85C2B5D1268CB
:10CF780009F1040409F103095FFA89F943EA002079
:10CF880015F80910E4B201F036FEBBE52A5D09F197
:10CF9800020309F1040409F10309DBB25FFA89F914
:10CFA800E95C15F809301B0443EA012313436420A4
:10CFB800584301F022FEE4B28DF81800012206A9B8
:10CFC80013205CE6641800209B500108E024002030
:10CFD8000E4B93F88124920703D593F87F24012AF6
:10CFE80006D90B4A92F81A1111B1916A013191626E
:10CFF800002283F80C2483F8102483F80F24D3F834
:10D00800402322F00202C3F840237047D81F0020B3
:10D018006418002010B5124C04F55A7006F012FF7F
:10D02800D4F84033012023F02003C4F84033FFF73D
:10D038007BF998B10B2811D00A4B93F8393084F852
:10D048003634092094F80E3484F8393484F83504D9
:10D0580001F064FFBDE81040FFF7BABF10BD00BF84
:10D06800D81F002064180020074BD3F84023012A5A
:10D0780006D03AB993F88204013818BF01207047E6
:10D088000020704701207047D81F0020034BD3F8B9
:10D098004003431E58425841704700BFD81F002024
:10D0A8002DE9F04FA5B0EFF3108172B6C04A002009
:10D0B8001368106081F31088BE4C002B00F0DA80F2
:10D0C800D9065FFA83FB6BD5BB4D95F81831022B57
:10D0D80002D0BA4BDB6A9847EFF3108872B6B84FA4
:10D0E80006F06CFE3E68D4F8B013361A3144B548E1
:10D0F80006F030FFB34806F0F3FED4F8B413B24894
:10D10800314406F027FFB04806F0EAFE88F310889D
:10D1180095F81831022B02D094F810348BB11623ED
:10D128000EA995F848008DF8383002F0D9FBD4F8EC
:10D13800B4130C900144A54806F00CFFA34806F070
:10D14800CFFE3B6894F81124EB620AAF38468DF89D
:10D158006020199306F0ACFDD5F82431009304AE95
:10D1680097E80600D5F82031304606F038FD96E8F5
:10D1780003001BAB83E80300D4F814341A9395F822
:10D188002C3195F84800003B18BF012318A98DF8E9
:10D19800613002F0AEFB94F810340BB984F83534E2
:10D1A8001BF0080F3AD08A4B834D5F681E89B3F98C
:10D1B8000A8093F90C90D5F8E42003920023079392
:10D1C80084F83834A4F81A3484F81D34C4F82034A8
:10D1D800A4F8243484F82634C4F8283484F818349D
:10D1E800C4F82C3484F83034744B94F88024DB6A07
:10D1F80084F87F24A4F87C8484F87E949847724845
:10D2080006F020FE3146384601F0DFFC8246002851
:10D2180000F0E680A4F8728484F874941BF0040F7C
:10D228001AD0654B93F81831022B02D0634BDB6A96
:10D2380098470220FEF72CFF84F8350401F06EFEB3
:10D2480094F8103413B1012384F80F3494F881341E
:10D2580043F0100384F881341BF0020F03D0062139
:10D268000520FEF78BFF1BF0010F03D004210320DC
:10D27800FEF784FF01F0C6FC94F88124D0065FD540
:10D28800002384F88234D4F84033190644BF23F0CD
:10D298008203C4F8403312F0050F00F0C5820C2059
:10D2A80001F056FE002800F0BF8294F88134DF07B1
:10D2B80000F1BA825E0740F1CB82D4F8403323F004
:10D2C8000203C4F84033D4F8402382BB94F8815455
:10D2D80015F001011EBF2B4662F3000384F8813468
:10D2E80094F881345E0744BF6FF3820384F8813475
:10D2F800012384F8823421B1D4F8443335481B68BB
:10D3080098476D070BD5344801F02EFE01F05CFEFE
:10D3180028B194F8813443F0040384F8813401F08F
:10D3280060FC94F881346FF3041384F8813401238A
:10D3380084F8823494F8813443F0200384F88134EB
:10D3480094F8813418070AD56FF3C303234984F886
:10D358008134D4F84433A1F12000DB68984794F86D
:10D36800813499070AD56FF341031C4984F8813445
:10D37800D4F84433A1F164005B68984794F880348A
:10D38800022B01D1FFF746F994F881349A0640F14F
:10D39800EC826FF3451384F88134D4F84033002BC2
:10D3A80040F0E38225B0BDE8F04FFFF7D3BA00BFE5
:10D3B800D41F0020D81F002064180020205701081F
:10D3C800F02400205823002070230020CC230020C4
:10D3D800E02400200C2400202024002054240020D5
:10D3E80095F81831012B0CD101F0F3FB804668B198
:10D3F800504601F0E3FB504601F0E5FB042384F8B6
:10D408007F347EB9012384F819344AE101F0E3FB43
:10D418000028F6D0404601F0D2FB404601F0D4FB8C
:10D428000523ECE73B7802935B09013B062B00F2EE
:10D43800ED81DFE813F00700EB019200EB018F00AC
:10D44800EB01DB01102EDDD995F82C310E97F6B2E1
:10D458008DF83C60002BD5D118A804F0F9F80EAA75
:10D4680018A9FF2002F04CF89DF84830C3F30303D5
:10D4780007468DF8203095F8480095F87D308DF8EE
:10D488002130072208A902F03EFA002F5AD10028BD
:10D4980058D09DF843309DF842201199C5F8E41002
:10D4A8001B0443EA02239DF8412002201343C5F8D8
:10D4B800E03004F0DBF89DF8483095F8480085F82E
:10D4C8002A71C3F30212C3F3030385F8703085F899
:10D4D80078309DF8493085F86920012B38BF012341
:10D4E8004FF47A725343AB651344EB654FF0010870
:10D4F8000DF14A03113E0CA90C9385F868808DF84C
:10D50800346002F008FA0223404685F82C3101F015
:10D518001FFD18B14146384601F0DEFC94F810347E
:10D52800002B00F0798194F8383413B10020FEF70D
:10D53800E9FD94F8813443F0100384F88134FEF750
:10D54800A7FD6BE6012001F003FD0028E6D00121CC
:10D558000720E1E7012384F8183495F87D308DF829
:10D56800223094F81C348DF8213095F88C3095F8D9
:10D5780048000D3308A98DF8203002F0B1F9A6F162
:10D588000D031BB2069023EAE37300B283423FF710
:10D5980039AF0B2E7FF636AFA24B219318A8FF2385
:10D5A80018978DF864608DF8883002F075F8804619
:10D5B80000287FF427AF9DF86C301A99C4F82C1412
:10D5C80013F00F0203D09DF8800000286CD19DF85D
:10D5D800880000286AD0002A7FF414AF9DF88020C4
:10D5E800002A0CBF0227032700220792D5F8EC2057
:10D5F80091425DD195F8E910002959D0D5F80C1160
:10D6080095F8EAA00968079195F81811022902D13E
:10D61800032184F87F14032F7FF4F4AE13F0600F16
:10D628007FF4F0AE03924FF00108152395F84800F7
:10D638008DF8203008A902F053F995F82A310690A0
:10D64800BAF1000F37D0BAF1010F3ED1012B34D116
:10D658006FF009063E4106F00106C6F10206F6B271
:10D6680081B2BDF86E2007AB304601F0CFFD70B334
:10D67800072824D1082384F8193495F82A315BB98E
:10D68800029B03F0E003A02B06D16A6B239B9A420E
:10D6980002D1012385F83A30079BC4F82834C4F82E
:10D6A8006034FEF74FFDB9E547469DE701279BE744
:10D6B8004FF0010AB9E70426D2E70326D0E7082885
:10D6C80003D10A2384F81934E6E70123FAE718ABF3
:10D6D80000930399079B3246504601F063FE20B140
:10D6E80002280CBF0B230C238DE6079BC4F82834B3
:10D6F800C4F860349DF86C3084F81904C3F34013FF
:10D7080084F8263484F8383494F87F3484F81A84FA
:10D71800012B98BFA862B8F1010FC4F8200484F85F
:10D72800240484F8350433D1022284F8182495F8A7
:10D738003A20002A3BD19DF86C20D20637D4012B21
:10D7480094F834149DF86C2005D8012901D1960667
:10D7580001D501F001FB022F37D0032F09D09DF826
:10D768006C10012F4A4601F00F011CA831D0FFF7B9
:10D778006BF99DF8803084F81B34219BC4F8203461
:10D788009DF8883084F82434012384F8253426E071
:10D79800029A02F0E002A02A11D195F82A1101227A
:10D7A80085F83A2009B92399696384F8182495F80B
:10D7B8001821002AC3D1012284F81D24BFE70022C2
:10D7C80085F83A2084F81824B5E79DF88810219840
:10D7D8004A46FFF739F99DF8803084F81B3494F8ED
:10D7E800813443F0020384F8813497E6DFF834800B
:10D7F800013EB2B2791C404604F000F80323A4F8B5
:10D808001834C4F8208484F82464E8E7012384F8F1
:10D818001934FEF797FC81E695F81831022B7FF44E
:10D8280088AE83E61022002094F881345D070FD576
:10D83800012001F08DFB88B3012001F05FFB08B9DE
:10D8480084F80C04D4F8403323F00203C4F84033BE
:10D8580094F88114C8077FF536AD94F834340BB1C9
:10D86800032B26D1424B94F80C0493F8682090427D
:10D8780008D28A0750D593F818311BB194F87F3431
:10D88800002B49D13B4806F0DDFAD4F8403323F0A9
:10D898002003C4F84033FFF79BFB14E5062001F092
:10D8A80057FB0028CED1072001F052FB0028C9D130
:10D8B800CEE7012B30D194F80F24002A3FF403ADB2
:10D8C80094F80E3494F80D04834204D211F0020245
:10D8D80018BF94F83824264D95F82A11002941D10B
:10D8E80032BB834218D20133DBB2DF0784F80E342F
:10D8F80012D522238DF8603095F87C308DF862308F
:10D9080095F8480095F839308DF8613018A901F07C
:10D91800E7FF0E9085F8390094F8813400206FF302
:10D92800041384F8813484F80F04FFF773FBCAE406
:10D9380094F838648EB902238DF8683005F50873B9
:10D94800189395F8480005F52D7318A9199301F057
:10D95800D5FF84F8106484F8386494F80E3484F899
:10D9680039348FE7002AD7D08CE725B0BDE8F08F8F
:10D9780064180020402300202DE9F04F8A468BB020
:10D9880091460746002800F08D81002900F08A8121
:10D998000368002B00F086814368002B00F0828129
:10D9A8008368002B00F07E81C368002B00F07A8129
:10D9B800104601F091FF002800F07681BC4CBD4D67
:10D9C800384601F03FFA4FF4EE620021204603F09A
:10D9D80029FF4FF4A1620021284603F023FFB64B2C
:10D9E800C4F8283100264FF001080F2305A948463E
:10D9F8008DF8143084F8489084F8186184F88C60A5
:10DA080085F80E8485F80D8401F06AFF801B18BF25
:10DA180001204FF00A0B84F81C0105A994F848006E
:10DA28008DF814B001F05CFF4FF0060984F8DC00B3
:10DA380005A994F848008DF8149001F051FF1023BF
:10DA480084F8DD0005A994F848008DF8143001F039
:10DA580047FF1123C4F89C0005A994F848008DF8E5
:10DA6800143001F03DFF1223C4F8A00005A994F872
:10DA780048008DF8143001F033FF1323C4F8A400D4
:10DA880005A994F848008DF8143001F029FF1423F3
:10DA98000DEB0301C4F8A80094F848008DF8143081
:10DAA80001F01EFF1723C4F8AC0005A994F848003C
:10DAB8008DF8143001F014FF182384F8B10005A97B
:10DAC80094F848008DF8143001F00AFF1923C4F8BF
:10DAD800B400C4F8BC0005A994F848008DF81430C7
:10DAE80001F0FEFEC0B21E2384F8B80084F8C0001E
:10DAF80005A994F848008DF8143001F0F1FE1F23B1
:10DB080084F8C40005A994F848008DF8143001F091
:10DB1800E7FE202384F8C50005A994F848008DF88D
:10DB2800143001F0DDFE2123C4F8C80005A994F8DB
:10DB380048008DF8143001F0D3FE0B23C4F8CC0054
:10DB480005A994F848008DF8143001F0C9FE0C239B
:10DB5800A4F8D00005A994F848008DF8143001F015
:10DB6800BFFED4F89C306365D4F8A030A365D4F820
:10DB7800A430E365D4F8A8302366D4F8AC306366E3
:10DB880004F5087307A90490A4F8D200079394F841
:10DB980048008DF8246004F52D73089384F8B0804C
:10DBA800C4F894B084F89890C4F84CB084F85090B5
:10DBB80084F8688001F0A2FEC5F848A3FEF7C8FD06
:10DBC80032463E4B00964FF0FF3105F55A70C4E9D6
:10DBD8000B66C5F8447385F8816484F81981C5F823
:10DBE800408306F0D1F83246354B00964FF0FF31AE
:10DBF80005F5607006F0C8F83246324B00964FF0D3
:10DC0800FF3105F5667006F0BFF832462E4B0096D8
:10DC18004FF0FF3102AE05F57D7006F0B5F83046DD
:10DC280006F046F896E8030004F5907383E80300CD
:10DC3800264BC5F84C33264BC5F85433254BC5F84D
:10DC48005C33254F254BC5F85033254BC5F8583361
:10DC580005F553703B68984704F5A47003F016FB6C
:10DC680020B1112630460BB0BDE8F08F204601F0F8
:10DC78009DFA0028F5D100F0C7FFB8B9194801F09E
:10DC8800F7FA06460028ECD17B69984703F094FD23
:10DC9800BB6D94F819019847FB6A9847012385F8EA
:10DCA8008234DFE70326DDE70926DBE71326D9E719
:10DCB80064180020D81F0020000300011DD00008B0
:10DCC800D5C8000815C900080DC10008E5C200083C
:10DCD8009DC20008C9C000082057010875C2000885
:10DCE8004DC200084C19002008B5034B0020C3F8AA
:10DCF8004003FEF7CDF908BDD81F002010B5FFF787
:10DD0800B3F90A4C60B90A4B93F81831022B02D1C7
:10DD1800084BDB6A98470123C4F84033002010BD44
:10DD2800D4F84003013818BF0120F8E7D81F0020B5
:10DD3800641800202057010838B5134C04F55A70B0
:10DD480006F080F804F5607006F07CF804F566705B
:10DD580006F078F804F57D7006F074F800F040FFDE
:10DD68000A4B0025DB6A9847C4F84053FEF7F2FDDA
:10DD7800074908484FF4EE6203F040FD0123C4F858
:10DD88004033284638BD00BFD81F0020205701085F
:10DD980064180020F410002030B52A4B89B00546DD
:10DDA80093F8DD008DF8020093F8DC009A6A8DF88C
:10DDB80003000020019202900C4600293ED00592F3
:10DDC800D3F8882006921A8FD3F82811039152BAF3
:10DDD80093F81A11ADF81C2093F87C2093F848307A
:10DDE8008DF810008DF811108DF81E208DF81F3059
:10DDF8000DF1030201AB0DF1020103A800F06EFE64
:10DE08009DF90200FEF766F9607002A800F0B6FFFF
:10DE1800B0B9029A0F2A0DD863789A420AD81544E5
:10DE2800AB42A3EB02012CBF002001202170C000EF
:10DE380009B030BD002323700820F9E70320F7E775
:10DE48001320F5E7641800201FB50446002800F0E9
:10DE5800FD8000783F2800F2F380DFE810F04000F2
:10DE680046004B005000540058005D00F100F100DE
:10DE7800F100F100F100F100F100F1006400680028
:10DE88006C0077007E0081008400890087008B0089
:10DE98008F009200950098009B009E00A200AA00A7
:10DEA800A600AE00B100B500BE00BA00BC00F1008B
:10DEB800C200F100F100F100F100F100F100F10001
:10DEC800F100F100F100F100F100F100F100F100C2
:10DED800CA00CE00D300D700DB00DF00E8005D4BAE
:10DEE80093F81831237104B010BD5A4B93F82C31B4
:10DEF800237102E0606803F065FB0020F3E76068C7
:10DF080003F0A6FBF9E7534B93F81A31F0E7514BAE
:10DF1800D3F8E0306360F0E74E4B211D93F82C01F5
:10DF280003F0AEFBE9E74B4B93F81931E0E7494BB7
:10DF380093F88C30DCE71D238DF80830454B02A997
:10DF480093F8480001F0CCFC6060D6E7424B0434FB
:10DF580093E8030084E80300CFE7404B0434F7E775
:10DF68003F4B0434F4E73F4B0434F1E71B23E3E76A
:10DF78001A23E1E7374B93F86830B9E7354B5B6D07
:10DF8800C8E7344B9B6DC5E7324BDB6DC2E7314BBD
:10DF98001B6EBFE72F4B5B6EBCE72E4B93F8DD3053
:10DFA800A6E72C4B93F83930A2E72A4B93F8DC30DC
:10DFB8009EE7284B93F838309AE7264BDB6CA9E7A5
:10DFC800244B93F8503093E7224BD3F884306360A6
:10DFD80093E7204B9EE7244B9CE71E4BD3F8CC30AD
:10DFE800F5E71C4BD3F82831636001F00DFDA06004
:10DFF80083E7184BD3F890308CE7164BB3F888308A
:10E00800A3807AE7134BB3F88A30F9E7114BB3F8DA
:10E01800D030F5E70F4BB3F8D230F1E70D4B93F85A
:10E0280048200AB1062A13D1B3F84C37E8E7094B60
:10E0380093F848200AB1062A0AD1D3F8503769E77D
:10E04800204604B0BDE8104000F0CEBD03204AE7EA
:10E05800182048E764180020D0180020181900205C
:10E06800D818002020190020F410002073B50446A9
:10E0780000285ED0A04DD5F840339A0700F15F82A2
:10E0880002783F2A00F25682DFE812F0400046008C
:10E098004E0056005A005F00640070007A007F004E
:10E0A800840089008E00930098009D00A700540208
:10E0B800AC00CC00DF000601280119012C013C014D
:10E0C8004001440148014C01500162018A01780174
:10E0D8009C01A201A901AE01B30154021802540225
:10E0E8005402540254025402540254025402540278
:10E0F8005402540254025402540254025402270295
:10E108002C02310236023B0240024A02007902B078
:10E11800BDE87040FEF7AEBA0379022B09D0774A02
:10E1280082F82C31002005E0406803F03DFA002811
:10E13800F8D0032002B070BD406803F079FAF6E722
:10E148006E4B027983F81A21ECE76C4B4268C3F8EE
:10E15800E020E7E7694D416895F82C0103F086FA5D
:10E168000028E6D16368C5F8E430E3E74168002990
:10E17800DFD0002001F0A8F90028D3D01120D9E77A
:10E1880041680029D5D00120F4E741680029D0D0A2
:10E198000820EFE741680029CBD00920EAE7416869
:10E1A8000029C6D00C20E5E741680029C1D00D2020
:10E1B800E0E741680029BCD00E20DBE74168002970
:10E1C800B7D00F20D6E74E4C4C4B007983F8190195
:10E1D800A36D9847E36A9847A4E7484B027983F808
:10E1E8008C209FE7454D037A8DF8003095F848005C
:10E1F80095F87D308DF801300722694601F083FBE0
:10E20800002896D0636895F8480000930022694674
:10E2180001F079FB00288CD06C35D4E9010185E840
:10E2280003007FE7354D037A8DF8003095F84800F4
:10E2380095F87D308DF801300722694601F063FBBF
:10E2480000283FF476AFB435E7E72C4D037A8DF814
:10E25800003095F8480095F87D308DF80130072298
:10E26800694601F050FB00283FF463AFD4E901018F
:10E2780005F1740383E8030095F81831022B7FF445
:10E2880051AF95F82C31002B3FF44CAF1C4BDB6A97
:10E298009847FEF7BFF945E7184D037A8DF8003027
:10E2A80095F8480095F87D308DF8013007226946C9
:10E2B80001F029FB00283FF43CAFBC35ADE74368CB
:10E2C800009301238DF804300C4B694693F84800FD
:10E2D80001F026FB00287FF425AF2AE74368009366
:10E2E8000023EFE703795A1E0E2A3FF622AF034AAE
:10E2F80082F8683016E700BFD81F00206418002095
:10E3080020570108904B42685A650BE78E4B4268CC
:10E318009A6507E78C4B4268DA6503E78A4B4268DF
:10E328001A66FFE6884B42685A66FBE6864C037914
:10E3380094F848008DF800300622694601F0E3FAA7
:10E3480000283FF4F6AE9DF8003084F8DD30E9E6A9
:10E358007D4C03798DF8003094F8480094F87C30AF
:10E368008DF802300522694601F0CDFA00283FF405
:10E37800E0AE9DF8003084F83930D3E6724C03796A
:10E3880094F848008DF800300A22694601F0BBFA7B
:10E3980000283FF4CEAE9DF8003084F8DC30C1E6AA
:10E3A800694C037994F848008DF8003009226946D1
:10E3B80001F0A9FA00283FF4BCAE9DF8003084F8BB
:10E3C8003830AFE6604B4268C3F89420DA64A9E6B7
:10E3D8005D4B027983F8982083F85020A2E65A4BC7
:10E3E8004268C3F884209DE6574B4268C3F8CC20A6
:10E3F80098E6012B40F0A380544C2421204603F0DA
:10E4080013FA636A984201D0172093E61C2104F19D
:10E41800280003F009FA636C9842F5D1FC2104F155
:10E42800480003F001FAD4F844319842ECD1D421E1
:10E4380004F5A47003F0F8F9D4F81C329842E3D13B
:10E44800902104F5087003F0EFF9D4F8B03298423F
:10E45800DAD14FF4946104F52D7003F0E5F9D4F89E
:10E4680054379842D0D1142104F5EB6003F0DCF95D
:10E47800D4F86C379842C7D1334E214630464FF412
:10E48800EE6203F0BBF920464FF4EE62002103F080
:10E49800C9F995F8113485F8E033736FC5F8E4339A
:10E4A80096F87D3085F8F03340F20123A5F8F23371
:10E4B800274B96F819019B6D984733E68379012B12
:10E4C8003FF637AE204B42684068C3F8282100F079
:10E4D80089FE00283FF42EAE50E61B4B4268C3F875
:10E4E80090201FE6184B8288A3F888201AE6164B5E
:10E4F8008288A3F88A2015E6134B8288A3F8D020D7
:10E5080010E6114B8288A3F8D2200BE60E4B93F845
:10E5180048200AB1062A14D1A288A3F84C2701E69C
:10E52800094B93F848200AB1062A0AD16268C3F851
:10E538005027F7E502B0BDE8704000F057BB012056
:10E54800F8E51820F6E500BF64180020F410002054
:10E55800205701082DE9F04186B00023ADF80030BE
:10E568000646002800F0E280FEF77EFD20B1012477
:10E57800204606B0BDE8F08100F02CFD0028F6D159
:10E5880000F022FD014618B96948142203F04AF93F
:10E59800684D95F88134012243F0040385F8492435
:10E5A80085F8813433788DF804300021013B8DF8EB
:10E5B80005208DF807100D2B00F2B080DFE803F07E
:10E5C80007AEAEAE525A7DAEAE85AEA28F9ED5F8DE
:10E5D800404314F02004CAD1DFF85C81574FFEF79E
:10E5E800B7F8224696F9051098F8480001F0E5F9C1
:10E5F80088F83900B37988F83830204607238DF831
:10E608000530FEF737F8FF2307F58670A5F80C31BB
:10E6180085F80441C5F8087103F01AF807F58A70FF
:10E6280002F0D0FF2046FDF77FFE044640B196F980
:10E63800051098F84800012201F0BFF988F8390060
:10E64800D5F884343361002C6CD000F0BDFC002870
:10E658008ED195F8813485F8100460F3820385F82B
:10E66800813485E700226946022000F0DBFA10B306
:10E678001324E5E795F811348DF808302E4BB2884D
:10E6880093F839108DF8091093F838108DF80A109E
:10E69800D3F880100391D3F88410049193F84800BC
:10E6A800ADF8142002A901F09DF9D5F8403343F0E4
:10E6B8000203C5F840330024C2E7214BB28896F91B
:10E6C8000C10B068DB6B9847EFE702A90D2000F04B
:10E6D80027FB0028EFD0002269460D20C5E7164B1E
:10E6E80093F81831D3B9347904F0070000F077FAB9
:10E6F8008DF80040012269461020B6E700226946DD
:10E708001220B2E78DF8072000F05AFA044638B90B
:10E7180000F053FA204600F055FA91E702248FE7FB
:10E7280001248DE701A800F0A1FB21E703241FE7DE
:10E7380020240020D81F002064180020DA1F0020A1
:10E74800205701082DE9F04F91B0002603910546A6
:10E7580018B9032011B0BDE8F08FFEF785FC82469A
:10E76800002840F06481B84C14220146074604F2A0
:10E77800344003F057F8012384F8353484F80E3414
:10E788002A789A4200F0B080032A00F0BF80002A5D
:10E7980040F0C98084F80D34022295F80490D5F829
:10E7A8000880AE8995F90EB062F347179A46A74BD1
:10E7B800022493F87C2093F848008DF8244009A996
:10E7C8008DF8262001F08CF8BAF1000F00F02D81A9
:10E7D8009E4B93F81A21B2B940B25845B8BF584673
:10E7E80093F87C208DF814008DF8162093F84800D3
:10E7F800052205A901F087F80028AAD0934B9DF8B7
:10E80800142083F83920198F1A8F93F82C0102915C
:10E81800996A069152BA002800F0058193F81B0105
:10E8280000B9186393F81801ADF83C20013893F843
:10E838007C208DF83E20D0F1000B93F848208DF80D
:10E848003F204BEB000B824A93F83A0093F81A41A9
:10E8580001900D914FF00100D3F88810D3F82831BA
:10E868008DF830000E910B93511C06AB0BA88DF858
:10E87800314000F033F9019B4FEA0B1B4BEA431B75
:10E888004FF0000A4BEA801B4BEAC413D0456E4C8C
:10E89800019308BF56463246414604F59C709B4694
:10E8A800CDE907AAA4F800A084F810A402F0A6FFF6
:10E8B800F9B2A770C7F34217F2B2042F634E019B57
:10E8C80084F8372233D0072F00F09D80022F32D0F2
:10E8D8000220029B33875C4B002283F810245A4B9A
:10E8E800D3F884342B6135E7EB7B082B28BF08234A
:10E8F80084F80D34042395F80490D5F80880AE897F
:10E9080095F90EB063F34717924650E784F80D3433
:10E91800D5F804802E8995F90AB067F01F079A4642
:10E928004FF0000943E7D346D046D1463FE74FF0C2
:10E93800010084F81004474F84F80D11042084F86E
:10E948000401FF20D6F8E41084F80C0184F814318F
:10E9580007A807F59B73C4F8087184F82891C4F8D0
:10E96800101184F83021C4F82C3100F043FC002841
:10E9780057D1079BA4F8380408A8A4F81631C4F89E
:10E98800403400F0FBF960BB089BABB196F9390045
:10E99800FDF7A0FB94F837322BB3089B0F2B19D83F
:10E9A80007F58B7208A90F2000F0F4F9C8B9089B85
:10E9B80063F3030B84F814B10398FDF7B5FC002842
:10E9C80087D1069B86F83A00B36200F0B7F980B3A6
:10E9D800132080E707F2864208A900F0DBF9002837
:10E9E800EAD0132075E707F286473A4608A900F0EF
:10E9F800D1F90028F5D1089B84F82801C4F82C71B6
:10EA080084F83031D8E7B8F1000FD5D0002AD3D038
:10EA18004146E01C02F0F2FE94F8373201332380BD
:10EA2800CAE7122055E7072055E7204657E7012097
:10EA380090E62B7884F8343494F8813443F0010359
:10EA480084F881344BE700BFD81F002064180020E9
:10EA58009C180020DA1F002037B50B4D8DF80400F4
:10EA680004460F2295F8480001A900F04CFF40B178
:10EA7800064A85F81C4192F8813443F0200382F855
:10EA8800813403B030BD00BF64180020D81F0020B7
:10EA980010B5FFF733F90446A0B90B4805F0D2F9D1
:10EAA8000A4805F0CFF90A4805F0CCF9094805F0FD
:10EAB800C9F900F095F8FDF74BFE074BDB6A98475C
:10EAC800204610BD0124FBE74023002058230020E6
:10EAD80070230020CC230020205701082DE9F04F97
:10EAE80090F802908BB004468A460192B9F1000F63
:10EAF80060D14579816890F9102090F911801960EA
:10EB0800002D55D0817C8DF81610C07C4FF0020B7B
:10EB180005A9CDE902238DF814B000F0E1FE029AB0
:10EB280047B2BA421646B8BF3E46BA420CDC039B0F
:10EB3800C3F800904D46019B8AF8006083F8008076
:10EB480028460BB0BDE8F08FA268A189E3898A4204
:10EB58000B4434BF002501259A42ECD3082305A9AC
:10EB6800E07C8DF8143000F0BBFEE289A368B3FBAB
:10EB7800F2F102FB1133012B4FFA80F8DBD122238B
:10EB88008DF81430E07CA37C8DF8156005A98DF80C
:10EB9800163000F0A5FE46B2B742CCD12579002D3B
:10EBA800C9D0E07C8DF824B007A900F0A7FEC1E722
:10EBB8001646C0E70025C3E770477047704770479F
:10EBC800002070477047704770470020704700204A
:10EBD800704700207047002070470020704770473A
:10EBE8007047704702207047022070470220704724
:10EBF800704700207047704770470020704700201A
:10EC0800704770477047000010B5054CFC2220463D
:10EC1800002102F007FE0020C4E9000010BD00BF7B
:10EC2800F42400202DE9F04180461546002942D001
:10EC3800244B002403F1010C1A462001103312F86A
:10EC4800016F002E39D19A42F9D11F4F3B680BB999
:10EC5800C7F800C07B680BB1C3F800C03B1800229E
:10EC680001349A6083F80C800D302301AAB238442D
:10EC7800FD50C7F804C002F0C1FDB8F1050F17D068
:10EC8800A8F10808B8F1020F8CBF4FF000084FF048
:10EC9800010807EB041400236371D7F8F83084F8EF
:10ECA800048001332B44C7F8F8303046BDE8F081C2
:10ECB8004FF00108EDE70126F7E701340F2CB9D131
:10ECC8000226F2E7FB240020F424002010B510B33C
:10ECD800124A1368984204D103681360002304E0C1
:10ECE8000B4613B119688842FAD15168884208BFA7
:10ECF80053600BB101681960D2F8F8308168013BA4
:10ED080000245B1A04602146C2F8F830102202F091
:10ED180089FD204610BD0120FCE700BFF424002037
:10ED2800054B1B6813B11A798242FAD1002B0B608C
:10ED38000CBF032000207047F424002010B5054BB9
:10ED4800186800B910BD037B04680BB9FFF7BEFF54
:10ED58002046F6E7F424002010B5074B186800B9E0
:10ED680010BD03790468052B02D0083B022B01D89B
:10ED7800FFF7ACFF2046F2E7F424002028B1044B4B
:10ED8800D3F8F8300360002070470120704700BFB7
:10ED9800F42400202DE9F04107460E4615463AB303
:10EDA80031B3144B1C6800232CB93046FFF7E6FF3B
:10EDB8000020BDE8F081A268F91A0132914210D30F
:10EDC8002279EA54581C22895FFA80F8611D55FAA5
:10EDD80080F002F013FDA368246898445FFA88F372
:10EDE800E2E720462468FFF771FF002CF9D1DCE741
:10EDF8000120DEE7F42400200238C0B211289ABFAF
:10EE0800014B185C00207047AB50010830B50B4B24
:10EE180093F820200446084672B100211C33057877
:10EE2800A54208D001319842CDB20CBF0448043045
:10EE3800AA42F4D8002030BD1046FCE7F025002097
:10EE4800FC25002010B5084C00232060142204F192
:10EE58000C00FF2184F82030C4E9010002F0E2FC34
:10EE6800012384F8213010BDF025002010B50E4A8A
:10EE780092F82010042915D8936804781C704478F7
:10EE88005C70C078D87001310020987082F820102A
:10EE980002F11C018B4214BF043302F10C0393608E
:10EEA800012010BD0020FCE7F0250020094B93F855
:10EEB800200068B15A6803F11C018A4200F1FF3052
:10EEC80014BF043203F10C0283F820005A600120B9
:10EED800704700BFF025002010B5074B93F820209D
:10EEE8000446084632B15968FFF790FF10B1012374
:10EEF8004470837010BD00BFF025002008B5064B94
:10EF080093F820202AB15968FFF780FF08B14078AC
:10EF180008BD0120FCE700BFF025002030B50A4AF3
:10EF280092F82010536882F8210061B19168012499
:10EF38001C32DD78587005B99C7093420CBF034BA6
:10EF480004339942F5D130BDF0250020FC2500207E
:10EF580008B5044B5968FFF759FF003818BF01205E
:10EF680008BD00BFF02500202DE9F3410422154E0D
:10EF7800044600210DEB020096F8208002F052FCB6
:10EF88000025EBB2984502D802B0BDE8F08173685D
:10EF9800197821705A7862709F785FB1336820467B
:10EFA8009B689847FFF782FF17B901A8FFF75EFF34
:10EFB8000135E6E7DB788DF804108DF805208DF82B
:10EFC8000730EFE7F0250020014B93F82000704749
:10EFD800F0250020034B93F82000042894BF00205C
:10EFE80001207047F02500201FB50024CDE9024418
:10EFF800C41F8DF800408DF801100C0AADF80420EC
:10F00800090C120C8DF803108DF806208DF80730C6
:10F0180002461B0A012168468DF802408DF8083027
:10F0280002F05DFA002818BF0F2004B010BD2DE9CA
:10F03800F04188B017460D460F9A064600284DD075
:10F0480000240121CDE904448DF810109DF83810F2
:10F058008DF81510ADF81630190CCDE900441B0ECB
:10F06800CDE902448DF81930ADF81A20130C120EB0
:10F0780007948DF818108DF81C308DF81D20E3B218
:10F088004FEA0318002D5FFA88F803DC002008B067
:10F09800BDE8F081013310218DF81F303A466B46E8
:10F0A8000DEB010002F0B1F90346C8B9102DAC46CA
:10F0B800A8BF4FF0100CDAB2624503F1010303DB7D
:10F0C800103D2DB20134DAE708EB020020326A4421
:10F0D800315C12F8202C4A403254ECE70A20D6E77B
:10F0E8000F20D4E70138032815D8DFE800F002081C
:10F0F8000C100A4B1B681B690B6000207047074BFC
:10F108001B685B69F8E7054B1B689B69F4E7034BD1
:10F118001B68DB69F0E70520704700BF1426002054
:10F128002DE9F041C4B00C464A9E17461D4680465C
:10F13800B8B3B1F5807F36D84FF48872002168469D
:10F1480002F070FB492300934FF48073ADF804304C
:10F158002B0C8DF80830330CADF80650ADF80A606A
:10F168008DF80C3022460023414604A82D0E360E99
:10F178008DF80E308DF809508DF80D608DF80F4020
:10F1880002F03CFB04F110014B9A3B4689B26846F9
:10F1980002F025F910B1012818BF0F2044B0BDE8CE
:10F1A800F0810A20FAE70E20F8E7000010B590B1C8
:10F1B8000A4C28220021206002F034FB2368084A08
:10F1C8001A6000204FF0FF32C3E90302C3E90522A9
:10F1D800C3E9072210BD0920FCE700BF1426002060
:10F1E80000010101024B1B6818600020704700BF36
:10F1F8001426002030B1044B1B68DB680133036020
:10F20800002070470A2070471426002073B50E4668
:10F21800002101911D4633B301A9FFF763FFD0B95F
:10F22800019C631C04D0A3B2D31A002B10DDE21892
:10F238000E4B2A601B689B786BB9121B63EB0303A8
:10F24800B24273F10003ACBF01200020C00002E00D
:10F2580003D12C60072002B070BD230C1B0403F5FA
:10F2680080331A44E4E70A20F5E700BF142600209B
:10F2780028B1044B1B681C334362002070470A20E6
:10F28800704700BF142600201FB50446F0B10023C4
:10F2980003A8039302F07AF90E4ABDF80C301268FD
:10F2A80020469380E38200F052FA60B904F1180313
:10F2B800009321680123132202F088F840B9204600
:10F2C80000F045FA00B1112004B010BD0A20FBE798
:10F2D8000F20F9E714260020F0B5054687B01C4634
:10F2E8003BB32F4E3368DB68834257D894F820200D
:10F2F800002A14BF09220822834205D3204600F0C1
:10F308005AFA70B111200AE0002301900093A36813
:10F3180094F82810606AFFF78AFE0028EED007B03C
:10F32800F0BD23792168B4F808C0A768043B9AB2F5
:10F3380009B90A20F3E7B2F5807F2DD8ADF80EC0E1
:10F348008DF817304FEA174C04F12C033F0E8DF857
:10F35800117000932F0C08234FF0490EADF80C00E4
:10F368008DF814708DF816002F0E0DEB0300CDF8F4
:10F3780008E08DF810C0ADF812508DF8157002F045
:10F3880025F808B10F20CAE7204600F014FA002833
:10F39800B8D13368DD60C2E70E20C0E70620BEE7BB
:10F3A800142600202DE9FF410A9D80460F46164687
:10F3B8001C46002D5AD0002303A910460393FFF7DB
:10F3C80091FE18B1062004B0BDE8F081039B9C4271
:10F3D80001D80133F6D1284600F05EF9002847D15C
:10F3E800264B1A78424503D01A79424542D101206A
:10F3F800AA68BA4240D103EB8002EB6A92F8018016
:10F408002979CDE900430439927828683B4689B2C6
:10F41800FFF786FE0028D6D195F820300194002BFE
:10F428004FF00103009314BF4246082295F82810B4
:10F43800686A3B46FFF7FBFD0028C4D1013E032E56
:10F44800C1D8DFE806F002070B0F0D4B1B681C61E3
:10F458001C62B8E70A4B1B685C61F9E7084B1B683C
:10F468009C61F5E7064B1B68DC61ACE70A20AAE75C
:10F478001020A8E70C20A6E70220A4E7B408002083
:10F48800142600201FB50A460B2A4FF00001CDE9CB
:10F498000011CDE9021107D00C2A13D00A2A0FD087
:10F4A8000B2005B05DF804FB012802D120238DF85C
:10F4B8000030684602F013F8002818BF0F20F0E764
:10F4C8003023F4E70B21F4E738B5054602F002F8DB
:10F4D800044678B97DB9094B1B680B219878FFF76A
:10F4E800D1FF38B90C21FFF7CDFF18B90A21FFF772
:10F4F800C9FF00B10F24204638BD00BF14260020E4
:10F508002DE9F04380468FB00C461746002A6BD091
:10F51800002969D0002529461D2206A8059504F072
:10F52800A3FE8DF81350344D2B680DF114099E88F5
:10F53800CDF804900DF1130302933B7900933B68D7
:10F5480032462146404601F0E6FF00284ED1386891
:10F558003A79494602F052F9384600F04FF8002847
:10F5680046D13C7AFA79BB79240444EA02241C4344
:10F578002B689A6894423DD99C609DF813000B2132
:10F58800FFF780FF034658BB0C21FFF77BFF0346BC
:10F5980030BB0A21FFF776FF034608BB7B7ABA7AAD
:10F5A800FF7A3F0447EA02271F433A46334621467B
:10F5B8000920FFF719FD034690B933463A4621461C
:10F5C8000820FFF711FD034650B92A689DF813106B
:10F5D80091700021D1604FF0FF31C2E904119161AF
:10F5E80018460FB0BDE8F0830A23F9E70F23F7E7C1
:10F5F8001023F5E70323F3E71426002010B504468B
:10F60800002845D00168002942D011F8013B437118
:10F618000322063002F0F2F82046032250F8091BB4
:10F62800043102F0EBF82168CB79E3600A7A43EA07
:10F638000223E3604A7A43EA0243E3608A7A43EAB0
:10F648000263E360CB7A23740B7B63742379212BE9
:10F658001AD110220D3104F1120002F0CFF81D2248
:10F668002168501C8B5C6362085C43EA0023901C91
:10F678006362085C033243EA004363628A5C43EADC
:10F6880002636362002010BD112B03DC0D22E7E743
:10F698000220F8E70120F6E710B50446002854D008
:10F6A8000168002951D00B7843714B7883608A78C0
:10F6B80043EA02238360CA7843EA024383600A79F3
:10F6C80043EA026383604B7903738B79C381CA79F8
:10F6D80043EA0223027BC38102F00F020831103093
:10F6E80002F08CF8237B002203F00F0384F820201B
:10F6F80084F82820227903F10800111A04290DDD65
:10F7080021680933043AD21A085C84F82000D2B27E
:10F71800606A84F82820194402F070F82379226876
:10F728001A44002012F8043CE36212F8031C43EA6E
:10F738000123E36212F8021C43EA0143E36212F870
:10F74800012C43EA0263E36210BD0220FCE710B516
:10F75800044660B3036853B30279162A29D942795B
:10F768001A700146082251F8060B013002F050F8D1
:10F778002146082251F80E0B093002F049F8236897
:10F78800E28A5A74E38A22681B0A93742368A2697E
:10F79800DA74A36922681B0A13752368628B5A7589
:10F7A8002368E27E9A7517232371002010BD01207B
:10F7B800FCE70220FAE738B50446002863D0016860
:10F7C800002960D0037B90F8282003F00F03002A5B
:10F7D80057D10833207904321344984255D36379BA
:10F7E8000B702368A2685A70A36822681B0A93707A
:10F7F80023686289DA702368E27A1A712368227BA7
:10F808005A712368E2899A71E38922681B0A2146A2
:10F81800D371227B51F8100B02F00F02083001F06F
:10F82800EDFF237B94F8282003F00F0303F108056C
:10F838002AB1226894F82010515503F1090520686F
:10F8480094F82820616A284401F0D8FF94F82830F9
:10F858002268E16A2B44D1545A1CE16A206892B2AA
:10F86800090A81549A1C2168E08D92B28854DA1CE6
:10F87800216894F82F0092B2043388542371002031
:10F8880038BD0933A6E70120FAE70220F8E70000AF
:10F89800024B1A8810431880704700BF18260020B2
:10F8A80008B5074B1B883BB1FEF728FA00280CBFA8
:10F8B80000206FF0020008BD6FF00100FBE700BFF9
:10F8C8001826002010B5034B00241C80FEF70CFA04
:10F8D800204610BD18260020B0FA80F04009704775
:10F8E80082B018B9084602B000F0D0B8002002B0C3
:10F8F800704710B9084600F083B9704710B9084638
:10F9080000F09AB970470346084611460BB900F053
:10F91800E7B90020704710B9084600F045BD7047A8
:10F9280010B9084600F008BA0020704710B4044621
:10F93800084611461A46019B14B910BC00F01ABAC1
:10F9480010BC70470346084611460BB900F044BA8C
:10F958000020704710B40446084611461A4614B9E8
:10F9680010BC00F0B1BA002010BC704730B4054696
:10F97800084611461A46DDE902341DB9029430BC26
:10F9880000F02EBB002030BC704710B9084600F0CC
:10F99800DFBB0020704710B9084600F043BD0020C7
:10F9A800704710B9084600F0EEBB0020704710B948
:10F9B800084600F0EBBB0020704703460846114696
:10F9C8000BB900F005BC0020704710B40446084687
:10F9D80011461A46019B14B910BC00F0FBBB092064
:10F9E80010BC704710B9084600F03CBD704710B411
:10F9F8000446084611461A4614B910BC00F05CBD0E
:10FA0800C8B210BC704700000048704703000101ED
:10FA1800064B10B51B6A0446984730B10448054B9D
:10FA2800204498428CBF0020012010BD20570108B7
:10FA3800403576C9405DC600F0B5114B85B00C461F
:10FA480010491F56054601F045F80F4BE4B25E6AAF
:10FA5800072D4FF00103CDE9024301460AD10522E3
:10FA68000023CDE900234FF47A727A431846B04751
:10FA780005B0F0BD08220020CDE900203A46F5E7A0
:10FA8800E7500108C0500108205701081FB500239E
:10FA980000930378013B382B00F28580DFE803F000
:10FAA8001D2383838320838383834042444B835372
:10FAB80056595C5F6265836D206F74797B7E7E80AA
:10FAC8008725838383838383838383838383838952
:10FAD8008B908383899083929600C378002B62D0A1
:10FAE800022300935FE08378F8E743788DF80430C9
:10FAF80007238DF805308378003B18BF01235B008E
:10FB08008DF8063010238DF80730334B1B6801A899
:10FB180003F59062CDE9022300F0BCFF009042E0BB
:10FB28004023DEE72023DCE7827890F9013042B9F0
:10FB38002A4AD35CD5E7827890F901300AB9284A75
:10FB4800F7E7284AF5E740F6B833CAE74FF47A737F
:10FB5800C7E74FF4FA63C4E741F28833C1E741F2DB
:10FB68007073BEE74FF48043BBE71F484FF47A71C8
:10FB780001F028FE00F5FA60D0E71C4BB1E7164B00
:10FB88001B6803F59063ACE7134B1B6803F28C43C7
:10FB9800A7E71023A5E7104B1B68A2E70123A0E7FE
:10FBA8004FF083430093009805B05DF804FB104BB9
:10FBB800F8E7104B95E740F21123ADF80030F2E773
:10FBC80003238EE790F901300B4AB2E70B4990F90D
:10FBD800010000F07FFFA1E720260020F750010870
:10FBE80007510108FF50010818FCFFFF00EA06371B
:10FBF8009A99094040F70937E7500108C0500108B1
:10FC080037B50B4B02781B680C2101FB02335B7A7A
:10FC180003EB4304074B1D6803690093C3684278EC
:10FC2800816805EBC40000F0D5FC03B030BD00BF0F
:10FC3800202600201C26002030B587B0027A6423D5
:10FC4800ADF80030012A4FF00003CDE90133CDE9CA
:10FC5800033301468DF802308DF8143027D0022A7C
:10FC68002ED012BB006800B34B68F3B1194A1A4C86
:10FC7800106069461822236001F0C0FD174B246804
:10FC880093E807000C3384E8070093E8070004F1C1
:10FC98000C05032385E80700A4F88C34012204F23C
:10FCA8008C4104F5906000F086FC07B030BD0A492D
:10FCB80008684360036100F28C4100F59060F2E748
:10FCC800054B1B68B3F88024B3F88C140A43A3F8D7
:10FCD8008024EAE71C260020202600202C44010866
:10FCE80008B503460A2924D8DFE801F006232323B0
:10FCF800230B161B23212100BDE808400068FFF7ED
:10FD080087BE90F900009978072271B900F013FCBA
:10FD1800003818BF012008BD052293F90000002112
:10FD2800F4E790F900005978EEE70221EEE70722A0
:10FD3800F3E70020EFE7000010B504791CB1012CAF
:10FD48000BD0002010BD0A4B01681B68012203F587
:10FD5800906000F030FC0120F4E7054B01681B6857
:10FD6800224603F28C4000F026FC2046EAE700BF5A
:10FD780020260020F7B50728144D1C46A8BF0720E9
:10FD880058700E462946174600F0A4FE94F9013033
:10FD9800A070072B13D1322000F09CFD0C4BDB6DBB
:10FDA8000546984704F10C02083403460192009472
:10FDB8003A463146284600F092FD03B0F0BD054AA8
:10FDC80055F82310D05C00F07DFDE7E7C05001082E
:10FDD80020570108E75001082DE9F04F344F90F9FA
:10FDE80001607B68D0F804908BB004468846984739
:10FDF8000546002859D1E37C73B92E4A2378126846
:10FE080003EB4303990002EB8303D3F80490B9F1A1
:10FE1800000F01D152F80190274B484613F906B05C
:10FE2800FB689847A37CD7F818A022890993072E66
:10FE380028D100230121CDE90223204A0693CDE9E8
:10FE48000431CDE907330521CDE900214FF47A7259
:10FE580002FB0BF24CF250311846D047637C13B3C7
:10FE6800174B995D7B6D0D31C9B228469847E07CE8
:10FE78003246494600F040FE88F8006001200BB089
:10FE8800BDE8F08F002101250823CDE90013CDE955
:10FE98000715CDE90511CDE903110292A1782B468A
:10FEA8005A462846D9E7074BDBE70020E7E700BFBB
:10FEB8002057010820260020E75001088545010049
:10FEC80007510108F75001082DE9F04F8DB090F95E
:10FED8000130DFF8F8A0DFF8F890CDE90A123D4AC2
:10FEE800017812F903B0DAF800203B4B0C2505FB2A
:10FEF80001221B68527A182101FB0233044693F948
:10FF0800021090F9020000F0E0FD3449064694F929
:10FF1800010000F0DFFDA26861688046304600F00D
:10FF280006FD2178DAF80020D9F80C306943074635
:10FF380050589847D9F81C309C4694F90130002550
:10FF4800072B4FF47A63CDE90753CDE905552DD139
:10FF58000123CDE903530523CDE901534FF47A7307
:10FF680003FB0BF300933946434646F2A812284692
:10FF78006746B8472378DAF800200C214B4394F9F8
:10FF88000110D05800F0DAFDA18994F90100FFF7BB
:10FF980053FD0B9B217B1860D9F8543028469847AD
:10FFA8000A9B01201E700DB0BDE8F08F01200823C8
:10FFB800CDE90350CDE901032A46CDF800B06546E6
:10FFC80043463946A84701200546D3E720260020A6
:10FFD80020570108E75001081C260020C0500108DE
:10FFE8002DE9F04F8FB0002405468A469146984681
:08FFF8000494ADF81440ADF8CB
:020000040801F1
:10000000024007264FF0010B2B7AA34206D96868FD
:1000100004A9204400F0F4FB00285DD102238DF8F0
:10002000083002A86B7A8DF80A30FFF733FDAB7AFF
:100030008DF81D309DF811308DF81E309DF812306E
:100040008DF81F309DF810308DF82030EB7A8DF848
:1000500021302B7B8DF822306B7B8DF823301023E1
:100060008DF81C608DF824303A4E8DF82C000DF17F
:1000700002030A93072332688DF82D30ADF834302F
:100080002B680C9206930DF1120204AB0DF11101D5
:1000900006A800F0CFFB072805460BD130680C22DC
:1000A000002100F5906001F0C1FB3368BDF802202B
:1000B000A3F880249DF811308AF800309DF81230A2
:1000C00089F800309DF8103088F80030189B2846D9
:1000D0001C700FB0BDE8F08F9DF81330BDF81470A0
:1000E000ADF802702044C4B2F3B917B3194A002026
:1000F0001168072602464FF00C0C062B1BD10CFB97
:1001000000FE51F80EE0BEF1000F04D00BFA00F231
:100110003A4397B2012201301028EED1002A3FF471
:1001200073AFADF802706FE75A1E042A01D9062B8F
:10013000DCD0062668E747FA00FE1EF0010FEAD081
:100140000CFB00FE51F80EE0BEF1000F08BF0626C2
:10015000E1E700BF2026002038B505464068FFF7DC
:100160005BFC0722841D002195F90000E4B200F039
:10017000E6F908B904F0FD0495F901000722002111
:1001800000F0DDF908B904F0FB04204638BD00207A
:100190007047000010B503780F2B044618D840684C
:1001A000FFF73AFC22780B4902EB42020968831CF4
:1001B00001EB820051F82220DBB21AB903F0FD03F3
:1001C00058B210BD032B06BF626842600223F7E7F6
:1001D0000020F6E720260020022070472DE9F0419C
:1001E0003A4D0446286896B00E46904600211F46B8
:1001F0000122032300F59060CDE90411CDE9061139
:100200008DF80C108DF80D10ADF80E3000F0B9F926
:1002100030B92A68B2F8803443F00303A2F880347E
:100220002A68637A8DF8203002F59061CDE90912D1
:10023000274A94F9083012680B921022ADF830204A
:100240000DF10E020D9222680E9262680F92D4E9AF
:100250000301A27A8DF8402001228DF8412011AAD5
:1002600082E80300227DE18A8DF8213018468DF85E
:100270004C20FFF7E5FB08AB15930DF10D0314902F
:100280000093CDF8048003AB04AA39460EA800F011
:10029000C1FB044678B99DF80C10013901F096FABB
:1002A00000F158030DEB030010F8483C3370204672
:1002B00016B0BDE8F0810C2801BF2A68B2F880347E
:1002C00043F00303A2F88034F1E700BF20260020AA
:1002D0001C260020F8B50679012E054601D8062017
:1002E000F8BD0F2E2BD80368187A40F303000722BD
:1002F000002140B200F023F92B680446187A40F33D
:1003000003100722002140B200F019F9A8B1B4FA95
:1003100084F4640929680B7A086843F3030243F301
:10032000031352B25BB29A42C8BF0124FFF774FBB9
:1003300048B9002CD3D10420D2E70124EAE70320F6
:10034000CEE70520CCE7002CFBD10C4F29683B6899
:1003500006EB460003EB80000C2201F053FA3A68EA
:100360000C2303FB062320465C72B2F880140123A1
:10037000B3400B43A2F88034B2E700BF2026002030
:1003800010B4017801290ED9084B18680C234B438F
:10039000C4180022C250C4E9012200F5906010BCCC
:1003A000102200F0D5B8002010BC70472026002095
:1003B0002DE9F04186B050238DF814300379102BCD
:1003C000074630D10368DD7B6DBB0224A846642656
:1003D000062C14D83A68535D03932A44517843EAB3
:1003E00001230393927843EA02437343CDE9033830
:1003F00063B968468DF80040FFF7C2FF0DE0CDF805
:100400000C808DF81480CDF81080F2E703AB01A8C2
:1004100001938DF80840FFF75DFF0134E4B2102C22
:1004200005F10305D4D106B0BDE8F0811FB502681F
:100430000379116851B901A88DF80430FFF7A0FFC6
:1004400078B9002040B205B05DF804FB02A8029222
:100450008DF80C30FFF73EFF0628F2D8024B185CEF
:10046000F0E70320EEE700BFE050010870B5114E41
:1004700001783268104B0C2505FB01221B68527A6B
:10048000182101FB0233044693F9021090F902008F
:1004900000F01FFB2378326861686B43D558A2686F
:1004A00000F049FA054BA289DB6B01462846BDE8FE
:1004B00070401847202600201C26002020570108E5
:1004C000074B9B56C91A431E584258414000884268
:1004D000B8BF08460528A8BF0520C0B2704700BFB6
:1004E000EF500108F0B59A42069D03DB9DF91430E8
:1004F0009A4220DD0020F0BD03EB430331F814C025
:1005000005EB830300264CFA06F7FF0707D51F7A91
:1005100007F00F0E724502DBB2EB171F0DDD01363F
:10052000102E03F10C03EED10134E4B22301DBB24F
:100530009842E1D8DEE70024F8E70120DBE78842B3
:1005400004DB9042CCBF00200120704700207047A0
:1005500010B51409B4EB111F03464FEA11100ED366
:1005600091420CD202B201F00F0133F81240012087
:1005700000FA01F124EA010123F8121010BD002055
:10058000FCE7F0B528B100EB4105012700209142BE
:1005900000D3F0BD002435F802CB234607FA04F659
:1005A00036EA0C0608BF013304F1010408BFDBB2D0
:1005B000102CF3D118440131C0B2C9B2E7E710B52D
:1005C00000B149B910BD31F8134020F81340013390
:1005D000DCB2A242F7D8F5E70023F9E782B030B5E4
:1005E000048804936AB9B3F5616F18D349F6AF254F
:1005F00042F21072AB4298BF4FF47A72944238BF05
:100600001446012C38BF01246143BDE83040C36863
:100610008B428CBF5B1A0023C36002B07047642218
:10062000ECE700002DE9F04F91B01546DDF86C8045
:1006300004939DF8683009930C46064603F0C2FB0C
:10064000684ADFF8A4B10590A8F5F633303BB3FB58
:10065000F2F3534303F5F63203F5A83303F5C07301
:100660000393182313FB05433032069208930025A9
:100670004FF0FF3A089BA34207D1002D14BF50460C
:100680004FF0FF3011B0BDE8F08FBDF97030ADF81C
:100690002C300B99CDF86C804046CDF8288003F0C3
:1006A00021FBB4F800906EB9B8F5616F5BD349F6E1
:1006B000AF2242F21073904598BF4FF47A73994578
:1006C00038BF99464B46012B38BF01230793002EB4
:1006D00052D1B9F1640F48D1A0605F46A1680EA85D
:1006E00003F022FB0F9B0093DDE90A120E9B0CA87E
:1006F00003F079FA049B0C9A0BB9099B2BB123697F
:10070000BB4202D1394B9A420DD9394BE76098452B
:1007100009D90023ADF83430069B0D990C93184687
:1007200003F0E0FAA060606800B9E760276126B1D5
:1007300003F052FBE3680344E360D4E903329342DD
:10074000059B1D996360079B88BFE2604B43E1688E
:10075000994202D20498A8B9A6B101231D44237579
:10076000EDB2183486E76423A9E7B9F57A7F0ABFAA
:10077000204F214FA060B1E7049B0BB9C4F80CB027
:100780005F46D0E700209342207506D85B1A9A4551
:1007900005F1010528BF9A46EDB2002EE1D1B9F16D
:1007A000640F164AADF8346019D049F6B023B9F594
:1007B0007A7F18BF1346904584BF039A9B180C9309
:1007C0001C9B00930CAF97E806001B9B384603F078
:1007D0000AFA97E8030003F085FA8246C1E74FF46E
:1007E0006163E8E78051010040771B007F51010001
:1007F0002FEC010080A81201002E930230EC0100C2
:100800000378032B14D1437803F00F021B098A707D
:100810004B7083788B80C27843EA02238B80037904
:10082000C3F3021203F00F03CA700B700520704768
:10083000002070472DE9F34798464379057990F9F0
:1008400007609146044690F906208A4683B190F9E4
:10085000087075B30F2A12D194F909200F2E1ED1FA
:1008600094F90A60072D24D1002F08BF012720E04A
:1008700090F90B7090F9092090F90A60E9E7A369F3
:10088000019394F915300093216994F91430207B79
:10089000FFF728FE0028E1D105F0FD05DEE794F919
:1008A0001D30B3420FDC94F91C30B342DADA05F0A4
:1008B000FB0528468AF8002089F8006088F8007057
:1008C00002B0BDE8F0871E46CCE70000024B03FAF9
:1008D00000F0B0FBF1F0704740420F004FF4FA53C4
:1008E000B3FBF0F0704730B54FF47A750C1F6A43D4
:1008F00000FB042252001EBF00F1FF341219B2FBAC
:10090000F0F2914238BF1146039A116082004843C9
:100910001CBF013040084FF47A71121A01FB1323F7
:10092000002BCABF03F2E73393FBF1F1B3FBF1F104
:10093000049B196030BD38B5400014460D46F1F7F0
:1009400069F801462846F0F7B3FF2146F0F7B0FFFB
:10095000F0F7A2FE03F0D8FCF0F77EFF40B238BDFE
:100960002DE9F74F019300231F469C461C01058A81
:100970005FFA84FE04F0F004A54206D8019B82F8D9
:1009800000C01F7003B0BDE8F08F0EEB4E054FEABC
:100990004309AD000024466836F809602641F60791
:1009A00027D5866806EB050A765916B3067836B958
:1009B000466926B136F809602641F60719D59AF836
:1009C000086090F901B046F303084FFA88F8D8455B
:1009D0000FDC46F3031676B25E450ADB9AF809602F
:1009E00006EB4608C66806EBC806367D4EB90137E9
:1009F000FFB20134102C05F10C05CCD10133DBB270
:100A0000B4E70CF101060EEB040801F80C805FFA64
:100A100086FCEEE72DE9FF4704464068DDE90C67F8
:100A20001D468A46914603F0D7F923681B1A3B609E
:100A30004FF000080123337085F80080636813B11C
:100A40002368834224D8CAF80080D4F81CC0A36964
:100A50009CF800E00393D4E9030101AB83E80300B1
:100A6000237D0093DCF80C10237A627A7046FFF73E
:100A7000D9FD334638602A46E0694946FFF770FFE2
:100A80002B782BB1C7F80080002004B0BDE8F087B8
:100A90003378002B14BF0B200C20F6E737B590F904
:100AA000002090F90250954204460FD0013A52B20C
:100AB00095420BD0A368019394F9013000936168CB
:100AC000E0782B46FFF70EFD0028EFD0104603B06C
:100AD00030BD8842B8BF08467047000051F820007A
:100AE000054B984205D0054BC31A58425841400067
:100AF00070470120704700BF90D0030020A107007D
:100B000005281FB50ED80C4B53F820300093CDE9C3
:100B100001120A4B01220021022002F069FE05B0F9
:100B20005DF804FBCDE90012054B012200210220F3
:100B300002F05EFEF3E700BF785101080F51010893
:100B40002E51010807B5054BCDE900010122002116
:100B5000022002F04DFE03B05DF804FB4A5101088B
:100B600010B5102204460021F13000F05FFE002194
:100B7000C4F814112046F022BDE8104000F056BE23
:100B800002460846102100F0A5B92DE9F0430446BD
:100B9000D0F8140185B00E46154604F2011988B349
:100BA000C0F110089045474628BF1746BAB24844DE
:100BB00000F028FED4F814313B440F2BC4F8143154
:100BC0002DD9A8452BD204F1F00304F5807113F858
:100BD000012F187C8B4282EA00021A70F7D104F1CF
:100BE000F10810224146684600F00CFE2246694694
:100BF000684600F0E9F910226946404600F002FE1E
:100C00003E44ED1B04F5807804F1F107102D09D85E
:100C1000AAB23146484600F0F5FDC4F8145105B0BB
:100C2000BDE8F08304F1F003711E13F8012F11F8F1
:100C3000010F434582EA00021A70F6D110223946AC
:100C4000684600F0DFFD22466946684600F0BCF9C0
:100C500010226946384600F0D5FD1036103DD5E724
:100C6000F0B589B00C46102200210546684600F018
:100C7000DDFD22466946684600F0A6F99DF9003080
:100C8000002B6A464FF0000143DA137812F8010F87
:100C900001315B0043EAD0130F2902F8013CF4D183
:100CA0009DF80F305B0083F08703D4F81401DBB2AA
:100CB00010288DF80F303BD104F58073694604F598
:100CC000887013F8016F11F8012B984282EA06022E
:100CD0001A70F6D104F1F00304F5807113F8012FB6
:100CE000187C8B4282EA00021A70F7D110220DEBB9
:100CF000020004F1F10100F085FD2246294604A816
:100D000000F062F910220021684600F08FFD09B062
:100D1000F0BD137812F8010F01315B0043EAD013E4
:100D20000F2902F8013CF4D19DF80F305B00BCE7BD
:100D30009DF90030002B6A464FF0000137DA137836
:100D400012F8016F01315B0043EAD6130F2902F854
:100D5000013CF4D19DF80F305B0083F08703471C02
:100D6000DBB28DF80F30102F04EB0003C0F10F063B
:100D70004FF0800288BF002600F5817083F80121C2
:100D80000021324620443E4403F072FAC4F8146154
:100D900004F58073694604F5887013F8016F11F843
:100DA000012B984282EA06021A70F6D192E7137874
:100DB00012F8016F01315B0043EAD6130F2902F8E4
:100DC000013CF4D19DF80F305B00C8E70A78037846
:100DD000534003704A784378534043708A7883784D
:100DE00053408370CA78C3785340C3700A7903793B
:100DF000534003714A794379534043718A79837927
:100E000053408371CA79C3795340C3710A7A037A14
:100E1000534003724A7A437A534043728A7A837A00
:100E200053408372CA7AC37A5340C3720A7B037BEE
:100E3000534003734A7B437B534043738A7B837BDA
:100E400053408373CA7BC37B5340C373704710B551
:100E50000B7814786340037054784B786340437088
:100E600094788B7863408370D478CB786340C37078
:100E700014790B796340037154794B796340437162
:100E800094798B7963408371D479CB796340C37152
:100E9000147A0B7A63400372547A4B7A634043723C
:100EA0008B7A947A63408372D47ACB7A6340C3722C
:100EB000147B0B7B63400373547B4B7B6340437316
:100EC000947B8B7B63408373CB7BD27B5340C37318
:100ED00010BD0000A1F11003DBB2102B2DE9F0478B
:100EE00004D8374C24FA03F3DB0705D4002382F837
:100EF000F030FF20BDE8F087531E4418A0424ED1C9
:100F000001F11C039B005FFA83F9C3F30313013B58
:100F10002C4D82F8F03001240B46D618B3FBF1F0CB
:100F200001FB103010F0FF0016F804AC16F803ECCB
:100F300016F802CC16F8017C36D115F80E8015F89B
:100F40000CE015F807C015F80A70E00900EB400046
:100F500084EA080800EBC0006400C0B2E4B2444078
:100F6000C246581AC0B212F800808AEA080A02F88B
:100F700003A01044043390F801808EEA080E86F82E
:100F800001E090F802E08CEA0E0C86F802C0C0780E
:100F9000DBB247409945F770BFD80020AAE710F8A8
:100FA000015B03F8015FA9E71829DAD9102801BF0E
:100FB00015F80AA015F80EE015F80CC0EF5DD0E7A3
:100FC00001010100905301082DE9F04FA3B092F800
:100FD000F0301D911B920193002B00F053810146CC
:100FE0001EA8FFF734FF1B9BA74CA84DA84E10333B
:100FF0000293002303939DF87C0004909DF88600E3
:101000000590205C06909DF87B000790205C08907E
:1010100004989DF881C0205C099014F80C000A9097
:101020009DF880000B909DF885009DF878809DF8D4
:101030007DE09DF882A09DF887900C909DF87A0045
:10104000029B1C9314F80A2014F8093014F80810B5
:1010500014F80E700D90205C0E909DF87F000F909C
:10106000205C10900B98205C11900C98205C1290E2
:101070009DF8840013909DF8790014909DF87E00EF
:101080001590205C16909DF883001790205C1890B6
:101090001398205C19901498205C1A9003980130E2
:1010A00003900298DDF804B0103002909DF80C0017
:1010B000834536D88DF878108DF87A2009990E9AE4
:1010C0008DF87C108DF882201199069A8DF8801089
:1010D0008DF87E201999169A8DF884108DF8862047
:1010E0000A99189A8DF87D108DF887201299109A18
:1010F0008DF87B301B9B8DF881108DF883201A9919
:10110000089A1D988DF885108DF87F201EA903EB95
:101110000B128DF87970FFF79AFE002023B0BDE81E
:10112000F08F15F808B082EA03008BEA000016F889
:101130000EB080EA0B008DF8780015F80E004B40D9
:10114000434016F80A0043408DF8793081EA0703DE
:1011500015F80A10594016F80930594016F80830A9
:101160008DF87A107A40534015F8092053408DF8D5
:101170007B30089A069B5340049AAA5C534016F8A9
:101180000C2053408DF87C30DDE908325A4015F8C8
:101190000C305340059AB25C53408DF87D30DDE948
:1011A00009325A40059BEB5C5340079AB25C5340AE
:1011B0008DF87E30069B0A9A5340049AB25C5A40DE
:1011C000079BEB5C5A408DF87F200E9B109A534092
:1011D0000B9AAA5C53400C9AB25C53408DF8803055
:1011E000DDE910325A400C9BEB5C53400D9AB25C27
:1011F00053408DF88130DDE911325A400D9BEB5C94
:1012000053400F9AB25C53408DF88230129A0E9B75
:1012100053400B9AB25C5A400F9BEB5C1C995A40AE
:101220008DF88320169B189A5340139AAA5C53405A
:10123000149AB25C53408DF88430DDE918325A407C
:10124000149BEB5C5340159AB25C53408DF885308B
:10125000DDE919325A40159BEB5C5340179AB25C9A
:1012600053408DF886301A9A169B5340139AB25CFD
:101270005340179AAA5C1EA853408DF88730FFF799
:10128000A5FDB8E6FF2049E79053010890510108F9
:101290009052010808B538B1044A05491060D822B7
:1012A00000F0B0FA002008BD0220FCE72426002050
:1012B000C05801080A4B1A6870B5002302F11805DE
:1012C00003EB03142E5D864204D1183422440A60D5
:1012D000002070BD01330B2BF2D10320F9E700BFD2
:1012E000242600202DE9F041CCB00646DDF84881E7
:1012F00017461C460D4631B3B8F1000F23D006A89F
:10130000FFF72EFC204601A9FFF7D4FF0446B0B931
:10131000019906A80131FFF733FC26B110223146AE
:1013200006A8FFF732FC3A46294606A8FFF72DFC2F
:1013300006A902A8FFF794FC029BC8F800302046DB
:101340004CB0BDE8F0810224F9E7000030B595B05B
:1013500013A90446FFF7AEFF002830D11B490C2328
:1013600003FB00F2555CA5422BD1139B187C109017
:10137000D87B0F90987B0E90587B0D90187B0C902B
:10138000D87A0B90987A0A90587A0990187A08902F
:10139000D879079098790690587905901879049033
:1013A000D8780390987802900A445B780193936808
:1013B00000930022064B1146022002F019FA15B0E4
:1013C00030BD01300B28CBD1F9E700BF085601082A
:1013D000905401080B2B10B402D810BCFFF782BF49
:1013E000032010BC704730B50D4685B01446014649
:1013F00068B103AA002000922A460390FFF772FF0B
:1014000018B90398001B18BF012005B030BD022099
:10141000FBE72DE9F0430D46BFB0144699468046E0
:1014200020B31BB311F00F0122D1F02201A800F06C
:10143000FDF920466946FFF73DFF044648B900988C
:1014400001AA10210130FFF745FD2E46AF1BFFB268
:101450001EB920463FB0BDE8F08301AA09EB0701A1
:1014600008EB0700FFF7B0FD103EEFE70224F0E7BE
:101470000524EEE7F0B5184E3468024685B00846FC
:10148000002304F1180103EB03154F5D97421ED1B1
:101490000D2A05F1190513D10023CDE90033CDE95B
:1014A00002330C2210216B46FFF7B3FF044630686D
:1014B00010226946284400F0A5F9204605B0F0BD89
:1014C00001461022601900F09DF90024F5E7013370
:1014D0000B2BD8D10324F0E72426002009B1FFF715
:1014E000C9BF022070471FB51446A0B10C2A01D114
:1014F0000B2912D10023CDE90033CDE902330A468E
:101500006B461021FFF785FF18B969462046FFF7A3
:10151000B1FF04B010BD0220FBE70320F9E7F8B5E6
:101520001E46DDE907479DF818505BB354B34FB32F
:10153000212D29D819462A46204600F063F90122B8
:10154000631C691EB018FFF764FFF8B9E37ADB0982
:101550003B70EBB96319204613F8012C13F8021CF9
:10156000120642EA014213F8041C0A4313F8031C52
:10157000012342EA0122291FFFF735FF003818BF77
:101580000120F8BD0220FCE70520FAE70720F8E774
:101590000420F6E710B5044628B1044B5B69984770
:1015A0002060002010BD0220FCE700BF205701088A
:1015B00008B5014630B1044B0822186800F022F942
:1015C000002008BD0220FCE72426002008B530B129
:1015D000044B0822196800F015F9002008BD02200C
:1015E000FCE700BF242600207FB5124E00230446EE
:1015F00002A801930D46FFF7E9FF33685B69019389
:101600006CB102AA082312F8011B41B9013B13F087
:10161000FF03F8D102A8A04702A8FFF7C9FF35B120
:10162000019B23B901A8A8473368019A5A61002099
:1016300004B070BD2426002008B5014638B1054B22
:1016400018680822104400F0DDF8002008BD0220D0
:10165000FCE700BF2426002008B538B1044B196808
:101660000822114400F0CEF8002008BD0220FCE75B
:1016700024260020034B1B6802280CBF1961596106
:10168000002070472426002041B1054B1B6802282A
:101690000CBF1B695B690B6000207047022070471C
:1016A0002426002030B58FB0002405460CA80994EC
:1016B000FFF78CFF9DF8373007939DF8363006937F
:1016C0009DF8353005939DF8343004939DF8333000
:1016D00003939DF8323002939DF8313001939DF8C9
:1016E00030300093224621461E4B022002F080F843
:1016F0000AA8FFF7B1FF9DF82F3007939DF82E3011
:1017000006939DF82D3005939DF82C3004939DF899
:101710002B3003939DF82A3002939DF829300193D2
:101720009DF82830009322460F4B2146022002F0FC
:101730005FF809A92846FFF7A7FF9DF82430039317
:101740009DF8253002939DF8263001939DF82730AF
:1017500000932246054B2146022002F049F80FB0C3
:1017600030BD00BFEC5401082A5501086855010836
:1017700008B50020FFF7EAFD0120FFF7E7FD09208B
:10178000FFF7E4FD0820FFF7E1FD0020FFF78AFFE7
:10179000002008BD10B504460B20FFF7D7FD0C2034
:1017A000FFF7D4FD0920FFF7D1FD0820FFF7CEFD9C
:1017B0000A20FFF7CBFD2046FFF774FF002010BD85
:1017C000014B1860704700BFBC0800200B4A30B5C1
:1017D00014680B4D43F2390305FB04331360091AF7
:1017E0006FF00042B3FBF2F2C2EBC27201319B1AFE
:1017F00093FBF1F201FB1233184430BDBC0800200A
:101800006D4EC64101380A44914200D1704711F82B
:10181000013B00F8013FF7E710440A44914200D130
:10182000704711F8013B00F8013DF7E702F020BDD9
:1018300030B530B10A4D01444FF0FF33814201D140
:10184000D84330BD10F8012B5340082243F3000465
:10185000013A2C4092B284EA5303002AF6D1EDE714
:101860002083B8ED01207047054B4FF400529A6277
:10187000044B1B6813B15B6803B11847704700BF86
:101880000004004828270020054B4FF480529A623C
:10189000044B1B6813B1DB6803B11847704700BFE6
:1018A00000040048282700200120704701207047CD
:1018B00001F048B901F036B910B501F019FE0E215A
:1018C000044640F61F1001F02DF92046012101F0D9
:1018D000F9FDBDE8104001F0D7BA000070B50C4E1C
:1018E00001EB40030D46B3654FF6FF71002304463C
:1018F0001A46084601F05EFB96F85600002101F0FA
:10190000E1FD29462046BDE8704001F095BA00BFD0
:101910004427002010B5044601F0AAFE01281CD17E
:1019200001F0AEFE34B11248214602F017FB104818
:1019300002F0DAFA0F4C104B00214FF48052A165EF
:101940009A6194F8560001F0BDFD63786BB16FF0B9
:101950007F40BDE8104001F053BA002340F26221FD
:101960001A46084601F026FBDCE7A0688001F0E794
:101970002C2700204427002000040048002001F00C
:10198000BFB9000008B501F0C7F80438C0B2032899
:1019900096BF024B0020185C08BD00BF1C57010811
:1019A00008B501F0BAFD033008BD01F049B901F0F6
:1019B00009B908B501F000FD00B208BD38B50D4603
:1019C000144601F05DFB284601F092FD0E2105460C
:1019D00040F61F1001F0A6F828460121074D01F03E
:1019E00071FD01F051FA4FF47A716143284602F01B
:1019F000B5FA2846BDE8384002F076BAA0270020A4
:101A000001F03EBB08B5084B002193F8560001F0E9
:101A100059FD00234FF4C0711A46084601F0CAFA76
:101A2000BDE8084001F024BA4427002010B5044660
:101A300001F01EFE01281CD101F022FE34B1124833
:101A4000214602F08BFA104802F04EFA0F4C104B70
:101A500000214FF48052A1659A6194F8560001F07C
:101A600031FD63786BB16FF07F40BDE8104001F04D
:101A70007DB9002340F262211A46084601F09AFA25
:101A8000DCE7A0688001F0E72C2700204427002035
:101A90000004004808B54FF0040001F017F9BDE854
:101AA00008400220F1F750B808B500231A4619463D
:101AB000184601F07FFABDE8084001F06DB900005A
:101AC0001D4B73B51D4D186000241D486C70C5E991
:101AD0000144AC6501F098FAAC8101F003FA2146AB
:101AE000204601F04BFC21460422012001F0FCFAC3
:101AF000144E154D4FF6FF7123462246084601F05D
:101B000059FAFFF7C7FF2246104B00944FF0FF3100
:101B1000304602F03DF90E4B009422464FF0FF3163
:101B2000284602F035F9304602F090F9284602B016
:101B3000BDE8704002F08AB9282700204427002021
:101B4000092B0108A02700202C2700206918010874
:101B5000891801080128084805D1084BC177197078
:101B60000E3001F0A7BB437D012B03D1034B8175E0
:101B70001970F5E7704700BF44270020C008002017
:101B80000D4B10B5044618735873012000F016F879
:101B90005CB134214FF4E86000F0C4FF4421BDE89B
:101BA000104040F2417000F0BDBF14214FF4E860D6
:101BB00000F0B8FF2421F2E74427002038B5114C8B
:101BC0000546207001F061FD052D04D8DFE805F021
:101BD000090B03171709032001F070FA0023637340
:101BE00038BD0020F8E7012001F068FA207B637B14
:101BF0008342F5D06073BDE83840FFF7C1BF0220D3
